:100000000C94E0370C94BA380C94BA380C94BA3883
:100010000C94BA380C94BA380C94959C0C94BA3859
:100020000C94BA380C94BA380C94BA380C94BA3888
:100030000C94BA380C94BA380C94BA380C94A99130
:100040000C94BA380C94BA380C94BA380C94BA3868
:100050000C94BA380C94BA380C94BA380C94BA3858
:100060000C94BA380C94BA380C94BA380C94BA3848
:100070000C94BA380C94BA380C94BA380C94BA3838
:100080000C94BA380C94BA380C94BA38557365721B
:10009000206167656E743A2025733C42523E0D0A1A
:1000A000004175746820696E666F3A2025733C4282
:1000B000523E0D0A00436F6F6B69653A2025733C11
:1000C00042523E0D0A00436F6E74656E742074795F
:1000D00070653A2025733C42523E0D0A004172671A
:1000E000756D656E743A2025733C42523E0D0A00D0
:1000F00055524C3A2025733C42523E0D0A004D6544
:1001000074686F643A2025733C42523E0D0A56656E
:100110007273696F6E3A20485454502F25642E250F
:10012000643C42523E0D0A436F6E74656E74206CDF
:10013000656E6774683A2025643C42523E0D0A00A1
:100140003C2F424F44593E3C2F48544D4C3E003CBE
:1001500048544D4C3E3C484541443E3C5449544C27
:10016000453E506172616D65746572733C2F5449F0
:10017000544C453E3C2F484541443E3C424F445937
:100180003E3C48313E506172616D65746572733CEE
:100190002F48313E003C2F5441424C453E3C2F42BB
:1001A0004F44593E3C2F48544D4C3E003C54523E27
:1001B0003C54443E253034583C2F54443E3C544437
:1001C0003E25733C2F54443E3C54443E25753C2F01
:1001D00054443E3C54443E25733C2F54443E3C54CE
:1001E000443E253034583C2F54443E3C54443E2534
:1001F0003034583C2F54443E3C54443E253034580F
:100200003C2F54443E3C54443E25753C2F54443EC0
:100210003C54443E25733C2F54443E3C2F54523EA4
:100220000D0A003C48544D4C3E3C484541443E3C40
:100230005449544C453E546872656164733C2F5474
:1002400049544C453E3C2F484541443E3C424F4476
:10025000593E3C48313E546872656164733C2F4896
:10026000313E0D0A3C5441424C4520424F524445D8
:10027000523E3C54523E3C54483E48616E646C656C
:100280003C2F54483E3C54483E4E616D653C2F54D3
:10029000483E3C54483E5072696F726974793C2FF5
:1002A00054483E3C54483E5374617475733C2F541B
:1002B000483E3C54483E4576656E743C42523E5141
:1002C000756575653C2F54483E3C54483E54696DF5
:1002D00065723C2F54483E3C54483E537461636BF6
:1002E0002D3C42523E706F696E7465723C2F5448CB
:1002F0003E3C54483E467265653C42523E537461F2
:10030000636B3C2F54483E3C2F54523E0D0A003C38
:100310002F5441424C453E3C2F424F44593E3C2FC6
:1003200048544D4C3E003C54523E3C54443E2530D3
:1003300034583C2F54443E3C54443E256C753C2F6D
:1003400054443E3C54443E256C753C2F54443E3C42
:1003500054443E253034583C2F54443E3C54443E93
:10036000253034583C2F54443E3C2F54523E0D0A05
:10037000003C5441424C4520424F524445523E3C81
:1003800054523E3C54483E48616E646C653C2F5468
:10039000483E3C54483E436F756E74646F776E3CC4
:1003A0002F54483E3C54483E5469636B2052656C60
:1003B0006F61643C2F54483E3C54483E43616C6C32
:1003C0006261636B3C42523E416464726573733C8C
:1003D0002F54483E3C54483E43616C6C6261636BF1
:1003E0003C42523E417267756D656E743C2F5448B5
:1003F0003E3C2F54523E0D0A003C48544D4C3E3C6E
:10040000484541443E3C5449544C453E54696D6511
:1004100072733C2F5449544C453E3C2F484541444F
:100420003E3C424F44593E3C48313E54696D6572F2
:10043000733C2F48313E0D0A00554E4B4E4F574EE0
:1004400000434C4F5345440054494D45574149548E
:10045000004C41535441434B00434C4F53494E478A
:1004600000434C4F5345574149540046494E57416C
:100470004954320046494E5741495431003C464F99
:100480004E5420434F4C4F523D2343433030303085
:100490003E45535441424C3C2F464F4E543E005330
:1004A000594E524356440053594E53454E54004CF6
:1004B000495354454E003C2F5441424C453E3C2F3D
:1004C000424F44593E3C2F48544D4C3E003C54440E
:1004D0003E25733A25753C2F54443E3C54443E001F
:1004E0003C54523E3C54443E253034583C2F5444F6
:1004F0003E3C54443E5443503C2F54443E3C5444B0
:100500003E25733A25753C2F54443E003C48544DDB
:100510004C3E3C484541443E3C5449544C453E5376
:100520006F636B6574733C2F5449544C453E3C2FAC
:10053000484541443E3C424F44593E3C48313E537D
:100540006F636B6574733C2F48313E0D0A3C544118
:10055000424C4520424F524445523E3C54523E3C50
:1005600054483E48616E646C653C2F54483E3C5490
:10057000483E547970653C2F54483E3C54483E4CAC
:100580006F63616C3C2F54483E3C54483E52656D4D
:100590006F74653C2F54483E3C54483E537461741C
:1005A00075733C2F54483E3C2F54523E0D0A002593
:1005B000733A2025733C42523E0D0A003C42523EA3
:1005C0003C42523E3C703E3C6120687265663D2272
:1005D0002E2E2F696E6465782E68746D6C223E72C3
:1005E000657475726E20746F206D61696E3C2F6149
:1005F0003E3C2F424F44593E3C2F48544D4C3E3CCC
:100600002F703E003C48544D4C3E3C424F44593EB6
:100610003C42523E3C48313E466F726D20526573FB
:10062000756C743C2F48313E3C42523E3C42523E37
:10063000003C68746D6C3E0D0A20203C6865616466
:100640003E0D0A202020203C7469746C653E4153A5
:10065000502044656D6F3C2F7469746C653E0D0AC3
:1006600020203C2F686561643E0D0A0D0A20203C65
:10067000626F6479206267636F6C6F723D222366DC
:100680006666666666223E0D0A202020203C6831A0
:100690003E4153502044656D6F3C2F68313E0D0A3A
:1006A000202020203C7461626C6520776964746846
:1006B0003D223330302220626F726465723D2231F8
:1006C000222063656C6C73706163696E673D2232D2
:1006D000222063656C6C70616464696E673D2230D2
:1006E000223E0D0A2020202020203C74723E0D0A5C
:1006F00020202020202020203C746420616C696729
:100700006E3D2263656E7465722220776964746839
:100710003D22313030223E3C623E46756E63746944
:100720006F6E3C2F623E3C2F74643E0D0A202020E9
:1007300020202020203C746420616C69676E3D227B
:1007400063656E746572222077696474683D223235
:100750003030223E3C623E526573756C743C2F62B1
:100760003E3C2F74643E0D0A2020202020203C2F88
:1007700074723E0D0A2020202020203C74723E0D11
:100780000A20202020202020203C746420776964E7
:1007900074683D22313030223E6E75745F7665722A
:1007A00073696F6E3C2F74643E0D0A202020202058
:1007B0002020203C74642077696474683D223230C4
:1007C00030223E3C256E75745F76657273696F6E7C
:1007D000253E3C2F74643E0D0A2020202020203C22
:1007E0002F74723E0D0A2020202020203C74723E7F
:1007F0000D0A20202020202020203C7464207769CE
:100800006474683D22313030223E6E75745F6D61D4
:10081000635F616464723C2F74643E0D0A20202083
:1008200020202020203C74642077696474683D2275
:10083000323030223E3C256E75745F6D61635F61BE
:10084000646472253E3C2F74643E0D0A20202020F3
:1008500020203C2F74723E2020202020200D0A20D2
:1008600020202020203C74723E0D0A2020202020D1
:100870002020203C74642077696474683D22313004
:1008800030223E6E75745F69705F616464723C2FE4
:1008900074643E0D0A20202020202020203C746417
:1008A0002077696474683D22323030223E3C256EE8
:1008B00075745F69705F61646472253E3C2F746477
:1008C0003E0D0A2020202020203C2F74723E0D0A6D
:1008D0002020202020203C74723E0D0A2020202061
:1008E000202020203C74642077696474683D2231A4
:1008F0003030223E6E75745F69705F6D61736B3C62
:100900002F74643E0D0A20202020202020203C74DB
:10091000642077696474683D22323030223E3C2581
:100920006E75745F69705F6D61736B253E3C2F74EB
:10093000643E0D0A2020202020203C2F74723E0DA2
:100940000A2020202020203C74723E0D0A20202006
:1009500020202020203C74642077696474683D2244
:10096000313030223E6E75745F67617465776179EE
:100970003C2F74643E0D0A20202020202020203CA3
:1009800074642077696474683D22323030223E3CC2
:10099000256E75745F67617465776179253E3C2FBC
:1009A00074643E0D0A2020202020203C2F74723ECB
:1009B0000D0A2020202020203C74723E0D0A2020A9
:1009C0002020202020203C74642077696474683DD6
:1009D00022313030223E7573725F646174653C2F42
:1009E00074643E0D0A20202020202020203C7464C6
:1009F0002077696474683D22323030223E3C257590
:100A000073725F64617465253E3C2F74643E0D0A09
:100A10002020202020203C2F74723E0D0A20202010
:100A20002020203C74723E0D0A202020202020200F
:100A3000203C74642077696474683D223130302230
:100A40003E7573725F74696D653C2F74643E0D0A68
:100A500020202020202020203C74642077696474AA
:100A6000683D22323030223E3C257573725F7469D6
:100A70006D65253E3C2F74643E0D0A202020202009
:100A8000203C2F74723E0D0A202020203C2F7461E0
:100A9000626C653E0D0A20203C2F626F64793E0D2A
:100AA0000A3C2F68746D6C3E6173702E6173700028
:100AB000474946383961A8003900F7FF00000000B7
:100AC000C0C0C0FEFEFEFDFDFDFCFCFCFAFAFAF91A
:100AD000F9F9F8F8F8F7F7F7F6F6F6F5F5F5F4F4AE
:100AE000F4F3F3F3F1F1F1F0F0F0EFEFEFEEEEEEFF
:100AF000EDEDEDECECECEBEBEBEAEAEAE8E8E8E74D
:100B0000E7E7E6E6E6E5E5E5E4E4E4E3E3E3E2E29D
:100B1000E2E1E1E1E0E0E0DEDEDEDDDDDDDCDCDCEB
:100B2000DBDBDBDADADAD9D9D9D8D8D8D7D7D7D638
:100B3000D6D6D5D5D5D3D3D3D2D2D2D0D0D0CECE8F
:100B4000CECDCDCDCCCCCCCBCBCBC8C8C8C7C7C7FE
:100B5000C5C5C5C4C4C4C3C3C3C2C2C2C1C1C1C068
:100B6000C0C0BFBFBFBEBEBEBDBDBDBCBCBCBABAAF
:100B7000BAB9B9B9B8B8B8B7B7B7B6B6B6B5B5B502
:100B8000B4B4B4B3B3B3B1B1B1B0B0B0AFAFAFAE52
:100B9000AEAEADADADACACACABABABA9A9A9A8A8A2
:100BA000A8A6A6A6A5A5A5A3A3A3A1A1A19F9F9F13
:100BB0009E9E9E9D9D9D9C9C9C9B9B9B9A9A9A9978
:100BC00099999898989797979696969595959494BD
:100BD000949393939292929191919090908E8E8E05
:100BE0008D8D8D8C8C8C8B8B8B8A8A8A8989898858
:100BF000888887878786868685858584848483839D
:100C0000838282828181818080807F7F7F7E7E7EE1
:100C10007D7D7D7C7C7C7B7B7B7A7A7A787878772B
:100C2000777776767675757574747473737372727C
:100C3000727171717070706E6E6E6D6D6D6B6B6BCD
:100C40006A6A6A6969696868686666666464646332
:100C500063636161615F5F5F5E5E5E5C5C5C5B5BAA
:100C60005B5A5A5A58585856565655555554545416
:100C70005353535151515050504F4F4F4E4E4E4C75
:100C80004C4C4B4B4B4A4A4A4848484747474646D4
:100C9000464444444343434141414040403E3E3E3C
:100CA0003D3D3D3C3C3C3B3B3B3A3A3A383838379B
:100CB00037373535353232323030302E2E2E2C2C1F
:100CC0002C2B2B2B2A2A2A2828282727272525259D
:100CD0002424242222222121211F1F1F1D1D1D1B10
:100CE0001B1B19191918181817171716161614148C
:100CF000141212121010100F0F0F0D0D0D0A0A0A08
:100D0000090909060606040404030303020202009B
:100D100000000000000000000000000000000000D3
:100D200000000000000000000000000000000000C3
:100D300000000000000000000000000000000000B3
:100D400000000000000000000000000000000000A3
:100D50000000000000000000000000000000000093
:100D60000000000000000000000000000000000083
:100D70000000000000000000000000000000000073
:100D80000000000000000000000000000000000063
:100D90000000000000000000000000000000000053
:100DA0000000000000000000000000000000000043
:100DB0000000000000000000000000000021F90415
:100DC00001000001002C00000000A800390000080C
:100DD000FF0003081C48B0A0C18308076AA933209C
:100DE000A1C38710234A9C48B1A2C58B0E49F4F2D7
:100DF0000502A3C78F20438A1C39F00F000040482A
:100E0000AA5CC9B2A5C511C24E527149B3A6CD950F
:100E10007C4E024073B3A7CF9F1073C43C6907A8F0
:100E2000D1A33E2F9CD209A00FD2A7504736F05035
:100E3000A312530083A26A6DD9A0A34A0544FE60A1
:100E4000C275F5A42C175B074E5D4143070F1B2F9E
:100E50004C60409036A109287E30ED52194353D999
:100E6000B2BCC4D0456A00C30E359154D9EA258C72
:100E700018B161BF74D13275E80C11130E046C7592
:100E8000D0028C255D4C47262053ECAFE945148CED
:100E900082808208B469D3C548E931E20169051C42
:100EA00067429916D900D0EBD79632DC1420A108FE
:100EB000A259BF93EB84958785819B0528000194F7
:100EC0002A794803860014CBF44939D3534008B833
:100ED000FFD43064502DEFE84F12CBA464F04A09E0
:100EE00030D25422EB3DA41500AF88CC085125FD2B
:100EF000C9443FB81752033CF8B18A7F08FE570235
:100F0000490F00514728A5F907520BC100A0840FD3
:100F100041C8A1422F081633CA193770D080661411
:100F200009E0400849F4E14A840926C84B181578BD
:100F300034400640ECB1628B007C044127DA41C1A9
:100F4000072CBC34C26282BB7012481A4EF8F0C241
:100F5000091E5800C1030F4060810729C47084181E
:100F6000817032148E5C02B04A15A94D44C0094DFF
:100F700014624B9727799400213ADDC20A9A7F15B3
:100F8000F30B2EB3B8920A2AA8A4E2CA2CB95408CB
:100F9000E79F5EFAD10408091C4440032634710718
:100FA00027F4FDE9511980462A6997C368C287185A
:100FB0005028B1C414691852DDA4695E64412EA0A2
:100FC000966AEAA93862840187A8B6EAEAAB3A6170
:100FD000FF24C01CB0D66AEBA41E1D30062DB7F648
:100FE000EA6B822081A0C52DBF166BEC5F212D41DD
:100FF000EAB1CC1A1BD2033108E1C41883803264F1
:10100000B3D89ECA52042FD4416CB6E0824A131E54
:10101000E1961B694B0FC8418CB9ECA2C9D20EBA3C
:10102000B5DBEA242E74F10930B0AA740019F2BAC3
:101030005A4C0E0219F0021B996C692A492530D2CC
:10104000AFAB7690A856A286CCB2AEB8213150850F
:101050006B0B9F2AC9030E3DF042148178C22BA06E
:1010600021E54049C6A816934703139D2803136141
:10107000D031C825B0F889E04729183231CAA6FA1C
:10108000C2450B1B2C70D1000840A0810A3510E12D
:1010900004166198F1861C71C801071A6470916981
:1010A000103460E4C11D06834A8C2EB0A0224A276A
:1010B0009548D2C8228CA4AD76249360D20929A881
:1010C000C0824BD7AFE662091D4BB400415D066D8F
:1010D000FF60462C7FCA694B2A90F491861548E040
:1010E000D0C2081D583001040E30A0400208546ED2
:1010F00039020A28D0C003114C60C1062254F9837A
:1011000012549061471F7DF0B1C752A7F2928A2016
:1011100054E8ED305415D490072F5CF6520A24831E
:10112000C001850E2858F0DC511C38026B2C813C24
:10113000F182784649C0831DA65CEB5D31B638224A
:1011400006102658A000DF0B8821FDA9C10012411E
:101150004F16B8408521E725C84A2256BCF0C0EC9E
:101160007C0FD4832BB63632414B02748003168336
:1011700044DFA22769C84107E20711100CC2569547
:1011800008934866B0053F8442173B430F316671B0
:10119000093B402105DB23A0440620041EC1AA12FE
:1011A0001A18491D12F48B510CA20B3BF800FC34A9
:1011B000D832370C0356A2B8006FBCE00ABA6947B0
:1011C00018BB68C5242C58030F4460852CBCC80B81
:1011D000F14EF6AA4314402A2E484215C040862EEE
:1011E000508109407881073218449618C0089B78CE
:1011F000951A8058C52E1AA401369843277E811E61
:1012000061104E107100C314A4C08536108213BB48
:10121000284B31AEE0C53A42C4001CF0C117029120
:101220008953ACE215B0B0D3281EB106204C910012
:101230002B1480012EC0040F32050A768C2444083A
:1012400000010C74A0031BA800032AF2802CF88272
:1012500029C1D8812447591319004E27ACB0002961
:1012600057C99214B0EE248C181F2B6729121090C6
:10127000822986601E2D7789910E6482296768080D
:101280002F87591109284227C460023197399104E8
:10129000D84127B8581033A7E990015C6128A7E02E
:1012A0000035B789901E7CAB127BE3A638077282AB
:1012B0002C02A011E11CA73823800540BC41960FE9
:1012C0000908003BE082201881085508431F1C31A3
:1012D000FF8952A8E292C0F8C52E1A063BAC280836
:1012E0001BACA0430F2E20AF8FC0248905B9D18D30
:1012F0000472B05FED44046C0806EA94354766A1B9
:10130000031CC918C522F2208624D0A0030F58C0A0
:10131000DC7A4200033C33011C30C5513088B9AC43
:101320007D491DCE18451D6204948A5649201A989D
:101330000225A8718EB5A9A31BBAA8C41CA4C0829B
:1013400008FC665E38A2A654A78AB0D3848B0291AB
:1013500030074D67C7AC73A0831A88C8804F20B38D
:10136000269850600767C88433F6E6A5AB304B1D5E
:10137000D0584520A68082051072281B321455F7DC
:10138000CAD75F09240BD310624183B40E5EDC60C0
:10139000290D208112EC108A66980D8E1CED062D09
:1013A000F870040D6488A2BEEA2BC23C23B4CE764A
:1013B000B65E0F5DD41D87321E1468E275BB4B47C5
:1013C0003586C0131238E10D93E005385285155B60
:1013D000FF75541DE2F8C523C09082811DD100869F
:1013E0001A8B67876B5588FE44402DA5C900B0A0B5
:1013F0008C39EE0E45AB8592943A228C666D755D04
:10140000E178862B06C1851734605E6A3A647310F2
:1014100072121D852085BE949D6A59FB979494E1B4
:1014200082AA241D56BADA8D5E78E20F5DC84105A6
:101430002EDBAB995475BC1B598C669A808BA55DCD
:1014400057742892060AD033DD8D6C40097490449D
:101450002926898A535CE2107600430F3AC0801A2D
:101460000D8DB30D06304664D29608740117376BA4
:10147000E12C30C0BA94CC0D514F8D5678432CE2FC
:101480000047C4001371001444A18D99EA528B6F78
:1014900005136EEB838A54A0E216D628875BB7AAA1
:1014A0000E509864A51A59CE70A3F21FE3D6B82740
:1014B000079BC80044800544AC82197DBAAE3ABA95
:1014C000090C4694E1082DA04002A692800BD0E0C2
:1014D000DF0A883025931CC12197D08BC657EEE9CF
:1014E0001D07628009AC800644A08218C01006283F
:1014F000E8C004DF35A478AD7986C0A62D1D7790AD
:101500006E9E27CD4301152C21A102566356008BF8
:10151000ED98432B65A5B4A8592534CE4A8BB85114
:101520004518C20220814BD0661DE2500294464D00
:101530006BAF0C40010D184C00149089ED3CE30397
:10154000BDAAB5B09B820111CC053887D8920B3F5C
:10155000B1002B0FFBD9FC3B7600E070B3AB30A29F
:10156000CAD0CE764FE632912E1CAB59768092329D
:10157000B54DEE8E84A52D4F90C6396CF605888C3E
:10158000BBDCF0A6221E65900B177EA3080140006D
:101590009EE3CD6F84E011039658B7367EC09A7EE5
:1015A0001B7CC43786D2196A310C3FD4AF220101AB
:1015B000003B656E6C6F676F2E6769660047494632
:1015C00038396147003900F7FF00000000C0C0C093
:1015D000FEFEFEFDFDFDFCFCFCFAFAFAF9F9F9F855
:1015E000F8F8F7F7F7F6F6F6F5F5F5F4F4F4F3F3A3
:1015F000F3F1F1F1F0F0F0EFEFEFEEEEEEEDEDEDF7
:10160000ECECECEAEAEAE8E8E8E7E7E7E6E6E6E554
:10161000E5E5E4E4E4E3E3E3E2E2E2E1E1E1E0E0A2
:10162000E0DEDEDEDDDDDDDCDCDCDBDBDBD9D9D9F9
:10163000D8D8D8D7D7D7D5D5D5D3D3D3D2D2D2CD62
:10164000CDCDCACACAC6C6C6C5C5C5C2C2C2BEBE3F
:10165000BEBDBDBDBCBCBCBABABAB9B9B9B8B8B8E0
:10166000B5B5B5B4B4B4B2B2B2B1B1B1B0B0B0AE58
:10167000AEAEACACACABABABA9A9A9A7A7A7A5A5CF
:10168000A5A4A4A4A2A2A2A1A1A1A0A0A09F9F9F43
:101690009C9C9C9B9B9B99999994949493939392D3
:1016A00092928C8C8C8B8B8B88888887878785859A
:1016B000858484848282828181818080807F7F7F13
:1016C0007D7D7D7C7C7C7B7B7B797979777777747A
:1016D00074747373737272727171716F6F6F6E6EF7
:1016E0006E6D6D6D6C6C6C6B6B6B6A6A6A69696947
:1016F0006464646363636060605F5F5F5E5E5E5CE2
:101700005C5C5B5B5B5A5A5A565656555555545459
:10171000545151514F4F4F4E4E4E4C4C4C4B4B4BE6
:101720004848484747474646464444444343434164
:1017300041414040403D3D3D373737353535323208
:10174000323030302B2B2B28282825252524242403
:101750002222221E1E1E1D1D1D19191918181814CB
:1017600014141212121010100F0F0F0D0D0D090985
:101770000906060604040403030302020200000033
:101780000000000000000000000000000000000059
:101790000000000000000000000000000000000049
:1017A0000000000000000000000000000000000039
:1017B0000000000000000000000000000000000029
:1017C0000000000000000000000000000000000019
:1017D0000000000000000000000000000000000009
:1017E00000000000000000000000000000000000F9
:1017F00000000000000000000000000000000000E9
:1018000000000000000000000000000000000000D8
:1018100000000000000000000000000000000000C8
:1018200000000000000000000000000000000000B8
:1018300000000000000000000000000000000000A8
:101840000000000000000000000000000000000098
:101850000000000000000000000000000000000088
:101860000000000000000000000000000000000078
:101870000000000000000000000000000000000068
:101880000000000000000000000000000000000058
:101890000000000000000000000000000000000048
:1018A0000000000000000000000000000000000038
:1018B0000000000000000000000000000000000028
:1018C0000000000000000000000021F904010000F9
:1018D00001002C00000000470039000008FF000351
:1018E000081C48B0A0C183050D2460D0A0410203AC
:1018F00008234A9C48D1E0820E2864004962054CC6
:101900009A356FE0BC5983C6CB93202F4620A8C8D8
:10191000B26580010F38B01852A5CD9F438D00E805
:10192000DCC9B327A4447DB4E4F070C0A551811094
:1019300040B438F2C50EA29E50A34A05A0E80C8E12
:101940000D472522D00003CA9B3E83204D1D4B9698
:10195000A7A034310A641558C0838B267116959D53
:101960004B97279A14461BA850E20650DDBF801DF6
:101970006DF950910718408F002B565C68875A8983
:101980008B23472E4302B2E4CB7F0BD98888B973EF
:101990005D22083D8B260BA9880083A3534FDDD21F
:1019A000A0A0EAD750C52C2008BBF6CE2BA705DA9D
:1019B000B60DC9C7C0DDB61BD1D00DBCF6A1120152
:1019C0008ADBAE3341F9DF447FF2B821B3850A9454
:1019D000254CA454D93266CD1C3E429C97C69583B3
:1019E00004C6090F1120461CA0A00206F1511FE9F0
:1019F0006172626556F83C076969317B2D71F18A25
:101A00009871C305FEB9A61C1F5CFC20428107012A
:101A10006748183358C02067B0F9D1850D13E436F4
:101A20006168A9E101C50B186C58516787E011C5C1
:101A30000D26B426224B912D4207163C9840C08AB1
:101A400047D5F508216C385143080ED0E8DF58859A
:101A5000ECA1C6143DA82081863EFA07092381DC4B
:101A60007146164F18A1C30A2350806492139690B2
:101A700001040914702596608629E698649669E643
:101A80009968A6A9E69A6CB6E9E69B70C629E79C18
:101A900074D669E79D78E6A9E79E7CF6E9E79F8022
:101AA000065A5140003BF561216E30B1C20381DA24
:101AB00079677986CAF7984E84A07184095766576A
:101AC0008001438144A85979CAC7C821735CA10326
:101AD000080A045A2748F8817AD2743399AF38C873
:101AE0001A489CC068A39C125594AB9122471520BC
:101AF000694451C307990AE8695A90F2FA6A8F5407
:101B00005525C81B5A08F10207A99689269ECA2A9C
:101B10004B59206F6C31840C1ECC69D8AA44259B8C
:101B20002DA8559578C8207AA4E1851340CCD041E2
:101B30000367397A2797E7E61B00113FE410430952
:101B40001B44C0009E59DACBAABE08938494A067B8
:101B50002AB925BE0923AC649249991BF1C51867BF
:101B6000ACF1C61C77ECF1C720872CF2C824976C27
:101B7000F2C928A7ACF2CA2CB7ECF2CB30C72CF3D1
:101B8000CC34D76CF3CD38E7ACF3490101003B65A9
:101B90006E7461696C2E67696600465753040D4583
:101BA00000007800055F00000FA00000193200431C
:101BB0000200000086040626BA016106BF029901F0
:101BC000000001000A006500EE000A015101103515
:101BD0004B34DB97160AA025A4031219712200E7E3
:101BE00071A52FF878B082A19A2C9916D5A4026716
:101BF000700444F9C8A4EFEA8782A0940BF428E5A6
:101C00004089880950802DBA52FB85D8DE8C0C4D56
:101C1000CA9B8C513631454004F76006F74D366556
:101C2000B80494E00BE1176A00103568C2F6F85D5D
:101C3000D98017BC4BA5E0BF21A9721BA43E6D1033
:101C4000FB8009EF200E474A6C7D100B9D20DFBD05
:101C5000401490470F2A5283D58095B8037C244FB7
:101C60005267943EF014766CA6C156A0009A5403B5
:101C7000069A6CFB800969C017A20EEA640B95F006
:101C80000998C01015F66D771060A8BABB260054ED
:101C90002128950A7600256601258988F5C02C66DD
:101CA00000AEDED896F58980259C02FA79B7C9C0C6
:101CB00014401035635AF6F9509EE5D396F6EE239C
:101CC00001584AB4BBB7EDC466EA0B72E8001035A0
:101CD000632EF6F653A646A66900957804C4654EB1
:101CE00044A1A9499A10865108403DE152B72E7C83
:101CF000378CC0155EFCF26F3D99496651812DC04D
:101D000018CA4B8CA754337A90802CEEBC372E9C8B
:101D1000B7B7710400103564F6F6F65C3628375A0A
:101D2000D300208185C635A8F1A4EE04A50025E5E1
:101D3000B431B659E5610096D00C3D248B3CAC978C
:101D40008EBF77A6FBE700B6DD8C6C606CC86C209C
:101D50006CCBEF46EBB7577B0C00007F030E000007
:101D600000010005417269616C126567696E74FF5C
:101D7000021A0000000200600F2370869B800000A2
:101D80000B8E0100FF00006503C0030142C00096F6
:101D9000060E0100020084CE1999C333377F94B038
:101DA00030680000000400FF021A00000003006019
:101DB00013A51086A17800010B8E0100FF000065BD
:101DC00003C00301A4A00096060E0200030084C60F
:101DD000C59F62CF79681438C0680000000400FF16
:101DE000021A000000040060222510869B280002D1
:101DF0000B8E0100FF00006503C00301D250009765
:101E0000060E0300040084D176C8576C85E9DB0612
:101E10008400680000000400FF021A0000000500B2
:101E200058456C62D9B28000020A8E0100FF0000A2
:101E30006503C0030190B00096060E0400050084FF
:101E4000C9C23A708E9E9158FBF0680000000400F1
:101E5000FF021A0000000600580F73030DB80000BF
:101E6000030A8E0100FF00006503C003018A000021
:101E700095060E0500060084CD0AAAA155559EBA06
:101E80005268000000040096060E0600020084C29C
:101E900090A690A5E9F77F0C00680000000400FF01
:101EA00004A401000000096106FFE320C000000057
:101EB000025801400000FFCEE1B78E76EEFFC5204C
:101EC00043AEA4E80CFFCA5863DE9D153C8826800B
:101ED0001E038024980323F4134CDC0D71803140E1
:101EE000803820616FF530624258000007842E0F61
:101EF000F4365B85D8167C3198A1C618943FBEFB9A
:101F000007DC3D010006E0D019B1067FFFE2BE29E3
:101F100071FFE320C05B269BE660019AA000D232ED
:101F200064C0A5C740B80877FFFFF8E02F8B808F0B
:101F30001C64C90740719183809AFFFFFFFC822CCB
:101F4000821648397483A441CB04109E228C453FED
:101F5000FFFFFFFFCC4899548B9F27CC8B404A371B
:101F60002491C6004E277D73E081E1A7018C58C6FD
:101F7000613046B24D382A0B74FFE320C01B1400B9
:101F8000EAC259D878021AF3DF07932D1A95554300
:101F90004B006832F5C44410D59212040FD368BCCC
:101FA000A763240D033C9A30B2F7D1F134B1ACAF42
:101FB0005962DC589A7373A02462010063FFF8B77A
:101FC000F21027C9686BEFB4000003037322791D78
:101FD000DC38B3919D342885BF9084EDD4EBD723B2
:101FE00030FFE320C02613A9A2DBF230C49673AC05
:101FF0003818B39E7F4FAF66F38B39BC4035B2EFD4
:1020000004135FE48884810AD2D4BD428201A0E631
:1020100080C77FEEF7EA4006AA89FEB118A7773B92
:1020200087C55BB9E281E10636D2E9BA531869F097
:102030000F5AAEBAAF73B3F9E5D2C99959E5741B1B
:10204000020E62A921F62448A7400097060D010060
:10205000B9DA176873884C510989DFFD2B266805AA
:102060000140540097060D0200B13B13B31B071D3E
:10207000838DE59310B60068050140540098060D65
:102080000300BD6C8AD91D17039170391E9ACC6468
:102090005068050140540097060D0400B5B96DCB9A
:1020A000C9BDFF6F7FDE8F30F868680501405400BE
:1020B00097060D0500B904F413F341EB883D7168F0
:1020C0007EB38068050140540096060D0600AD7889
:1020D000AF1C2837A8379E9DFFF4006805014054C7
:1020E00000FF040400000000000000400098060DFE
:1020F0000100BDD273A4ECE293D4527A7004EA9248
:1021000000680A0280A40097060D0200B53EE9F7B8
:10211000C6BE3F5F1F7961642260680A0280A40026
:1021200098060D0300C16609660B45A5485A5487F9
:10213000A5FF182A680A0280A40097060D0400B9BA
:10214000B566D5B26E561B9587A3463D34680A0224
:1021500080A40097060D0500BD0212042CD0473262
:1021600008E65A56B4C0680A0280A40096060D0616
:1021700000B185D85F09DAC9DAC7A721FDCC680AA2
:102180000280A400FF046C0000004002D500FFE3C1
:1021900020C03210D8CEDBEC7A506EB934D722573B
:1021A000BF5763DAA7659F569FFFFAFD6002AA0733
:1021B000A0DE0F40B232CA4355A4CDECEEC341F8C5
:1021C000AD1CF7AE5448B30D1CC0F54ED17FACDC4E
:1021D00050C38936459507B7628FF249FA40A87512
:1021E00008272C6C02EE8F76C729DAB77FEB04261E
:1021F000A4724B25B5A4400098060D0100C16441AE
:10220000644338C75518EA9C028295A068100401FF
:10221000040097060D0200B5F4EFA7C6BB215D9040
:10222000795DD416A068100401040099060D03001E
:10223000C510E68873D161FD561FD5E95345CB80A3
:1022400068100401040098060D0400BD5042A08CE3
:102250009B42C6D0B1E8AF8F128068100401040021
:1022600097060D0500BD8C1B183CD00E6A01CD5A97
:102270008DBC4068100401040097060D0600B538B7
:10228000A9C5C26A726A71E9B0FFA580681004012D
:102290000400FF0404000000000000004000980655
:1022A0000D0100C1CF11CF1338EAF51D5E9C03C2AA
:1022B000886068150541540097060D0200B94ED597
:1022C0003B71AE1257091E569902D8681505415444
:1022D0000099060D0300C561ECB0F6D15A7255A7FE
:1022E00025E92905980068150541540098060D0454
:1022F00000BDB803700C9AEAF6BABDE88E8EDB809A
:1023000068150541540097060D0500C102A902ABEE
:1023100027E975FA5D5AC6C46068150541540097EF
:10232000060D0600B5AA6D53C25E9A5E99E998FF44
:10233000D880681505415400FF04D40000008004D3
:102340000902FFE320C0491040CECFED4C400229E6
:10235000D5E7C27CE8190868E698CE4B2A1C235AB8
:102360004743B1E787D2A270A490EC2A24989F3803
:102370004E2FA5C9AA67A9F1BAE96A9A71657C7C52
:10238000D6DEB7BF7FD337FF16F67D9902590ED43C
:102390000E7E73AB7C768EC3F7552D3703E09F041A
:1023A00082C7A7ED8D9CD46F654DFFE320C06328E5
:1023B0007BE6C41F8F58024F3BDC948EB7D2070DCB
:1023C0000E550F63F92CFDB5EF6328DDF6C657B641
:1023D0002DD3FCD43AE4A8E1D0433327BDE6E5058C
:1023E00081E113ECE7BFFFFFFFF6FFFFFFFFFED722
:1023F00093C9070742761A6A83954089D841927536
:10240000FEF7809DE8B662B598B5CB6FFD7E8BEA8E
:10241000D4A5400098060D0100C51AE48D72CE4483
:1024200000488007013A9EF8681A0681A4009706C2
:102430000D0200B9A4D69371AD72D6B95E55BD0038
:1024400000681A0681A40099060D0300C5AF84D761
:10245000C2D1529E1529E1E8FFC56780681A06813E
:10246000A40098060D0400C10EAD0EAF26A349A826
:10247000D27A1B73A920681A0681A40097060D055D
:1024800000C13D9D3D9F27C9F1F27C5B04CCE06813
:102490001A0681A40097060D0600B9113444F09481
:1024A000D194D17A604002A0681A0681A400FF048A
:1024B0000400000000000000400098060D0100C567
:1024C00051E8A8F4CE4DE8C9BD17017C9B90681F68
:1024D00007C1F40097060D0200BD028A051C6B3D82
:1024E000D59EE72A6CFD10681F07C1F40099060D00
:1024F0000300C9011D40477452941529417A35F1F2
:102500004CE0681F07C1F40098060D0400C145A502
:1025100045A7268945A2517A13439B20681F07C10E
:10252000F40097060D0500C17D517D5327A771E981
:10253000DC5B42D4E0681F07C1F40097060D06007B
:10254000B955F557F0923092307A5A200F00681F33
:1025500007C1F400FF046C0000004002FD00FFE32F
:1025600020C01C102996E7EDC31002114BA3D50E15
:10257000D219D749D92888180CF6EDEAF95FB120AD
:10258000D2C157AEA9606A1AF4A38B445FAEB0D033
:10259000549AAAFFFF2F71A3C36D4E5311D4D28951
:1025A000E8B158442C250D961C50C2DB0DCFA8264F
:1025B00002176C3E5006BC756297A7DA5F4B100499
:1025C0004A4E727F8DB8400098060D0100C580F616
:1025D000C07BCE57E64AFCC701C098A868250942CF
:1025E000540097060D0200BD2F125E2C6B22159130
:1025F0000729F8FA3068250942540099060D0300AE
:10260000C92440491034507D0507D07A2C314280CE
:1026100068250942540098060D0400C175B975BBC0
:10262000266ECD9BB37A0B538DA0682509425400CA
:1026300097060D0500C1B4B9B4BB278479E11E5BD0
:102640007EDDE068250942540097060D0600B99723
:10265000F65FF08FA78FA77A54301B406825094298
:102660005400FF0404000000000000004000980631
:102670000D0100C5ADF0D6F8CE6233CC467701FE31
:1026800095D0682A0A82A40097060D0200BD5C520C
:10269000B8AC6B0C3586172984F750682A0A82A4D7
:1026A0000099060D0300C9459A5166B44E5804E5D9
:1026B000807A22D13900682A0A82A40098060D0483
:1026C00000C1A485A4872652F994BE7A0373808042
:1026D000682A0A82A40097060D0500C1EA65EA6728
:1026E000275FF5D7FD5BBEE700682A0A82A4009742
:1026F000060D0600B9DCE773B08D438D437A4E00BA
:1027000027A0682A0A82A400FF04D40000008004E5
:102710003102FFE320C03610D06AFBF840464AE0A1
:102720007D74B1404FD4EADF9AFFB0720016AA83DD
:10273000FC432875594ECA714CBB4FF08915AFB692
:102740004644C45F91DE8BB74B69EAB57B5F36A028
:10275000B7FFE0E78F195078CA21D11E2AE40E1D79
:10276000C7848281B15C481C0296B833A402C6DBE0
:10277000BF5FBA77EA00237FE0F5FFE320C04D1288
:10278000019AEBEC18C4963088229A1629BB1B5884
:102790003DCABE618EFCF8BE4935342BDADB35BA52
:1027A000B3FA2A2D6BFB052A1369682249C9960ED4
:1027B0003D81922556593329A26D4D2C24112E515D
:1027C000F3519FBEF9601ABFCFCE5DA078DA1D6EBF
:1027D00005C955D254D5AF5BEEC5C566E31191E589
:1027E0004A7F400098060D0100C5DE08EF04CE6D5B
:1027F00029CDA537023292D0682F0BC2F40097067C
:102800000D0200BD8E9B1D3C6B01D580E72910F4A5
:1028100058682F0BC2F40099060D0300C969155AB8
:1028200045744C1324C1327A19A12E80682F0BC233
:10283000F40098060D0400C1D72DD72F2634458DFE
:102840001173F76DCD00682F0BC2F40097060D05CC
:1028500000C512228911C9CE0D738358805EFA68B3
:102860002F0BC2F40097060D0600BD15522AAC22AC
:10287000C9E2C9DE91FC0CF8682F0BC2F400FF041A
:102880000400000000000000400098060D0100C98F
:10289000033B40CEF39E01D3C039C0992412683463
:1028A0000D03440097060D0200BDBD0B7A1C6AF8AB
:1028B000F57C77289AF17068340D03440099060D71
:1028C0000300C9869D61A77449D3D49D3D7A10C188
:1028D00026E068340D03440098060D0400C5018EFF
:1028E00080C7C9856E615B9CF9FB666068340D0327
:1028F000440097060D0500C52B0A9585C9C42C71A7
:102900000B18889F9268340D03440097060D06004B
:10291000BD3A82750C224722471E9074100068341D
:102920000D034400FF04D400000080042501FFE3F0
:1029300020C06010E15EEBF228C4924A1F2FD5CC74
:1029400069E72DC064EB39113DCAD685182541DFF2
:102950000AA2592DFB52255B804FD449E6C521566A
:10296000CAB3F72D5FD206AA88CA501D88E3C29C5D
:102970004910BAAFDD89AB294D264EB2C246DBE91C
:10298000294507CB9AD6DA7F55174DDFFBB7EABB4F
:10299000FAA7CADE4765FFE320C07711B8F2D7EC8B
:1029A000618672D7FE689446BD5D1F655EBD7FFF80
:1029B000EDD94DFDECDC54806B53629EBF77A006D1
:1029C000AA876F8B996F0C12B4BDA6572D8981F120
:1029D000F48662B02A6ADA184419C3236593C8BE24
:1029E0001E9972981B642A220BC441AC5AE432B17E
:1029F0008D758834AD0917068E3188593BDD40004E
:102A000098060D0100C9165A4596B3A0C7F418FDE3
:102A1000C0A6A37068390E43940097060D0200BD4E
:102A2000EBFBD7FC6AF6957B472824EE8868390EC5
:102A300043940099060D0300C9A24A6892B4478BDB
:102A40005478B57A0831200068390E43940098060E
:102A50000D0400C516D28B69C97D845F611CF62BFD
:102A600059E068390E43940097060D0500C54304EC
:102A7000A182C9B9FC6E7F1891402E68390E43942B
:102A80000097060D0600BD60FAC1FC21D061D05E42
:102A90008EE8130868390E439400FF040400000018
:102AA00000000000400098060D0100C92ACA4AB281
:102AB000B3A3BAD47759C0B122C6683F0FC3F4009C
:102AC00097060D0200C10FED0FEF1AC0756039C9EE
:102AD000EABAE4683F0FC3F40099060D0300C9BFCA
:102AE000B56FED744521E4521E73FF646180683F49
:102AF0000FC3F40098060D0400C52DD096E8C974E4
:102B0000CF5D33DCF2734D20683F0FC3F4009706AE
:102B10000D0500C55CD8AE6CC9AEEC6BBB189A60F5
:102B2000C6683F0FC3F40097060D0600BD8BEB1778
:102B3000DC216FA16F9E8D501600683F0FC3F4001B
:102B4000FF046C00000040021900FFE320C08B125C
:102B5000F296C3EC6184B675A64F3374D29CBC3731
:102B60000F12314E0673B4862B9A7F77A51480001E
:102B7000001AFFFF2E55C0A8DE433CB9B25712FD24
:102B8000CE463987472C3DD6CB9F67BEE864336A73
:102B9000D994AA0AE0BAAFD7D2CD57CEABFED56E44
:102BA000CC95D3EAEFDDED6F4F3BEA75A13A332ABE
:102BB000C806400098060D0100C93B984EE633A6B2
:102BC0009BF4D37DC0BD22386844110444009706AD
:102BD0000D0200C127D927DB1AC35561A9C9CC3A18
:102BE0002A68441104440099060D0300C9D785756D
:102BF000E17442C7742C7773EEE44C80684411048E
:102C0000440098060D0400C5418EA0C7C96C4E5BF8
:102C1000139CEEBB40E068441104440097060D0588
:102C200000C572CCB966C9A41A690698A3216C685C
:102C3000441104440097060D0600BDB4CB699C21E5
:102C40001261125E8BC418F8684411044400FF043A
:102C50000400000000000000400098060D0100C9BB
:102C60004B4552D173A9873530E5C0C8A1B068493A
:102C70001244940097060D0200C13FED3FEF1AC7C2
:102C8000D563E9C9AE396E68491244940099060DBE
:102C90000300C9ED6F7B5BF4406664066673DEC4B7
:102CA0003C0068491244940098060D0400C55488FD
:102CB000AA44C9638D58E35CEB1334E068491244BD
:102CC000940097060D0500C587C0C3E0C999086642
:102CD0004218AC220E68491244940097060D060073
:102CE000BDDECBBD9C20C1A0C19E8A281BF06849D7
:102CF00012449400FF04D400000080044D01FFE35F
:102D000020C09A158892BBEC7A524E73A2108CA404
:102D10002329D56877790849C00434E73BC0C59FAB
:102D2000C01C20419F10C8E1EB00022699623026AA
:102D300084E85409C440E9829F0887AD71E3097EA5
:102D400010D5000FB84035B250015BD1E91F1A3BD6
:102D5000A2002AAA296A89D566ADAB7283E48B49A1
:102D60008F2C2AB73186FFE320C09E184B26D7F957
:102D70004B10035C832E33C2DBBE933289CB52A748
:102D80009226E34C5981DF1C68261F69DA4A98BBFA
:102D9000720955BB362CE78762965FB91CED05CFEB
:102DA000CFB8F277511FFCACFE59D3C82E4E7D260A
:102DB000F79775AC3FF3CF7FFAD7FFEF76F3BFCA33
:102DC000D57566629F0DEB3ABAE7E3CD77EA40002E
:102DD00098060D0100C95C035700F3AC9FF593FD05
:102DE000C0D1A120684E1384E40097060D0200C1F3
:102DF0005A595A5B1AD05D682DC98EB8B2684E1305
:102E000084E40099060D0300CD0259A04B3CDEF28C
:102E1000C3DE5873CF242880684E1384E4009806DC
:102E20000D0400C56904B482C959FA567E9CE77343
:102E300028C0684E1384E40097060D0500C59E4E19
:102E4000CF27C98D09634258B5C2B4684E1384E4D4
:102E50000097060D0600C106910693082318231754
:102E6000A22607B6684E1384E400FF0404000000A5
:102E700000000000400098060D0100C9695B5A5629
:102E8000F3AF9BB5F375C0DC20AC68541505440066
:102E900097060D0200C172B172B31AD8856C41C990
:102EA0006F37F668541505440099060D0300CD0BE5
:102EB0005CA16B9CDDBDB3B7B673BF641D80685465
:102EC0001505440098060D0400C57A68BD34C95044
:102ED000BE542F9CE3CB1D20685415054400970673
:102EE0000D0500C5B12CD896C98179605E58BF0325
:102EF0006268541505440097060D0600C11C951C18
:102F0000970816081607A1BD0874685415054400F3
:102F1000FF046C00000040024100FFE320C0973036
:102F200012AAA40D9AC0006F58EFFBBD775F5E51E7
:102F30008C8A8A9756F2D55C71A63C2A121124F32A
:102F40005A34F3698B8244C81D7FD02833F960AAB4
:102F5000401165A9BFFF3541504AB9CAD76318E38C
:102F6000112FBA85AE04CF88C70C603FCE697BF9BC
:102F7000F284D8B5012BA6BEC907DA71E711DBE4EC
:102F80001B94400098060D0100C9758B5D62F3B279
:102F90009DB653B5C0E7A03A685916459400970608
:102FA0000D0200C18B198B1B1AE26D7135C94F37A9
:102FB0003A68591645940099060D0300CD136D2209
:102FC0006DACDC878390F073B00416006859164529
:102FD000940098060D0400C58AFAC57DC9474F5173
:102FE000D3DCE03B120068591645940097060D05A6
:102FF00000C5C2FAE17DC975B75D6DD8C8A4126875
:10300000591645940097060D0600C13309330B0885
:103010000C980C97A1560930685916459400FF0486
:103020000400000000000000400098060D0100C9E7
:10303000829060A433B5CBD6B979A1DF7F08685EF2
:103040001785E40097060D0200C1A5B1A5B31AF0DB
:10305000D57869C92F367A685E1785E40099060D20
:103060000300CD1BFE237FCCDB4223684473A164A5
:103070000E80685E1785E40098060D0400C59CDE8E
:10308000CE6FC93D034F40DCDCC30660685E178528
:10309000E40097060D0500C5D62AEB15C969035A49
:1030A00040D8D244BE685E1785E40097060D06003E
:1030B000C14B954B97080B380B37A0ED09E6685EBE
:1030C0001785E400FF04D400000080047501FFE3CD
:1030D00020C0310FD076FBF9C718021B717F13BDDA
:1030E000BD1BF764C23C073FFA00086D7FF9C608B4
:1030F00004DD4B4AEC8F65D8B282A77C12B3B2A331
:10310000AF30BCCF4CA8747DDD9DD9969D7EAA9B27
:103110005936F76BD7DA6A73060F2CEE2F59DF7921
:103120002241D172B1874F7896753F9D652596777C
:10313000B0A806AA0FADFFE320C04C11E9E2EFF200
:103140002884B6CC81B0464CB35A8BFD2758431C1B
:10315000A719214E2261C48A636CA8B8E5F1BF6348
:103160000E1576FF70BD84793A49407AD88094383C
:10317000756063D33B784F5A495A89572C8A2FEA96
:103180005AFF9506AA89DB1163D62E48D39D693C68
:10319000DB1259A4DC24847C958302EF5D7440002B
:1031A00098060D0100C98C6B631AF3B8D4771A8D99
:1031B000A1F37D98686318C6340097060D0200C11C
:1031C000BE29BE2B1AFE757F39C90EB5C0686318BB
:1031D000C6340099060D0300CD222224444CDA0B9C
:1031E0003B41677392440D00686318C6340098062B
:1031F0000D0400C5ABCAD5E5C933344CCD1CD9325A
:10320000FB80686318C6340097060D0500C5E5D637
:10321000F2EBC95CE4573918DC2576686318C634CC
:103220000097060D0600C162D962DB0809780977AC
:10323000A0820AA0686318C63400FF0404000000DE
:1032400000000000400098060D0100C99529654A5C
:1032500073BBDE177BC1A2097C3868681A0684003C
:1032600097060D0200C1D69DD69F1B0DDD86EDC8C9
:10327000EDB50068681A06840099060D0300CD2795
:1032800059A4EB3CD8D5631AAC7383840F8068686B
:103290001A06840098060D0400C5B9E6DCF3C929B6
:1032A0003C4A4F1CD5CAF0E068681A0684009706AD
:1032B0000D0500C5F480FA40C950A75429D8E60688
:1032C0003668681A06840097060D0600C17A757A7A
:1032D00077080B880B87A0190B5868681A068400BA
:1032E000FF046C00000040026900FFE320C05F1192
:1032F00000CACBEC62466E8337AFBB6E2E8C2B7F41
:10330000AC87FC89E256A0055F3A96B40BA0C324B3
:10331000AB9B1C2AE425C1352A319AC535EB4DE714
:10332000800D11D6B729C5BCBD7C35BD4A5986FD77
:1033300040006D7FF9F85580B200A295C240821519
:103340001119070460D868B03B2AB2019026593899
:10335000A587400098060D0100C99E7F679FF3BFB7
:103360001357E269A21A7AD0686E1B86E4009706AA
:103370000D0200C1F111F1131B22559129C8CC3463
:103380003E686E1B86E40099060D0300CD2CE5A572
:103390009CBCD790C2F2187375241180686E1B868E
:1033A000E40098060D0400C5C912E489C91E6147EE
:1033B000985CD25AE5E0686E1B86E40098060D051D
:1033C00000C9021D40877250DC1437063C09BB005F
:1033D000686E1B86E40097060D0600C19409940BE5
:1033E0000816E816E73F5A3038686E1B86E400FF7F
:1033F000040400000000000000400098060D0100D9
:10340000C9A4F0693C328435E10D7688C1E6A06834
:10341000731CC7340098060D0200C504AC8256C662
:10342000CD5F66AF722ACCE18068731CC734009907
:10343000060D0300CD303CA6079CD65E0ACBC173B7
:1034400066241A0068731CC7340098060D0400C572
:10345000D57EEABFC9142145085CCEF2DBA06873B3
:103460001CC7340098060D0500C9085D4217724D4F
:10347000BE136F863E91EC0068731CC7340097063C
:103480000D0600C1AC35AC3708214821473E7E33DC
:103490002068731CC73400FF04D400000080049D22
:1034A00001FFE320C0761518CABFEC7A526E1408EB
:1034B00097531D4703800E0CD0A051A1026F6111DC
:1034C000AC4B778A1C8B9FC8316244188A05D2594D
:1034D000C9B14516513D34FFF500002B7FF9F85373
:1034E0004819082E9C3AADCB6FCFFB4C93286491C2
:1034F00098B3F55CDA1A89B9AFD3949F77ECDDE91C
:103500005CCF699A9EC8B25ECCFFE320C07C1308F2
:1035100036D3F260C226D6E88674436FEAAB74C92C
:10352000B7EAA39D6909305AB3C942227E2043916C
:10353000236F5FD2FA00006B7FF9A917225025157F
:10354000264F2373BDB9C4904943E256D78823E779
:10355000F7B7CB934D13BA7FD4FE88DFA22BBD3FC4
:103560006573AAB976A73AD66AE46E844DACE7F9DA
:1035700098400098060D0100C9AA486A92328A3E16
:10358000A28FA68921E2A068781E07840098060D04
:103590000200C510C08860C6D2A1695072224CB129
:1035A0008068781E07840099060D0300CD32AF268F
:1035B00055ECD52E1AA5C3735764250068781E07ED
:1035C000840098060D0400C5E112F089C909C842BB
:1035D000721CCB7AD18068781E07840098060D058E
:1035E00000C90E134384F24A9B12A6C6A08C87C062
:1035F00068781E07840097060D0600C1C495C4971D
:10360000082FB82FB73DA435F868781E078400FF4F
:10361000040400000000000000400098060D0100B6
:10362000C9B0076C01F290972425C68969DE6068ED
:103630007D1F47D40098060D0200C51DBA8EDDC659
:10364000D9476CA37219AC8200687D1F47D40099DA
:10365000060D0300CD3550A6AA1CD3F0F27E1E73D2
:1036600049A43100687D1F47D40098060D0400C5A9
:10367000ED86F6C3C5FD14FE8A7320CB1D00687D60
:103680001F47D40098060D0500C91438450E32476F
:103690003B51CED6A1DC93C0687D1F47D40097066E
:1036A0000D0600C1DEC9DECB08488848873CCA3811
:1036B000B8687D1F47D400FF046C000000400291F1
:1036C00000FFE320C08A139256CFF26084B66320D5
:1036D0006A051AB13088687D24C59977529E18B260
:1036E000D39632E7BC30A2005BBFCB854D83504CF4
:1036F0002EB92E273DFCFAE4214C8728872D47B0B0
:10370000F2E7BFDBA997F37D6ECBFD1F557F5D2AE6
:1037100095B959590AAED75A6BDB55A5D16F4EAC46
:10372000A64A7CA9A6BBDBB1AA400098060D010001
:10373000C9B3256CC972968925A24689C9DB606820
:103740008320C8340098060D0200C529A094D0C675
:10375000DF776FBB72110C5380688320C8340099E7
:10376000060D0300CD35F7A6BEFCD2C7F258FE7396
:103770003AA44180688320C8340098060D0400C52F
:10378000F760FBB0C5E800F40073138AF580688326
:1037900020C8340098060D0500C918DE4637B2442B
:1037A000129104A6A328A080688320C8340097063D
:1037B0000D0600C1F779F77B085FA85FA73BE83BE0
:1037C000A8688320C83400FF040400000000000043
:1037D00000400098060D0100C9B68B6DA2F29CC78F
:1037E0002731C68A19D82068882208840098060DD7
:1037F0000200C536569B2BC6E725739272084C23F0
:103800008068882208840099060D0300CD36B5A68D
:10381000D6BCD1930A3261732C8453806888220805
:10382000840098060D0400C900FA403EB17448BAFD
:10383000245CC182B38068882208840098060D0544
:1038400000C91DDB4776F240AD502B56A480AD80F9
:1038500068882208840097060D0600C508EC847667
:10386000C2207E207DCEC18F9A688822088400FF06
:1038700004D40000008004C501FFE320C096151A9F
:1038800052DBF248C4B6AD1434EAC92870F374456B
:10389000597957D5DA592B50002DFFF9BE44C2A0F3
:1038A000363EC87F1BA7ECEDBB9AA561062990B3F5
:1038B0006A5D7FAD592E4D3CA7F9F3232877959E7D
:1038C00093A91F22F95A865CF2D8EC4C8BCB87CB9C
:1038D0001323E7FF3CA9D59979E70BD019C4A1E9D7
:1038E000B1FFE320C09C14AA9AD7EC58C4B6167056
:1038F0008450CA60448FC86D6ADFF75F9F91622170
:10390000D6BAF257FFA006AA8DB5922600527E3F86
:10391000128F8C22A5C8AC21442A1AF9772D43B7FF
:10392000EEF9276764EEDD357F4B3A0FA5511BBFDB
:10393000AB0A2DD58CAB6445BADAE7A7DAFFFB9D5D
:10394000E72CC529951E58A383400098060D010059
:10395000C9B7866DE1B2A296A8A5A68A89D6806865
:103960008D2348D40098060D0200C541F8A0FCC67E
:10397000EE4B772571FF2BF480688D2348D4009996
:10398000060D0300CD35A2A6B45CD0738A0E717308
:103990001D846A80688D2348D40098060D0400C9F0
:1039A000050F4143F16EF6B77B5CBE3AAA80688D85
:1039B0002348D40098060D0500C92170485C317B6E
:1039C000083D841A9722EA80688D2348D400970620
:1039D0000D0600C515568AABC2287A2879CE881004
:1039E00052688D2348D400FF04040000000000004A
:1039F00000400098060D0100C9B77E6DDFB2A851E6
:103A0000AA14668AF9D48068922489240098060D45
:103A10000200C54D74A6BAC6F5E57AF271F68BC5FB
:103A20008068922489240098060D0300CD33C2A635
:103A3000785C9EB317ACC5CC39120C6892248924EB
:103A40000098060D0400C908BA422EB169A1B4D08D
:103A5000DCBAEAA16068922489240098060D05006A
:103A6000C9248549217174B83A5C1A9C43200068C6
:103A7000922489240097060D0600C521BE90DFC25E
:103A800031923191CE4F910A689224892400FF042B
:103A90006C0000004002B900FFE320C0A41822928D
:103AA000D3F248C6B73942385215424A5247482BDA
:103AB0007D8BBB4D2C28B963E48AB1FFD004AAAF3B
:103AC000587DC5188221552C2525360936201C75B0
:103AD00033C4636CD8AAA21352A765A55A8D5B2A7A
:103AE00033A5C3046B7FFFAFFFFE7107C88E862A24
:103AF0009156FE9F4B6775B7902353FB6EF4446F4E
:103B0000400098060D0100C9B78E6DE3B2AE50AB10
:103B100094268B5DD30068982609840098060D02D0
:103B200000C559A2ACD1C6FF157F8A71ED4B9680B6
:103B300068982609840098060D0300CD31D9A63B6C
:103B40003C9C6B571AD5CBFE1274689826098400EA
:103B500098060D0400C90CA64329B163DA31ED1CA7
:103B6000B7A2980068982609840098060D0500C938
:103B700027D549F5716DF436FA1AA1B355806898C6
:103B80002609840097060D0600C52EE29771C23DF6
:103B9000B63DB5CE1611BA689826098400FF040414
:103BA00000000000000000400098060D0100C9B5AB
:103BB000816D6072B3D82CF6068BD1D220689D2718
:103BC00049D40097060D0200C564C0B260C20F3A26
:103BD0000F39C791AD9E689D2749D40098060D0303
:103BE00000CD2E5F25CBEC9A50F6943DCBC012EC65
:103BF000689D2749D40098060D0400C90F7943DE5B
:103C0000715E82AF415CB4728F40689D2749D400D9
:103C100098060D0500C929E24A78B167B433DA1A6B
:103C2000A6F38C80689D2749D40097060D0600C531
:103C30003B3A9D9DC2490E490DCDDC1272689D270D
:103C400049D400FF04D40000008004ED01FFE3200C
:103C5000C09E16A2A2D3EC4884B71AE30CA36D0051
:103C600007ED7FF9C9010103E86722DD15905B923A
:103C700005AF1D77162C32034A9843C9C45F739A67
:103C800052F39EACF94FDDBC938D61DD68F5FF47C3
:103C9000777FA6AFF3A39B7A36DE4F3D2AC9524801
:103CA000CBF08183C282AF74A49D4EF395DC55FDA9
:103CB00020CFEDFFF8FFE320C09E121A92DFF2182A
:103CC00044B6708087769B3B96E486249B6D731C7C
:103CD000B578A4B7228C9AD3230870A70F57251E56
:103CE000ACCEC8BBC11E90E232B2D5E8C6BB2B0732
:103CF000165EC757D3464638E93ADA879343FE92B1
:103D000052E426BF8265710BBDE7D9DB4977DFD668
:103D1000F7A28F48006D77799D14059A924000981C
:103D2000060D0100C9B2826CA0B2B9442E51068CB6
:103D30005DD1C068A2288A240097060D0200C56FD5
:103D4000AAB7D5C2212E212DC76D2CE468A2288ADE
:103D5000240098060D0300CD2A2425448C9844762F
:103D6000111DCB80936868A2288A240098060D0450
:103D700000C911E64479B1592DAC96DCB12286C058
:103D800068A2288A240098060D0500C92B704ADC19
:103D900031617EB0BF5AAC23C50068A2288A2400D6
:103DA00097060D0600C54780A3C0C2557E557DCD40
:103DB000A1132868A2288A2400FF04040000000040
:103DC000000000400098060D0100C9AF7A6BDEB21A
:103DD000BEEA2FBA868CD1D1A068A729CA740097F1
:103DE000060D0200C57B20BD90C2367E367DC748D9
:103DF0002C2868A729CA740098060D0300CD25CB8E
:103E000024B96C9628A58A29CB4313EC68A729CA44
:103E1000740098060D0400C9147B451EF1536929EE
:103E2000B49CADE27E0068A729CA740098060D050F
:103E300000C92D214B48715AD92D6C9AB193FC8041
:103E400068A729CA740097060D0600C5545CAA2EFF
:103E5000C265466545CD6593DA68A729CA7400FF37
:103E6000046C0000004002E100FFE320C0B0141A1F
:103E700096E3F218CAB63042F90D96559654756E0F
:103E800054BAAA03AB51DDAEC864E9BB0E43A3DA52
:103E90003FC2A5A99072689EA44A5722304567097F
:103EA00010EDFEFDC290A20CD09D8E93F9CCB32FE5
:103EB000CFF9C3F22FE43AA00461CD31AD2D6129D1
:103EC000F454110026060726E2BAC040055AEFFF57
:103ED0002C400098060D0100C9AAA46AA9318825C2
:103EE00044129A3597480068AC2B0AC40097060D17
:103EF0000200C58590C2C8C24A3E4A3DC7222B7007
:103F000068AC2B0AC40098060D0300CD201F2403C3
:103F1000EC943C550F15CB02148068AC2B0AC400FE
:103F200098060D0400C916154585714E1F270F9C74
:103F3000AAA275E068AC2B0AC40098060D0500C95A
:103F40002DB54B6D7154C22A611AB6E4368068AC47
:103F50002B0AC40097060D0600C56068B034C27312
:103F6000FE73FDCD2A949268AC2B0AC400FF0404B2
:103F700000000000000000400098060D0100C9A4E8
:103F8000ED693B719231C918DA38174B0068B22CD1
:103F90008B240097060D0200C58FC2C7E1C25EDE0A
:103FA0005EDDC6FDAAB668B22C8B240098060D0310
:103FB00000CD19CBA3397C9260F4983DCABF151887
:103FC00068B22C8B240098060D0400C9174C45D309
:103FD0003148DC246E1CA75A6D8068B22C8B2400FB
:103FE00098060D0500C92DD24B74B14EBC275E1A40
:103FF000BC046F8068B22C8B240097060D0600C5A8
:104000006C54B62AC283D683D5CCEE954668B22CC2
:104010008B2400FF04D400000080041502FFE3207D
:10402000C0BA156A96EFF218C4B6CE1E0B1489A258
:10403000AFD6A438F22C8328573A8DB6EE4569EAFC
:10404000A949C4A65E448C731197FF760B765FFF77
:10405000C56D3AD19AAA562E9BAA8BDDBF5FEC5A4A
:104060003BB2FDACD42EA26545FBB9FFFFFFFD14AA
:1040700010002D3FF9A1CC05A827474D0C46396CFF
:104080006A5E721F46FFE320C0BF1752AAE7F2190B
:1040900046BAADFA0DEA8D9D465D17EAF38E7BFCBC
:1040A000E567A1E2287BBFFFEA7B23FAA528FB5145
:1040B00066987AAF6E96E79AAC6AB5DBD8CA648D1B
:1040C0005200B15887AEBFA7D7ADFB7986084179BA
:1040D000C208F4805155AEFBEA3D0486D0E9FB737B
:1040E0002FABABD879F35377BB489CC724400098DB
:1040F000060D0100C99F1367C4F19C9F4E4F9A3A69
:1041000067500068B72DCB740097060D0200C59A62
:1041100056CD2BC277067705C6D62A0068B72DCBB9
:10412000740098060D0300CD134422688C907A2405
:104130001E89CA7D95B668B72DCB740098060D040C
:1041400000C91895462571432EA1975CA43265A03D
:1041500068B72DCB740098060D0500C92DF84B7E6D
:1041600031484DA426DAC174AA8068B72DCB7400FB
:1041700097060D0600C578B2BC59C2973A9739CC5C
:10418000B195FC68B72DCB7400FF0404000000005B
:10419000000000400098060D0100C997AF65EBF1E3
:1041A000A60A53051A3D27568068BC2F0BC40097FA
:1041B000060D0200C5A3F0D1F8C28D5A8D59C6B0C4
:1041C000A94A68BC2F0BC40098060D0300CD0BA3B1
:1041D00021746C5D876EC3B728DC598068BC2F0BD7
:1041E000C40098060D0400C919004640307C027CCA
:1041F000027283E9778068BC2F0BC40098060D0516
:1042000000C92D264B49B14273A139DAC6B4E60084
:1042100068BC2F0BC40097060D0600C58440C22061
:10422000C2A952A951CC7516B468BC2F0BC400FFAB
:10423000046C00000040020901FFE320C0BC1333FE
:1042400042F3F8294ADAF98F6B9E4437DAA6D6F79B
:10425000F7C7F0FDBC3BBA8E7EFF6D1E69202E674E
:10426000FFFD9FFFFA218E6022EC89FFFECBAFFF9E
:10427000314B932630488369FFFFFFFD54C02DAAC0
:10428000C020FE4DDD826236238E71DC54115663F0
:10429000791DF8F26B3CF2638E983ECC7DD93200EA
:1042A00041400098060D0100C98F8D63E371AF2373
:1042B000D791DA3FF75F0068C1304C140097060DC4
:1042C0000200C5AD3ED69FC2A482A481C68B2892AF
:1042D00068C1304C140098060D0300CD0372A06E27
:1042E0005C5A414D20A727BE5C3068C1304C140099
:1042F00098060D0400C9191046443071C471C47287
:104300007689590068C1304C140097060D0500C924
:104310002BE94AFA70796579656B30148868C13089
:104320004C140097060D0600C58F9CC7CEC2BC82F8
:10433000BC81CC37976A68C1304C1400FF0404007C
:10434000000000000000400098060D0100C9872A07
:1043500061CAB1B8895C449A42C7670068C731CC6A
:10436000740097060D0200C5B6C6DB63C2BF5ABF14
:1043700059C663A7DC68C731CC740098060D0300EA
:10438000C9F6037D80F15BB7ADDBDC9A817BA06869
:10439000C731CC740098060D0400C9191A4646B0FE
:1043A00066B866B87269E93B8068C731CC7400971B
:1043B000060D0500C92A9C4AA7306D1D6D1D6B4571
:1043C000557A68C731CC740097060D0600C59B3C32
:1043D000CD9EC2D376D375CBF8982468C731CC7400
:1043E00000FF04D400000080043D02FFE320C0CAA7
:1043F000154B46E7F239CEDAA31B77B3FBBD28C8CD
:10440000EF6FFD340985FFFFFBEEFFDFCDAA04E768
:1044100031EDF4FFB29962AFEFE804DA351A03D256
:104420002C9A7FFFFB7FF8A0B52002C534C9CA0FC4
:10443000380E66D2ED4F87CDA0D7A7493F30623BFB
:104440009B5A6DE117C7FF1F7FFBEF0F2D72F35CC7
:1044500047EB0DFFE320C0CF14D342EBF85ACEDB7D
:104460009800230FFFFFB99CEACCCC3FA1DB06925A
:10447000C732E9FF5EBF6FE448B950725A6FF76503
:10448000657EDF6FFFC6C35D40800AD759B87A20CA
:104490004035401E9ED3CCB84C82B13DB518613B2F
:1044A000388C53BE76787567CFE372E8B331BF7747
:1044B000F710E4DB362DFE7CD9C6C7400097060D09
:1044C0000100C97D8F5F63F081D481D469185DCA12
:1044D00068CC330CC40097060D0200C5BF60DFB086
:1044E000C2D822D821C63CA72668CC330CC4009879
:1044F000060D0300C9E37678DDB14FEFA7F7DC9531
:10450000D9876068CC330CC40098060D0400C91824
:1045100069461A705CB95CB9725CE91E0068CC33FC
:104520000CC40097060D0500C928804A2030620C93
:10453000620C6B59D66A68CC330CC40097060D0622
:1045400000C5A614D30AC2E8DEE8DDCBBA98DC6861
:10455000CC330CC400FF0404000000000000004045
:104560000097060D0100C9734D5CD37091D891D8A6
:1045700069259DFC68D1344D140097060D0200C5D5
:10458000C7A6E3D3C2F1AAF1A9C616267668D1342C
:104590004D140098060D0300C9CFE173F87144CFA4
:1045A00022679C9109932068D1344D140098060D20
:1045B0000400C9175D45D77052E152E1724FE9011D
:1045C0008068D1344D140097060D0500C925FE49B9
:1045D0007FB0573757376B6E576468D1344D14002E
:1045E00097060D0600C5B0A6D853C2FF4EFF4DCBAF
:1045F0007B199A68D1344D1400FF04D40000008068
:10460000043101FFE320C0D6145B42C7EC7A8ED898
:10461000139F1E5F62974AAB011484DC1E7F494AD8
:10462000CBD5AB67FEF9B1659FEBC9F722E4330444
:104630004CE24EEBA9CBB52990E5F7FFA9C2EB5DA3
:10464000AA3A8ABE64765C00235779EAD03028669D
:104650000AA1402D3CB6FA20B4D89C82BCB21761A6
:10466000B325DADDF8A17D9B7E6337FFE320C0DF51
:10467000145B46DBF25A0EDBEF9BF9518BFEAF1E4B
:104680005D81B2DA6295EA46DFD0FCE1792E9E4682
:10469000E977C98F253F534CB7842F27E02424485E
:1046A000C8A8E6841DE995EBE9CACCD0AE10D14D7F
:1046B00006A9A387D650EA0067F8A34909F08BA1A1
:1046C000F2E0C002D77970A85013A9B20654D8C737
:1046D000A740F3400097060D0100C968BF5A2FF0AC
:1046E000A24BA24B69331E2A68D6358D640097060B
:1046F0000D0200C5CFF4E7FABE1DF43BE717B497EF
:104700000068D6358D640098060D0300C9BBDD6EC8
:10471000F770734A734A7230C67D0068D6358D646F
:104720000098060D0400C9163D458F704845484560
:10473000724308E58068D6358D640097060D050044
:10474000C9235D48D7704BAF4BAF6B83985A68D67F
:10475000358D640097060D0600C5BB50DDA8BE333D
:104760006466C72CEE694068D6358D6400FF04048A
:1047700000000000000000400097060D0100C95D28
:104780003E574FB0B0C0B0C069425E6468DB36CD02
:10479000B40097060D0200C5D770EBB8BE5414A83C
:1047A000271718944068DB36CDB40098060D030037
:1047B000C9A68669A1B05FE45FE4721C66AE80683A
:1047C000DB36CDB40097060D0400C914824520AF36
:1047D0007D80FB01C8D7232868DB36CDB40097065F
:1047E0000D0500C92014480530415F415F6B9859A1
:1047F0005268DB36CDB40097060D0600C5C53EE213
:104800009FBE649CC9372BEE6C4868DB36CDB40084
:10481000FF046C00000040022500FFE320C0E81AFE
:104820003342DFF23186DA0A28D73B1D8405811E28
:1048300095771064E9A91B22F368AE20DCAF74BF42
:104840007D7B3D29D7479115DFC7ADD3BAB50ECBD8
:104850005765355369D560D9CC8654E7FF3037A307
:10486000BBDCA8E458C7483693A1070C53893F79AD
:10487000631C32800AD779BABC241C4C61394DA71D
:10488000FC7C400097060D0100C95138544E30BEE3
:1048900060BE6069521EA268E1384E140097060D92
:1048A0000200C5DE86EF43BE8B851707167691782A
:1048B00068E1384E140098060D0300C9906D641B22
:1048C000704DEF4DEF720786E08068E1384E1400BE
:1048D00097060D0400C91274449D2F6AD4D5A9C847
:1048E000A222BA68E1384E140097060D0500C91CD3
:1048F00070471C2F6EB6DD6DAEB0694068E1384E72
:10490000140097060D0600C5CED2E769BE97BD2FED
:10491000772AF06F3868E1384E1400FF0404000075
:104920000000000000400097060D0100C944DF515F
:1049300037EF98833105A5867B8868E6398E640059
:1049400097060D0200C5E578F2BCBECAB59567159D
:10495000D48EC068E6398E640097060D0300C979CD
:10496000DF5E77EF785EF0BDAF95713868E6398E1F
:10497000640097060D0400C9103C440F2F56BAADD1
:1049800075C86EA25268E6398E640097060D050060
:10499000C9189B4626EF5968B2D1AF026D3868E658
:1049A000398E640097060D0600C5D84CEC26BED3A0
:1049B00015A62729E8723068E6398E6400FF04D412
:1049C00000000080045901FFE320C0DA1B5AE2DB3B
:1049D000F24986BAA0A6080C20425325E39D0A524C
:1049E0009951C9FBCE8AA863A85946FE2E59532F68
:1049F000FDCE4E568736864674C7E1AD2E5846B476
:104A0000A644DACFCA65E8418F47973AC040024CC6
:104A1000504008213629F3D2A416769AF36BF2009F
:104A200080D01AA68FCA99150CA05C600C8544FF33
:104A3000E320C0C7173AD6E7F24144BAB36489AC61
:104A40002CE44D7679C042C051C4F1DAEA4BFFFE46
:104A5000C7F4BF35FDB3864650189581413C556576
:104A600095ACC8CA9195341D1D1C82BA6CACACAA19
:104A7000CAD991A23A3A1A394B2CB36C99680A896F
:104A8000DA1CA965B2CB2B2AB2B298934274347463
:104A900074965959599594400097060D0100C937ED
:104AA000DA4DF6AFB05B60B5A5CA7C9868EB3ACE3C
:104AB000B40097060D0200C5EBACF5D6BA09C827BD
:104AC0001C54CA304068EB3ACEB40097060D030080
:104AD000C96272589CAF5A8AB515AEE5746868EB26
:104AE0003ACEB40097060D0400C90D8C43632F44E1
:104AF000D689ADC838A1E868EB3ACEB40097060D68
:104B00000500C914474511EF468E8D1DAF51713018
:104B100068EB3ACEB40097060D0600C5E116F08B9F
:104B2000BA1498525CA399D4C068EB3ACEB400FF93
:104B3000040400000000000000400097060D010082
:104B4000C92A644A992E8CFE33F69855F70068F00E
:104B50003C0F040097060D0200C5F16EF8B7BA804D
:104B60009A025C5252258068F03C0F040097060DB3
:104B70000300C94A73529CEE7F61FD86B8C1DE8096
:104B800068F03C0F040097060D0400C90A9142A486
:104B90006E66C19B07200E860868F03C0F040097E4
:104BA000060D0500C90FA143E86E68B1A2C6BE811B
:104BB000D4E068F03C0F040097060D0600C5E97AC2
:104BC000F4BDBA86BA1ADC9F89E10068F03C0F0494
:104BD00000FF046C00000040024D00FFE320C0C550
:104BE00017221EDFF24946B6C8D0CD074720696CB0
:104BF0007943518080000E9959458148090A886798
:104C000007EE3F4D8206E9F9BFD33C6CD1A7092CD2
:104C1000C0702C2C2EC0C998B1A85451B8B0AFEBBD
:104C2000156EA1711BBE15146D42C2ACFAC55B8B2B
:104C30000B8AFE2A29A858559AB58AB71617676EA7
:104C40002A0000400097060D0100C91CA547296EE7
:104C5000B97AE5E69971FBC068F63D8F6400970666
:104C60000D0200C5F6DEFB6FB60DD06E713EC86B4F
:104C70000068F63D8F640097060D0300C932174C9B
:104C800085EE4BDD2F76B5E1EBC068F63D8F640015
:104C900097060D0400C9075D41D76E413D04F71F1B
:104CA0003E848868F63D8F640097060D0500C90AAA
:104CB000BF42AFEE42150856BFC9E52068F63D8FEA
:104CC000640097060D0600C5F18CF8C6B61310985F
:104CD000726D67B40068F63D8F6400FF0404000045
:104CE0000000000000400097060D0100C90E74434B
:104CF0009D2DBD0DE85C355A00A068FB3ECFB40089
:104D000096060D0200C5FBAEFDD7B209A099C4D22C
:104D1000A10268FB3ECFB40097060D0300C919330A
:104D2000464CED458A2C5ACB87E28068FB3ECFB4D7
:104D30000097060D0400C903CE40F3AD4052029C1B
:104D4000799A0BA068FB3ECFB40097060D0500C909
:104D5000058041602D40BA05DC81F1F56068FB3EBD
:104D6000CFB40096060D0600C5F902FC81B20C20F6
:104D7000C1C9739F9468FB3ECFB400FF04D4000008
:104D80000080048101FFE320C0C31CDB7ECFEC4820
:104D9000C6DB000000000000000000000000000072
:104DA0000000000000000000000000000000000003
:104DB00000000000000000000000000000000000F3
:104DC00000000000000000000000000000000000E3
:104DD00000000000000000000000000000000000D3
:104DE00000000000000000000000000000FFE320C1
:104DF000C0AA13389A6BEC430C4C00000000000072
:104E000000000000000000000000000000000000A2
:104E10000000000000000000000000000000000092
:104E20000000000000000000000000000000000082
:104E30000000000000000000000000000000000072
:104E40000000000000000000000000000000000062
:104E5000000000000040003F03020000000700893E
:104E6000060D01001C37EA05A00489060D02001C8E
:104E70004A9A05A00489060D03001C5FAA05A00438
:104E800089060D04001C762A05A00489060D05007C
:104E90001C845205A00489060D06001C931A05A067
:104EA00004BF03E9110000070026BE5800007D067C
:104EB000FFE320C0000000025800000000F77AC4A1
:104EC00001083800839E9EC4390431CF264D360335
:104ED00017112818B80606681113FE9E80022800D4
:104EE00081387C4050E1707DE1F28B07CB9F04302C
:104EF000FFE20706394749F87CBBFFF5430000088D
:104F0000200841A69209F8280209002C984C730445
:104F10000C60E2F62E0B1D89FFE320C05B1018E148
:104F20009001461800DB11010FC4877350F735CC90
:104F3000B26A715EFEE8C526138E44A05214F8D6FC
:104F400029E4955E87D5B99DBC7BC3A6BEB3B67A6E
:104F5000D0B8211B4359653210BAE6FEFFEDC247B7
:104F6000885CFBED0BA6D8F2CE95C6B14F4D7A3FCB
:104F7000BC4F12D163B8AAA8B28647D7EADCEF3794
:104F8000FFE320C0752A33123D75997800F7FFE3DF
:104F900054638CFE13C778BC486FE242BBC4A5DBE8
:104FA000E4859F6AFFAFFFFFFFFFFF55F9F8F6F8B2
:104FB000A7A45BEABEDEB99987CF7FEB287FF2F02A
:104FC0006C5EABFA554630D4490E6114916E6E1684
:104FD00006478A47534FEFAD53FBC38F4110E99FFC
:104FE00097FFFFC7832D2471FFE320C02714293EBC
:104FF000835DCF30008506DEF76170FAB52D08BFFE
:10500000FF6264DA2CA53C7A810040322813B9157E
:1050100087CA0AD073B02159F04240D36A7498000D
:105020001242624D5343818B9C28201527317BFF10
:10503000E8E5250DFE76977B3391400432F7F3DCEB
:10504000E145726223E74B867DCFEB9685BB2B193A
:10505000FFE320C031143A66C3FE1886B6673428D1
:105060008F9D237885110D14C41B422242B97BF316
:105070004A410403EFCFE5C85C29453FD4493705D1
:10508000BB7FFF861E4E70682DCE8B76FC4108E2FA
:105090001DEDA9F49D8D23D2A85BD4FF3BE43232F1
:1050A000F6DAEBFFD193FEC757D5AF53EDAE9A9D1D
:1050B000195D5C5A108C7700FFE320C03B11CA6E6B
:1050C000F7FE1884B6104674538B0EA81000206AA1
:1050D000340000004A11AB28C469FC28123D6AF56F
:1050E000E4B21FEE32926FE8CED9B24391BAD4E85F
:1050F00000C4229D139FAAB18CFDC2083EFA6485AC
:1051000042CA456949871B82C3960202042F8FCF8A
:10511000FA1FFFF5127B91B7484502137255D36110
:10512000FFE320C04E11A986E3FE284492E24EF62A
:105130000C02CABD97F1C7A7CF49FEFF796AF0B844
:105140008A2CD17CB7C4139C233D0B90CB633F17B3
:10515000223336434A135410507E91D792110E04D5
:105160000173C84B562A36BA95C73483F77FD91ACC
:10517000A5A98358907FD37631BB5520E246465F80
:1051800017BAC37929902E2CFFE320C06213A19295
:10519000FBFE50469218B1C7B68467B37F5B8A5650
:1051A000F4F74854AC0983106E006D740F02097B4C
:1051B000489DF451F3AAB2EE21E0A39B0BBC1A7AEE
:1051C0004BEF1641301AC60083039AB74D4DCF9767
:1051D000672000004271AAA3E4A9371CEE4744618E
:1051E00006D7B9032DA0B2B6DE2EF7FAA555D7D44F
:1051F000FFE320C06E13F996C000C086945919D3FE
:1052000045987665CC5423C5770276B8F11A5B7A57
:10521000709C0EDD511B7532115AC3ED1D57277A54
:10522000AABFB725BEF94FFFE00972A6FB9DEE535A
:10523000FFFBFB200453724D28C208E2CD184C1B23
:105240005A3764C6B2771DD3DC652D1CD65418813D
:1052500083B9087199B90956FFE320C0791500FA9E
:10526000E3FE7944717767A898810ADF9460743E01
:10527000C701836073EB18604E39C5351902B83E1B
:1052800070784DC359177D35944A6830972DBFE328
:105290003FFAC000117C440A2129D29FA622A6020F
:1052A0007DB758DFF89ACDE8ACECDFAB9BBF388E0A
:1052B0004B2AAA68C75B3AD089A58D97748C792F41
:1052C000FFE320C08014916303FE388A922A3A4F8C
:1052D000C25D0FD09D8C9A19EFAFCF73CC653AE7C2
:1052E0003D8EDD3952C3CB4E39737A7E92409DA3F9
:1052F000D55A3FA76540000043722A036244F20E6C
:10530000443F08633653EA5F7E76ADF643313AD9BF
:105310004F3223019DCC6C893B54B88F5A11123DFA
:1053200058D9FB93FFC04B23FFE320C088155AB226
:10533000E7F87886B87E9A4477488F50537047399B
:1053400092DB15BA49DF363DDE188310432106ABE8
:105350007BD01870B5251887A7EE7357BE689249A1
:1053600045DB7FFF8264F1B3220DE3BC35A2DD9201
:105370004CF7A6ED7B1E1F66875A23D245375CD9B2
:1053800067C5AE45913D6CBF90A7FFA1E5F327210E
:10539000FFE320C08D16B262EFFE6886B446896EC8
:1053A000AC18C5BB82FED8962B2D865B17B79730FD
:1053B000B5C128EF889C6127C87F3517DE7704E9DF
:1053C0009EEC000ADD004618990BE54131789AAB56
:1053D000E219CBD9076A9AEBAF5BB91EE8902FDBD5
:1053E000A6D253BDE1FAF95E1B31539ADBBE627F50
:1053F0009ED9B1B1DE3FF72CFFE320C08D15B25B23
:105400002FFE6886B7413292D768E9154F55859EC1
:10541000782F4D201860729BFEFBA172713FFFFD3B
:10542000C08F9D25F5DD166A7236FFB2DFDD70286C
:1054300006CA92200D81C68C5DC1A216B53237EC2A
:10544000C9EB746DF8F2B12CCDC4DC26C2CC45A1F9
:105450005E96513E3AE8A3CFF74CFFCD90FDDFBCFE
:10546000FFE320C09117F1C6EFF8588C959342875F
:10547000DF4B1A3BEB56E49FFE572B4E11E7EFFB39
:10548000114086D37D7589687F97C3EBF7DF60484D
:10549000B6DD93233500ACD18B8F87952D4BA99723
:1054A000EEE52D4E0FFA3A781CAF349A3EE16A1EB3
:1054B00044F10FC13BE599539F3790F7F723CDE1B6
:1054C000CDDCD2EEA494266FFFE320C08C149A7238
:1054D000FBFE3946B577B9C64F329FEF768559BF87
:1054E00099B94222165B353F3048A4148D80804222
:1054F0001B1DB903E2E99EF0CDBCF9DCCA751E2A7A
:1055000008D40E31513CA44D4DB1E948512E1CF345
:1055100023B9471334C3D23B69FFFB0A0438B3B540
:105520000552F562EF61AAAA6A281CB197B88B29C7
:10553000FFE320C094133A7F03FE3886B46B9F824A
:1055400003DF9DA10D2A04730E3579BD77FB1FFF84
:10555000FFFFBD0DA333D7D66C2F6D8044828B71B6
:10556000800160B286A580B13C88BC4DEBEF3DF474
:1055700056382E8E8E85574CB56959D18E4AB1F06A
:10558000C1C56FEB67973D99A7DD2BD5BDB7F9DE98
:105590001CB7F1064FA6B7B7FFE320C0A21949DF39
:1055A00007FE494697ADDBF98B6FBE1F31EDA73E75
:1055B000EEFCAC63202C066D11B2AD724C5A304338
:1055C0003939FE1177EB4914DB71AA88C3C8986B8F
:1055D000016622FDE9DCB5D1EE46B32310C7CE71DA
:1055E0005F3375676A582840CC45AA958A2C316C80
:1055F0002233454232F7776CEA0E7CAF967FD75C58
:10560000FFE320C09717422AF7FE414CB4DCC1FFEC
:10561000E650130D71016038488064E6AB82A2E861
:1056200069136912B8B0945C22DD49EE2C486E35DE
:1056300074002524DC964AA8C5C514EA1899D37DC0
:105640005AF843911501317AC82BD9AA1EA92E46C2
:10565000203EB2989FD93FD29B1FD59FFDC8C19DC8
:1056600024245669BC804F18FFE320C0951789FB9E
:105670000FFE4086B64AEC280D145AA089C71C2C90
:105680008130940EF621C55D7D38A0D3638CDFF6A2
:10569000CE92D4580802DC920C8BE1E711138A8A6F
:1056A0008635A36AFEA809F47426ABEB57D4EC8FB9
:1056B0003C3B99D4C150A3530C2F3CF6CC28E1308D
:1056C000A55C37E6572884C4EBC2A45C55558A40D4
:1056D000FFE320C0911531D317FE288696C4967A31
:1056E000C84F32FFBB8CC010814D43F2C81A8EA444
:1056F0000F1400A837F5B75000004A71820962AE56
:105700002C317D05AAE4E75EAEDDAEFC5999F2735B
:105710000C84EE7F104B91210466E55D994C367444
:1057200039C33386A77FFDDF5B6C35524B55505B29
:1057300030A31C8F0A098E98FFE320C09715AA2278
:10574000FFFE3886B4B0681419140F81CEB5333219
:105750006654184D2A1507AB073FFC60043E7C31A8
:1057600023A5F58330443EE026A4DFF06272D29197
:105770007E927B9CE91872244F22B8463D9594BED8
:105780008314E68C7A46CB762334BC3CC3E46216A1
:105790003333A24334E19111ACEC6FCA1F533F5530
:1057A000FFE320C09B15A9CEF7FE5886941CD4CCED
:1057B0008D1A2DDBA550B56FB7F3C87DE77FD000FC
:1057C000016884BC9335AC150476B6D516D3FDC6F6
:1057D000B216DA35BA745F7FCC2908C392D080DB69
:1057E000F46685841FC1EB99E9E670F7AE08871C63
:1057F0001A76B2C68F071931C1922CE2C45E18091D
:10580000810983F6BDF61A22FFE320C09F157A1A9C
:10581000E8E478C6B5397928B359400000027182AE
:10582000AD8564D651A59237EDAB36DE6702C9DE91
:105830007A8507318676595E6E08814D412D245D4B
:10584000A6673D521F96C4E877D5B32A8649191832
:105850007732A21C13140404E14E66B3058E8E1138
:10586000940E26B0B05C72E1CD01D4A1C68C041BAD
:10587000FFE320C0A413A9BAF3F6788694F480005D
:10588000004272008B0558E81D8D7302F34ECD9FC8
:10589000BF57B57356DAAA3D15B2B29482D48B3491
:1058A0005681D351D9349A92EE7DC8A2832EE52B2E
:1058B000BCAD444671DD4ACCEF9C94FBE5631E8E83
:1058C000EEB236BE3BE966603B7C634579FDA15A8A
:1058D000C000024B928000C4FFE320C0B01589B61F
:1058E000F7FE784694C4E705576945EE4D9DFF5F86
:1058F00074BA1913FACF108FC43A5BF491B05A1AE4
:1059000031C6BDE27159F1BBD56E210DFBF6FEF635
:105910009A32EBCC6BCC634FF67A2EE7D7F970EF67
:10592000FFC76EF310C5B6F7D473558D2DC482C36F
:10593000FB179FE46100DBA138C4E5ADFFFFDADDB2
:10594000FFE320C0B414526AF7FE6884B5A069C8AA
:1059500025BADFBDE50905183D55059EA2BCCDC79A
:10596000367115E266720C64466449D5571431A845
:1059700061B68B14AAE0CAC202862AA5D895D16B5B
:105980001A1D767430E167539BFB218DF8A9CAA2DA
:105990006AA6309CC56384925102D94799B67DA806
:1059A0006D7AF6B3A0C20D1CFFE320C0BD18A2366D
:1059B000EBFE5A0CB5132AB3E54027BA9AAFEA5862
:1059C0004926D3962A92C4EA690E0D1FB85EFAB42E
:1059D000BFABFD6BF5BDD95A8BA2559CFFFDEE54B4
:1059E00094E1C50A24D6CEE6E7B9DCED1BDDBD6F38
:1059F000D9ABC2A7F89CC3259DF6A5DF7E7EDFD07C
:105A00001A4DFA13E236564F1EAF1A6AA288EFED0E
:105A1000FFE320C0B5192ABF1FFE294ABA32F1346C
:105A2000CCD3BF7EE7CFE911C0D0B0B87E3B0B57D7
:105A30005350B6280A0000DB758000E4A1A240D3D1
:105A400009C68A4FA36CECD2294CF3B0F8F2ADEE44
:105A5000B47DD58F565C229EFC2193CF953BD0051B
:105A6000E655EAD397ED53F634A5D5119C846E65BF
:105A700068BCC9C72565B59AFFE320C0AB19FAB366
:105A800003FE48CCBAEB454DC29313717211B16558
:105A90000E260F6FFB65148FDD6A2F086055A6A8D0
:105AA000AF2536DFFF9D2AB5FFFBA7FF6024A2D3F9
:105AB000922A88C65010D47A3528BA6BC8824CEA2C
:105AC00053E57E656AB1AC0C6C10554858D8445CFF
:105AD0008A84EE4164214E1428F118882A9682CBDC
:105AE000FFE320C09E1A99CED7FE408C95216B49CA
:105AF000AA34260548703A3D00C345478DAAAEEF4B
:105B00001640158F8790E40FE553A057A86D3824F1
:105B1000BB57D5E291428555E2B6A9BFCE5FEFE80B
:105B20007A2A532CE860DF03A97B7014F0FD2AEB7E
:105B3000A2513C28C41B333FBF4A4434131A10926D
:105B4000D431AC506909CBDEFFE320C08E14B0DE47
:105B5000F3FE18446ED3BAD97F3263DB9B533FFF09
:105B6000AEFB115A74ECF32FCAAB0988CE9C3A975E
:105B70001F74B33FCB2424A4DC924B0AC4E826A7AD
:105B8000063FE1F7ACB532F51D54EB320D62C8A506
:105B90008B30AAA0E0B141D93F0ADC39108425E15D
:105BA000F953E297FAA41C34027040F3FD6F3D9D57
:105BB000FFE320C09616F2BB03FE28C6BAFDCBF564
:105BC000D6B9577F999DB4AE42857D566313276041
:105BD0006900139A83E2D43081C5FBFA5EFDD5AC2F
:105BE00000A49371485350242568480461D8F4B93F
:105BF000EB477644771B6B9562A341514ADCD52570
:105C0000D83A67309E8A96708CE0B232A59C9D6C23
:105C1000A083E2AB0B614543FFE320C09517327EC2
:105C2000E3FE1946B60CB40198C0FC9D8CF0C4ACE0
:105C3000A8CCB91913C22693E5552BBD5E7AFCB0EA
:105C4000DD051810A1C1758556C9E239946A36641C
:105C50005D02E576282522C476752AC233898BD861
:105C600014DD1F1AF914E60E211B469354F570310A
:105C70004B5617123CA09E22DEB73187C19BB4D28F
:105C8000FFE320C09319F28EC7FC4146B6242CEFE7
:105C900051B2B484C76838EE09AAD2EE6AEE66AE95
:105CA000C9B9AE82C29CA62124532C99FC6A0B5719
:105CB0002AE13159CBF91A8EA9BE7BEDFFFEBFA8B0
:105CC0008BFFEEBD4069C805DB7FDFE5AA8C3A2477
:105CD00031757477FFE57871780543221D22E31E44
:105CE000A1A769CB4BF43EA1FFE320C0861899DA47
:105CF000CFFE385097F4CBD7FFFF2732F766E1BECF
:105D00001467E9268CDFB15D5A31B5C99C58220A67
:105D1000141C0D1CB68FB1DD4CA9A0E6F53844C9A2
:105D2000A0AB56D8DFEA493605BB7FD5E2D0242E9A
:105D30008E120D2B9DFFEFF7B642335E4605570CD2
:105D40006B2E759C8929CB0620A5205268AA45DFB9
:105D5000FFE320C07E15028EDFFE4046B65C9CE964
:105D6000867699D6591451291911B7CD4E899D2E91
:105D700017CCE2F202557E64CC45FED49FAB51BEF7
:105D800067DD1851014526C98BD475F56FD69FA0E4
:105D900024A0C39AD52B66A260D0F171506997CE2A
:105DA000FFFBEA7EC784762A02A589C58ADD61F8F1
:105DB00051549490ED513BC8FFE320C0851732B297
:105DC000CBFE2886BAC0CF8AE4517A90CD1B96D2FA
:105DD000AA8BEF3E1AAB82AA7491A19F57DBFA6D92
:105DE000AA40D2C635E66AB4AA9336E47C8C7F8892
:105DF0005F6DE689EC01D1FFFD76F1505A4E7811C6
:105E00006F177A40692728DB7FFDE19584859058DC
:105E1000C0D9593A72FD21D95AF98D5431667F6A39
:105E2000FFE320C0831992A6A7FE38C6BB9CD5CE3F
:105E30004F949483011D0428F97455FF3AA6EB0F83
:105E4000E3D24A5C32510059BAC32368FECE7BA824
:105E500092A022431C6301294FE33102154123C95B
:105E60007ED221268342C1D3CA1299F06DEC42E959
:105E7000469950006BFFF035C30A8298F5523F9C5B
:105E80003964E2C98A41094BFFE320C07718626A8E
:105E9000A7FE2886B6F0CC33098509B29FB37555A5
:105EA0007EAAF5674BE1EA19A7FF4E46F52D7D5412
:105EB000C830A63C31E67386DCF0CA419AC752DB93
:105EC000C2A9513566573F5C2A9C3CDBCE804F5AB5
:105ED0005901DEC15703596326139A058938F830F2
:105EE0000E464DA906110A84BA2BF3AE23D4567977
:105EF000FFE320C07016C29E63F61846B6FA88C645
:105F00000F712CEAD3ACB01424157C78C0A05424B3
:105F10001D0D068F42A13705425962AC0A01460F9A
:105F20000100A1202B8243C055FFFF09288D40505E
:105F30000000000000000000000000000000000061
:105F40000000000000000000000000000000000051
:105F50000000000000000000FFE320C07011E049D5
:105F6000FC0030462400000000000000000000009B
:105F70000000000000000020002000200020002081
:105F80000020002000200020002000200020002011
:105F90000020002000200020002000200020002001
:105FA00000200020002000200020002000200020F1
:105FB00000200020002000200020002000200020E1
:105FC000FFE320C083000002580000000000200012
:105FD00020002000200020002000200020002000C1
:105FE00020002000200020002000200020002000B1
:105FF00020002000200020002000200020002000A1
:106000002000200020002000200020002000200090
:106010002000200020002000200020002000200080
:106020002000200020002000FFE320C0DE0000024E
:106030005800000000200020002000200020002048
:106040000020002000200020002000200020002050
:106050000020002000200020002000200020002040
:106060000020002000200020002000200020002030
:106070000020002000200020002000200020002020
:106080000020002000200020002000200020000030
:10609000FF0303000000070000FF040400000000ED
:1060A00000000040000000666C6173682F65676E39
:1060B0006974652E737766003C48544D4C3E0D0A5A
:1060C0003C484541443E0D0A3C5449544C453E65CC
:1060D000676E6974653C2F5449544C453E0D0A3C2B
:1060E0002F484541443E0D0A3C424F4459206267C7
:1060F000636F6C6F723D2223303030303030223E7F
:106100000D0A3C212D2D2055524C277320757365A7
:106110006420696E20746865206D6F7669652D2D29
:106120003E0D0A3C212D2D20746578742075736511
:106130006420696E20746865206D6F7669652D2D09
:106140003E0D0A3C212D2D652067206E20692074AC
:10615000206520652067206E2069207420652065F9
:106160002067206E20692074206520652067206EDE
:1061700020692074206520652067206E20692074C6
:10618000206520652067206E2069207420652065C9
:106190002067206E20692074206520652067206EAE
:1061A00020692074206520652067206E2069207496
:1061B000206520652067206E206920742065206599
:1061C0002067206E20692074206520652067206E7E
:1061D00020692074206520652067206E2069207466
:1061E000206520652067206E206920742065206569
:1061F0002067206E20692074206520652067206E4E
:1062000020692074206520652067206E2069207435
:10621000206520652067206E206920742065206538
:106220002067206E20692074206520652067206E1D
:1062300020692074206520652067206E2069207405
:10624000206520652067206E206920742065206508
:106250002067206E20692074206520652067206EED
:1062600020692074206520652067206E20692074D5
:10627000206520652067206E2069207420652065D8
:106280002067206E20692074206520652067206EBD
:1062900020692074206520652067206E20692074A5
:1062A000206520652067206E2069207420652065A8
:1062B0002067206E20692074206520652067206E8D
:1062C00020692074206520652067206E2069207475
:1062D000206520652067206E206920742065206578
:1062E0002067206E20692074206520652067206E5D
:1062F00020692074206520652067206E2069207445
:10630000206520652067206E206920742065206547
:106310002067206E20692074206520652067206E2C
:1063200020692074206520652067206E2069207414
:10633000206520652067206E206920742065206517
:106340002067206E20692074206520652067206EFC
:1063500020692074206520652067206E20692074E4
:10636000206520652067206E2069207420652065E7
:106370002067206E20692074206520652067206ECC
:1063800020692074206520652067206E20692074B4
:10639000206520652067206E206920742065202DEF
:1063A0002D3E3C4F424A45435420636C61737369F0
:1063B000643D22636C7369643A4432374344423625
:1063C000452D414536442D313163662D39364238ED
:1063D0002D343434353533353430303030220D0AF5
:1063E00020636F6465626173653D22687474703AFE
:1063F0002F2F6163746976652E6D6163726F6D65B1
:106400006469612E636F6D2F666C617368322F63F0
:106410006162732F7377666C6173682E63616223A8
:1064200076657273696F6E3D342C302C302C3022BF
:106430000D0A2049443D65676E69746520574944DB
:1064400054483D353530204845494748543D34305F
:10645000303E0D0A203C504152414D204E414D45A9
:106460003D6D6F7669652056414C55453D22656707
:106470006E6974652E737766223E203C504152410E
:106480004D204E414D453D7175616C6974792056C2
:10649000414C55453D686967683E203C504152413A
:1064A0004D204E414D453D6267636F6C6F722056C3
:1064B000414C55453D233030303030303E203C4556
:1064C0004D424544207372633D2265676E69746571
:1064D0002E73776622207175616C6974793D6869E5
:1064E0006768206267636F6C6F723D2330303030B5
:1064F0003030202057494454483D353530204845F8
:10650000494748543D34303020545950453D22616C
:1065100070706C69636174696F6E2F782D73686F2A
:10652000636B776176652D666C6173682220504CD1
:106530005547494E53504147453D22687474703A5F
:106540002F2F7777772E6D6163726F6D6564696148
:106550002E636F6D2F73686F636B776176652F6441
:106560006F776E6C6F61642F696E6465782E6367F8
:10657000693F50315F50726F645F56657273696F27
:106580006E3D53686F636B77617665466C617368C7
:10659000223E3C2F454D4245443E0D0A3C2F4F4282
:1065A0004A4543543E0D0A3C2F424F44593E0D0A82
:1065B0003C2F48544D4C3E0D0A666C6173682F6643
:1065C0006C6173682E68746D6C003C48544D4C3E91
:1065D0000D0A3C484541443E0D0A3C5449544C4543
:1065E0003E466F726D3C2F5449544C453E0D0A3C5B
:1065F0002F484541443E0D0A3C666F726D20616331
:1066000074696F6E3D226367692D62696E2F666FD4
:10661000726D2E63676922206D6574686F643D2218
:106620006765742263656C6C7370616464696E671E
:106630003D223622206267636F6C6F723D222338E1
:106640003038303830223E0D0A3C68313E466F7299
:106650006D3C2F68313E3C42523E0D0A3C746162F3
:106660006C6520206267636F6C6F723D222345303A
:106670004530453022206865696768743D223133B2
:1066800030222077696474683D22343536223E0D0D
:106690000A3C74723E0D0A3C544420686569676880
:1066A000743D223239222077696474683D2238367D
:1066B000223E20506172616D313A3C2F54443E0DB0
:1066C0000A3C5444206865696768743D2232392267
:1066D0002077696474683D22333630223E3C696E0F
:1066E00070757420747970653D2274657874222009
:1066F0006E616D653D225431222073697A653D22B9
:106700003438222076616C75653D22303034392270
:106710003E3C2F54443E0D0A3C2F74723E0D0A3C01
:1067200074723E0D0A3C5444206865696768743D84
:10673000223332222077696474683D223836223E43
:1067400020506172616D323A3C2F54443E0D0A3C38
:106750005444206865696768743D2233322220778B
:10676000696474683D22333630223E3C696E707530
:106770007420747970653D227465787422206E618E
:106780006D653D225432222073697A653D2236229E
:106790002076616C75653D2231223E3C2F54443E8B
:1067A0000D0A3C2F74723E0D0A3C74723E0D0A3C79
:1067B0005444206865696768743D22383422207724
:1067C000696474683D223836223E506172616D33CF
:1067D0003C2F54443E0D0A3C544420686569676868
:1067E000743D223834222077696474683D22333640
:1067F00030223E3C544558544152454120747970F2
:10680000653D227465787422206E616D653D225469
:1068100065787422206D61786C656E6774683D22BE
:106820003136302220636F6C733D343120726F77C4
:10683000733D353E3C2F74657874617265613E3CF2
:106840002F54443E0D0A3C2F74723E0D0A3C5444B2
:1068500020636F6C7370616E3D3220616C69676E8E
:106860003D6D6964646C65206865696768743D2284
:106870003237222077696474683D22343530222013
:106880003E3C696E7075742074797065203D2022DD
:106890007375626D697422202076616C75653D2286
:1068A00073656E64222073697A653D2238223E0D3D
:1068B0000A093C696E7075742074797065203D20FA
:1068C000227265736574222076616C75653D226362
:1068D000616E63656C222073697A653D2238223EC1
:1068E0003C2F54443E0D0A3C2F74723E0D0A3C2F3F
:1068F0007461626C653E0D0A3C703E3C61206872BA
:1069000065663D222E2E2F696E6465782E68746D43
:106910006C223E72657475726E20746F206D6169B1
:106920006E3C2F613E0D0A3C2F666F726D3E0D0A64
:106930000D0A3C2F48544D4C3E0D0A666F726D2E69
:1069400068746D6C00416C6C6F77656420696E6370
:106950006C75646520636F6D6D616E647320617228
:10696000653A3C703E0D0A3C636F64653E266C746C
:106970003B212D2D23696E636C75646520766972E9
:106980007475616C3D2671756F743B2F6E657773FE
:106990002F6E6577732E68746D2671756F743B204A
:1069A0002D2D2667743B3C2F636F64653E3C6272FD
:1069B0003E0D0A3C636F64653E266C743B212D2DB1
:1069C00023696E636C7564652066696C653D26712C
:1069D000756F743B55524F4D3A66696C652E7478ED
:1069E000742671756F743B202D2D2667743B3C2FE8
:1069F000636F64653E3C62723E0D0A3C636F646582
:106A00003E266C743B212D2D2365786563206367DA
:106A1000693D2671756F743B2F6367692D62696EDE
:106A20002F746573742E6367693F706172616D3D89
:106A300076616C75652671756F743B202D2D266708
:106A4000743B3C2F636F64653E3C62723E0D0A0DE1
:106A50000A696E636C7564652E696E63003C6874C8
:106A60006D6C3E0D0A3C686561643E0D0A3C2F6802
:106A70006561643E0D0A3C626F64793E0D0A0D0A41
:106A80003C696D67207372633D22656E6C6F676F42
:106A90002E676966223E3C696D67207372633D22F2
:106AA000656E7461696C2E676966223E3C703E0DAE
:106AB0000A0D0A3C68313E57656C636F6D65207442
:106AC0006F2045746865726E757420485454503C4C
:106AD0002F68313E0D0A0D0A3C6120687265663DE3
:106AE00022666C6173682F666C6173682E68746DC2
:106AF0006C223E466C6173682064656D6F3C2F614B
:106B00003E3C703E0D0A3C6120687265663D227312
:106B100073692E7368746D6C223E5365727665726C
:106B2000207369646520696E636C756465206465B3
:106B30006D6F3C2F613E3C703E0D0A3C61206872D7
:106B400065663D226173702E617370223E41535021
:106B50002064656D6F3C2F613E3C703E0D0A3C68C1
:106B6000323E4347492053616D706C65733C2F681A
:106B7000323E0D0A0D0A4C6F67696E3A20726F6FD4
:106B8000743C62723E0D0A50617373776F72643A9F
:106B900020726F6F743C703E0D0A0D0A3C612068D4
:106BA0007265663D226367692D62696E2F74657335
:106BB000742E6367693F45746865726E7574223E12
:106BC000506172616D657465722064656D6F3C2FF4
:106BD000613E3C703E0D0A3C6120687265663D2254
:106BE000666F726D2E68746D6C223E466F726D20FA
:106BF00064656D6F3C2F613E3C703E0D0A3C612028
:106C0000687265663D226367692D62696E2F7468DC
:106C100072656164732E636769223E5468726561B0
:106C200064206C6973743C2F613E3C703E0D0A3CDD
:106C30006120687265663D226367692D62696E2F07
:106C400074696D6572732E636769223E54696D6560
:106C500072206C6973743C2F613E3C703E0D0A3C9F
:106C60006120687265663D226367692D62696E2FD7
:106C7000736F636B6574732E636769223E536F6332
:106C80006B6574206C6973743C2F613E3C703E0DE3
:106C90000A0D0A3C2F626F64793E0D0A3C2F68741E
:106CA0006D6C3E0D0A696E6465782E68746D6C00BB
:106CB0003C68746D6C3E0D0A3C686561643E0D0A6B
:106CC0003C2F686561643E0D0A3C626F64793E0D3D
:106CD0000A0D0A3C696D67207372633D22656E6C14
:106CE0006F676F2E676966223E3C696D672073721D
:106CF000633D22656E7461696C2E676966223E3C55
:106D0000703E0D0A0D0A3C68313E5365727665721D
:106D1000207369646520696E636C756465206465C1
:106D20006D6F3C2F68313E0D0A0D0A2D2D2D2D2D36
:106D300020496E636C7564656420706172742073A1
:106D400074617274202D2D2D2D2D3C62723E0D0A22
:106D50003C212D2D2023696E636C75646520766956
:106D6000727475616C3D222F696E636C7564652E5B
:106D7000696E6322202D2D3E0D0A2D2D2D2D2D20E7
:106D8000496E636C75646564207061727420656E11
:106D9000642020202D2D2D2D2D3C62723E0D0A0DDC
:106DA0000A3C2F626F64793E0D0A3C2F68746D6C4B
:106DB0003E0D0A7373692E7368746D6C00FFFFFFDC
:106DC000FFFFFFFFFFFFFFFF3EFFFFFF3F343536B2
:106DD0003738393A3B3C3DFFFFFFFFFFFFFF000123
:106DE00002030405060708090A0B0C0D0E0F10110B
:106DF0001213141516171819FFFFFFFFFFFF1A1BB8
:106E00001C1D1E1F202122232425262728292A2B4A
:106E10002C2D2E2F30313233FFFFFFFFFF4854540B
:106E2000502F25642E25642025642025730D0A53D8
:106E300065727665723A2045746865726E75742065
:106E400025730D0A00436F6E6E656374696F6E3A49
:106E500020636C6F73650D0A0D0A00436F6E7465D5
:106E60006E742D4C656E6774683A20256C640D0A4B
:106E700000436F6E74656E742D547970653A2025E9
:106E8000730D0A005757572D41757468656E746904
:106E9000636174653A204261736963207265616C55
:106EA0006D3D222573220D0A003C48544D4C3E3C5A
:106EB000484541443E3C5449544C453E25642025B8
:106EC000733C2F5449544C453E3C2F484541443E69
:106ED0003C424F44593E25642025733C2F424F4489
:106EE000593E3C2F48544D4C3E00343034204E6FB8
:106EF0007420666F756E643A2025730A003430344E
:106F0000204E6F7420666F756E643A2025730A00F8
:106F100035303020496E7465726E616C2065727216
:106F20006F720A0035303020496E7465726E616C84
:106F3000206572726F720A0035303020496E7465B8
:106F4000726E616C206572726F720A00353030208B
:106F5000496E7465726E616C206572726F720A00A0
:106F600035303020496E7465726E616C20657272C6
:106F70006F720A0035303020496E7465726E616C34
:106F8000206572726F720A0035303020496E746568
:106F9000726E616C206572726F720A00343030203C
:106FA0004265616420726571756573740A00FFFF44
:106FB000FF30FFFFFFFFFFFFFFFFFFFFFFFFFFFFB0
:106FC000E5E5F0E080EC8083A5E3B0E0E5E3F0E008
:106FD000808180688C93A4E3B0E0E4E3F0E08081FA
:106FE00080688C93A5E3B0E0E5E3F0E08081806405
:106FF0008C93A4E3B0E0E4E3F0E0808180648C93C0
:10700000E0E0F3E881EE8083E1E0F3E880E4808370
:10701000A5E5B0E0E5E5F0E090818FE789238C936A
:1070200080E090E09D9B05C0019641F09D9BF8CFCC
:10703000FBCF019619F09D99F3CFFBCFA5E5B0E00A
:10704000E5E5F0E0808180688C93A5E3B0E0E5E3BE
:10705000F0E090818FE789238C93A4E3B0E0E4E330
:10706000F0E090818FE789238C93A5E3B0E0E5E31E
:10707000F0E080818F7B8C93A4E3B0E0E4E3F0E068
:1070800080818F7B8C93E9E2F0E087E08083E9E9FF
:10709000F0E087E0808311241FBECFEFD0E1DEBF98
:1070A000CDBF17E0A0E0B1E0EAEAF4EE01E00BBFEB
:1070B00002C007900D92AE37B107D9F718E0AEE7DE
:1070C000B7E001C01D92A639B107E1F7EDE5F0E0A8
:1070D0008FEF9FE79183808386E998E09C018FEF93
:1070E0009FE7821B930B21E08138920768F086E9C5
:1070F00098E09C018FEF9EE7821B930B26E938E016
:10710000BC01C9010E9458830E94AF8D009711F104
:107110008CE598E09A838983E2EBF3E0FC83EB83D0
:10712000F9E0FD83EB81FC8100808B819C810196DD
:107130009C838B83E981FA81008289819A810196FF
:107140009A8389839D8191509D83ED81EE2351F730
:107150000E94E78D81E890E4EBEBF3E020E831E07A
:1071600040E050E0BC01CF010E94788E0E940000F8
:107170000C9454F20C940000CF93DF93CDB7DEB79C
:1071800026970FB6F894DEBF0FBECDBF9A838983D2
:107190007C836B838CE091E029813A81BC01C90139
:1071A0000E943EF1009779F48B819C81E5E1F1E04A
:1071B0009C0149E150E061E070E0CF010E9426E7C8
:1071C0001E821D821DC08FE291E029813A81BC019F
:1071D000C9010E943EF1009779F48B819C81E8E31C
:1071E000F1E09C0147E150E061E070E0CF010E94D6
:1071F00026E71E821D8204C08FEF9FEF9E838D8342
:107200008D819E8126960FB6F894DEBF0FBECDBF4E
:10721000DF91CF910895EF92FF920F931F93CF9339
:10722000DF93CDB7DEB728970FB6F894DEBF0FBE59
:10723000CDBF9C838B837E836D8380E591E06D81E0
:107240007E81EB81FC819C0148EC50E0CF010E94E3
:10725000F16580910A0190910B01EB81FC812FEF88
:107260003FEF4FEF5FEFBC01CF010E944C668B8177
:107270009C812FE431E0BC01C9010E942BE8ED8123
:10728000FE810190F081E02DF887EF838F81988552
:107290008230910581F08F8198858330910581F04E
:1072A0008F8198858130910509F00FC083E591E0C9
:1072B0009A8389830EC087E591E09A83898309C008
:1072C0008CE591E09A83898304C081E691E09A83FA
:1072D0008983ED81FE81E480F580ED81FE818281EC
:1072E00093812AE030E0B9010E94E0F18C01ED8148
:1072F000FE81828193812AE030E0B9010E94E0F1B1
:10730000CB01FF92EF921F930F939F938F938981ED
:107310009A819F938F938EEF90E09F938F938B81B1
:107320009C819F938F930E9405E88DB79EB70C9622
:107330000FB6F8949EBF0FBE8DBFED81FE81868192
:1073400097810097C1F0ED81FE81868197819F939F
:107350008F9380EF90E09F938F938B819C819F937D
:107360008F930E9405E88DB79EB706960FB6F894E6
:107370009EBF0FBE8DBFED81FE81808591850097F8
:10738000C1F0ED81FE81808591859F938F938DED76
:1073900090E09F938F938B819C819F938F930E940A
:1073A00005E88DB79EB706960FB6F8949EBF0FBE40
:1073B0008DBFED81FE81828593850097C1F0ED81BF
:1073C000FE81828593859F938F9386EC90E09F93B7
:1073D0008F938B819C819F938F930E9405E88DB73B
:1073E0009EB706960FB6F8949EBF0FBE8DBFED8177
:1073F000FE81848595850097C1F0ED81FE818485AD
:1074000095859F938F9385EB90E09F938F938B81CE
:107410009C819F938F930E9405E88DB79EB7069637
:107420000FB6F8949EBF0FBE8DBFED81FE8186859D
:1074300097850097C1F0ED81FE81868597859F93A2
:107440008F9381EA90E09F938F938B819C819F9390
:107450008F930E9405E88DB79EB706960FB6F894F5
:107460009EBF0FBE8DBFED81FE81808991890097FF
:10747000C1F0ED81FE81808991899F938F938CE883
:1074800090E09F938F938B819C819F938F930E9419
:1074900005E88DB79EB706960FB6F8949EBF0FBE4F
:1074A0008DBF8B819C8120E431E0BC01C9010E9429
:1074B0002BE88B819C810E947EE280E090E0289600
:1074C0000FB6F894DEBF0FBECDBFDF91CF911F91F5
:1074D0000F91FF90EF900895CF92DF92EF92FF927D
:1074E0000F931F93CF93DF93CDB7DEB728970FB6D7
:1074F000F894DEBF0FBECDBF9C838B837E836D83EC
:1075000080914B0890914C089A83898380E591E0A3
:107510006D817E81EB81FC819C0148EC50E0CF01C4
:107520000E94F16580910A0190910B01EB81FC8131
:107530002FEF3FEF4FEF5FEFBC01CF010E944C6692
:107540008B819C8123E232E0BC01C9010E942BE8BF
:1075500080914B0890914C089A83898376C0E98189
:10756000FA8183899489FC0180819181A281B38110
:107570008F3E2EEB92072DEAA2072EEDB20729F0DF
:1075800087EB91E098878F8304C08CEB91E098871C
:107590008F83E981FA8120893189E981FA818389A0
:1075A0009489D901A81BB90BE981FA810089118955
:1075B000E981FA81858996897C01E981FA81878947
:1075C000908DAC01E981FA8187859927880F991FF1
:1075D000FC01E155FE4F60817181E981FA81828968
:1075E000E82FFF2789819A819C012A5F3F4F89817B
:1075F0009A81CF80D884DF92CF92BF93AF931F93AD
:107600000F93FF92EF925F934F937F936F93FF934C
:10761000EF933F932F939F938F938CEA91E09F93E7
:107620008F938B819C819F938F930E9405E88DB7E8
:107630009EB746960FB6F8949EBF0FBE8DBFE981E8
:10764000FA81808191819A83898389819A810097C7
:1076500009F085CF8B819C8125E931E0BC01C9010E
:107660000E942BE88B819C810E947EE280E090E06A
:1076700028960FB6F894DEBF0FBECDBFDF91CF9135
:107680001F910F91FF90EF90DF90CF900895CF93CF
:10769000DF93CDB7DEB72A970FB6F894DEBF0FBEE3
:1076A000CDBF98878F837A87698780E591E0698568
:1076B0007A85EF81F8859C0148EC50E0CF010E946B
:1076C000F16580910A0190910B01EF81F8852FEF10
:1076D0003FEF4FEF5FEFBC01CF010E944C668F81FF
:1076E000988529EF33E0BC01C9010E942BE8809105
:1076F0005308909154089E838D838D819E810097BD
:1077000009F461C08F81988521E733E0BC01C9018C
:107710000E942BE819821A821B821C824FC0ED81C5
:10772000FE81208531854285538589819A81AB818F
:10773000BC81820F931FA41FB51F89839A83AB83DB
:10774000BC83ED81FE8186859785DC01ED81FE811C
:1077500084859585BC01ED81FE812481358146813A
:1077600057818D819E81FC01BF93AF937F936F936F
:107770005F934F933F932F9389819A81AB81BC8113
:10778000BF93AF939F938F93FF93EF9386E293E022
:107790009F938F938F8198859F938F930E9405E885
:1077A0008DB79EB742960FB6F8949EBF0FBE8DBFA1
:1077B000ED81FE81808191819E838D838D819E816B
:1077C000009709F0ACCF8F8198852FE033E0BC01A2
:1077D000C9010E942BE88F8198850E947EE280E09B
:1077E00090E02A960FB6F894DEBF0FBECDBFDF91B2
:1077F000CF9108950F931F93CF93DF93CDB7DEB74B
:107800002A970FB6F894DEBF0FBECDBF9E838D833F
:1078100078876F8380E591E06F817885ED81FE81C7
:107820009C0148EC50E0CF010E94F16580910A0173
:1078300090910B01ED81FE812FEF3FEF4FEF5FEF56
:10784000BC01CF010E944C668D819E812CE035E009
:10785000BC01C9010E942BE88091EC079091ED07D3
:107860009A83898301C1E981FA818389282F33278B
:107870003A87298789859A858530910509F465C0FD
:1078800029853A85263031050CF589859A8582301F
:10789000910509F441C029853A85233031055CF40E
:1078A00089859A85009709F464C029853A85213035
:1078B000310569F163C089859A858330910589F125
:1078C00029853A852430310589F158C089859A8502
:1078D0008830910509F443C029853A85293031055E
:1078E0005CF489859A858630910529F129853A8548
:1078F0002730310579F142C089859A858930910513
:10790000F9F029853A852A30310571F137C08FEABF
:1079100094E09C838B8336C087EA94E09C838B83BE
:1079200031C08FE994E09C838B832CC08DE794E079
:107930009C838B8327C084E794E09C838B8322C045
:107940008BE694E09C838B831DC081E694E09C834E
:107950008B8318C089E594E09C838B8313C081E5F9
:1079600094E09C838B830EC088E494E09C838B839B
:1079700009C081E494E09C838B8304C089E394E094
:107980009C838B83E981FA81808D918D0E94523D89
:107990008C01E981FA8184899589A689B789BC011E
:1079A000CD010E9485B39C0189819A811F930F9319
:1079B0003F932F939F938F9380EE94E09F938F93A9
:1079C0008D819E819F938F930E9405E88DB79EB70E
:1079D0000A960FB6F8949EBF0FBE8DBFE981FA815B
:1079E000868D978D0E94523D8C01E981FA81828DAE
:1079F000938DA48DB58DBC01CD010E9485B31F93DD
:107A00000F939F938F938DEC94E09F938F938D8131
:107A10009E819F938F930E9405E82DB73EB7285F04
:107A20003F4F0FB6F8943EBF0FBE2DBF8D819E8194
:107A30002B813C81BC01C9010E942BE88D819E8174
:107A4000EFEBF1E09C014CE050E061E070E0CF0131
:107A50000E9426E78D819E810E947EE2E981FA8163
:107A6000808191819A83898389819A81009709F025
:107A7000FACE8D819E8126EB34E0BC01C9010E94C3
:107A80002BE88D819E810E947EE280E090E02A9624
:107A90000FB6F894DEBF0FBECDBFDF91CF911F911F
:107AA0000F910895CF93DF93CDB7DEB722970FB62E
:107AB000F894DEBF0FBECDBF9A83898389819A81F6
:107AC000082E892F902D9A83898389819A81229605
:107AD0000FB6F894DEBF0FBECDBFDF91CF910895F2
:107AE000CF93DF93CDB7DEB72C970FB6F894DEBFF8
:107AF0000FBECDBF9A8789877C876B8780E591E031
:107B00006B857C85E985FA859C0148EC50E0CF01C6
:107B10000E94F16580910A0190910B01E985FA8537
:107B20002FEF3FEF4FEF5FEFBC01CF010E944C669C
:107B300089859A8524E036E0BC01C9010E942BE8C2
:107B4000EB85FC8580859185009709F443C08B8582
:107B50009C850E949C6D9A8389831C821B8233C002
:107B60008B819C812B853C85BC01C9010E94B56D30
:107B700098878F838B819C812B853C85BC01C901B3
:107B80000E94F16D9E838D832FEA35E08D819E8169
:107B90009F938F938F8198859F938F933F932F937C
:107BA00089859A859F938F930E9405E88DB79EB72C
:107BB00008960FB6F8949EBF0FBE8DBF8B819C8137
:107BC00001969C838B832B813C8189819A81281724
:107BD000390734F289859A852CEB35E0BC01C9015F
:107BE0000E942BE889859A850E947EE280E090E0E1
:107BF0002C960FB6F894DEBF0FBECDBFDF91CF91AC
:107C00000895CF93DF93CDB7DEB727970FB6F894DB
:107C1000DEBF0FBECDBF9F838E838E819F81898300
:107C200000C00E9460A39D838C838C819D810097FE
:107C3000A9F4898199279F938F938CEC91E09F936E
:107C40008F930E9481E70F900F900F900F9068E83C
:107C500073E180E090E00E940389E3CF8C819D81F5
:107C600060E570E00E9454A70E947A839C0189819C
:107C700099273F932F939F938F9389EE91E09F9342
:107C80008F930E9481E78DB79EB706960FB6F89442
:107C90009EBF0FBE8DBF14C0898199279F938F937C
:107CA00088E092E09F938F930E9481E70F900F905E
:107CB0000F900F9068EE73E080E090E00E940389DF
:107CC0000E947A8320E28030920730F32C813D813C
:107CD00086E192E0BC01C9010E94D1E19B838A83C5
:107CE0008A819B81009779F4898199279F938F934B
:107CF0008AE192E09F938F930E9481E70F900F900B
:107D00000F900F9008C08A819B810E948C728A819B
:107D10009B810E946BE18C819D810E94EBA98981EE
:107D200099279F938F938EE392E09F938F930E9466
:107D300081E70F900F900F900F9073CFCF92DF924B
:107D4000EF92FF920F931F93CF93DF93CDB7DEB7E0
:107D5000A9970FB6F894DEBF0FBECDBF80E092ECBE
:107D6000A1E0B0E08E879F87A88BB98B85E796E06E
:107D700040E060E070E00E94558D80912607909170
:107D8000270721E532E0E3E5F2E0AC01B901CF01DC
:107D90000E949FE480912607909127070E9426E386
:107DA0009C01CE010E96AC0161E071E0C9010E9418
:107DB00049E068EC70E080E090E00E9403890E9456
:107DC000248E9F938F9389E592E09F938F930E94D7
:107DD00081E70F900F900F900F908BEB96E040E0B3
:107DE00060E070E00E94558D009721F084E792E0FA
:107DF0000E94A9E78EE892E09F938F9383E992E037
:107E00009F938F930E9481E70F900F900F900F9098
:107E10008EE892E00E9410B8009709F49EC0CE014F
:107E2000429699A388A3E4E5F3E0FBA3EAA3F7E075
:107E3000FCA3EAA1FBA100808AA19BA101969BA3C0
:107E40008AA3E8A1F9A1008288A199A1019699A32A
:107E500088A39CA191509CA3ECA1EE2351F783EA47
:107E600092E09F938F930E9481E70F900F90CE0135
:107E70004296EEE8F2E020E63AEE40E050E0BC0147
:107E8000CF010E940753009709F47CC083EB92E076
:107E90000E94F1B2DC01CB0189879A87AB87BC874E
:107EA00082EC92E00E94F1B2DC01CB018D839E83D3
:107EB000AF83B88780ED92E00E94F1B2DC01CB0184
:107EC00089839A83AB83BC838EED92E09F938F93DB
:107ED0000E9481E70F900F908D819E81AF81B885C0
:107EE00029853A854B855C85BE016E5E7F4FEEE845
:107EF000F2E07C018D01CF010E94BCB6009741F5F4
:107F000089819A81AB81BC810097A105B105D9F027
:107F100089EE92E09F938F930E9481E70F900F90DC
:107F20002BEB36E089819A81AB81BC8169017C01B0
:107F30008D0120E030E040E050E060E070E080E063
:107F400090E00E941BB08CEB91E00E94A9E71AC060
:107F50008CEF92E00E94A9E715C08EE892E020E63F
:107F60003AEE40E050E060E070E00E940753009776
:107F700029F08CEF92E00E94A9E704C08CEB91E01D
:107F80000E94A9E78091800890918108A0918208C1
:107F9000B0918308BC01CD010E9485B39F938F935C
:107FA00083E093E09F938F930E9481E70F900F905F
:107FB0000F900F9021E030E040E050E06FEF7FEF56
:107FC0008FEF9FEF0E948B6581E097E040E060E0DB
:107FD00070E00E94558D8BE099E32DE033E0BC0109
:107FE000C9010E94FF5F8CE69AE326E133E0BC0101
:107FF000C9010E94FF5F87E49BE322E233E0BC01FA
:10800000C9010E94FF5F8AEF9BE32DE233E0BC01D0
:10801000C9010E94FF5F80E79DE329E333E0BC01D3
:10802000C9010E94FF5F82E493E02CE433E0BC01CD
:10803000C9010E94CC5E0E943E810E9425788CEB93
:1080400098E30E94FB7781E08D8732C0CE0149968C
:108050009EA38DA3EBE5F3E0F8A7EFA3F7E0F9A764
:10806000EFA1F8A500808FA198A5019698A78FA3EE
:10807000EDA1FEA100828DA19EA101969EA38DA3DC
:1080800099A5915099A7E9A5EE2351F78D85805DBB
:108090008E8F8D85992761E07EE3FE01799620E041
:1080A00033E0AC01CF010E94788E8D858F5F8D8784
:1080B0008D85853058F28EEF0E944E8560E67AEE0F
:1080C00080E090E00E940389F9CFCF93DF93CDB792
:1080D000DEB722970FB6F894DEBF0FBECDBF8A83FE
:1080E0008091AC0389838A818093AC03898199272D
:1080F00022960FB6F894DEBF0FBECDBFDF91CF91B1
:108100000895CF93DF93CDB7DEB723970FB6F894DA
:10811000DEBF0FBECDBF9B838A830E9478868EE927
:108120009EE3EDEAF3E020E033E040E050E0BC0104
:10813000CF010E94788E8EEF0E944E8500C00E9473
:1081400029850E94B3858091AC038F3FC1F3E5E59B
:10815000F0E080818C718983A5E5B0E0E5E5F0E091
:108160008081982F937E8091AC03892B8C93A5E519
:10817000B0E0E5E5F0E0808180628C938895A5E52C
:10818000B0E0E5E5F0E080818F7D8C93A5E5B0E07F
:10819000E5E5F0E08081982F937E8981892B8C938F
:1081A000CECFCF93DF93CDB7DEB726970FB6F89437
:1081B000DEBF0FBECDBF9A8389837C836B835E83D2
:1081C0004D83E981FA8180819181009731F0E981C5
:1081D000FA81808191810E94CEE88D819E810196F5
:1081E0000E94A7E8E981FA8191838083E981FA817D
:1081F000808191810097E9F08D819E81009779F0CF
:108200004D815E81E981FA81808191812B813C8160
:10821000FC01CA01AC01B901CF010E9405F1E9815D
:10822000FA81208131818D819E81F901E80FF91F4A
:10823000108226960FB6F894DEBF0FBECDBFDF9139
:10824000CF910895CF93DF93CDB7DEB722970FB6C6
:10825000F894DEBF0FBECDBF9A83898389819A814E
:108260000097E1F0E981FA8181A592A5009731F0AC
:10827000E981FA8181A592A50E94CEE8E981FA817F
:1082800083A594A5009731F0E981FA8183A594A58F
:108290000E94CEE889819A810E94CEE822960FB68C
:1082A000F894DEBF0FBECDBFDF91CF910895CF937D
:1082B000DF93CDB7DEB761970FB6F894DEBF0FBE80
:1082C000CDBF9D878C877F876E878DE290E00E946F
:1082D000A7E89F838E838E819F81009719F4198A66
:1082E000188A67C28E819F812DE2FC01DF01822FF7
:1082F0001D928A95E9F7EE81FF8180EC98EAA0E073
:10830000B0E085A396A3A7A3B0A78C859D85DC01CB
:1083100050968E819F81FC0131968D919D910D909B
:10832000BC91A02D80839183A283B3838C859D858E
:1083300084519F4F04969B878A878E859F85805F97
:10834000904099878887BBC1EA85FB858081882317
:1083500059F48A859B8501969B878A8788859985AC
:10836000019799878887ABC18A859B85FC013196E7
:1083700080818D838D81282F332788859985821769
:1083800093070CF4A7C1EA85FB858081853369F4E6
:108390008D81813009F09EC18A859B85FC013296D2
:1083A0008081EE81FF81808376C1EA85FB858081B3
:1083B0008C3079F48D81482F55278A859B859C01C7
:1083C0002E5F3F4F8E819F818996B9010E94D140D7
:1083D00062C1EA85FB8580818F3079F48D81482FD9
:1083E00055278A859B859C012E5F3F4F8E819F81FB
:1083F0008B96B9010E94D1404EC18D81843008F422
:108400004AC18A859B85FC01329680819927AA27DB
:10841000BB2789839A83AB83BC838A859B85FC01B8
:10842000339680819927AA27BB272227382F492FE7
:108430005A2F89819A81AB81BC81820F931FA41F1F
:10844000B51F89839A83AB83BC838A859B85FC0196
:10845000349680819927AA27BB27AC01332722278E
:1084600089819A81AB81BC81820F931FA41FB51FA4
:1084700089839A83AB83BC838A859B85FC0135966F
:1084800080819927AA27BB27582F442733272227E3
:1084900089819A81AB81BC81820F931FA41FB51F74
:1084A00089839A83AB83BC83EA85FB858081813095
:1084B00059F4EE81FF8189819A81AB81BC818583EA
:1084C0009683A783B087E7C0EA85FB8580818C31DE
:1084D00059F4EE81FF8189819A81AB81BC818187CA
:1084E0009287A387B487D7C0EA85FB8580818330D4
:1084F00059F4EE81FF8189819A81AB81BC818587A6
:108500009687A787B08BC7C0EA85FB8580818630B8
:1085100009F070C0EE81FF8189819A81AB81BC81B5
:10852000818B928BA38BB48B8D81883008F4B3C080
:108530008A859B85FC01369680819927AA27BB27CF
:10854000EE81FF81858B968BA78BB08FEE81FF81AB
:10855000258936894789508D8A859B85FC01379608
:1085600080819927AA27BB27BA2FA92F982F882760
:10857000820F931FA41FB51FEE81FF81858B968B01
:10858000A78BB08FEE81FF81258936894789508D71
:108590008A859B85FC01389680819927AA27BB276D
:1085A000DC0199278827820F931FA41FB51FEE8136
:1085B000FF81858B968BA78BB08FEE81FF812589FC
:1085C00036894789508D8A859B85FC013996808143
:1085D0009927AA27BB27B82FAA2799278827820F70
:1085E000931FA41FB51FEE81FF81858B968BA78BF0
:1085F000B08F51C0EA85FB858081863359F4EE81C6
:10860000FF8189819A81AB81BC81818F928FA38FF9
:10861000B48F41C0EA85FB8580818A3389F48981E2
:108620009A81AB81BC81BC01CD010E94E443DC0195
:10863000CB01EE81FF81858F968FA78FB0A32BC0D2
:10864000EA85FB8580818B3389F489819A81AB81AE
:10865000BC81BC01CD010E94E443DC01CB01EE8171
:10866000FF8181A392A3A3A3B4A315C0EA85FB85D0
:108670008081833381F489819A81AB81BC81BC0183
:10868000CD010E94E443DC01CB01EE81FF8185A393
:1086900096A3A7A3B0A78D8199279C018A859B8566
:1086A000820F931F02969B878A878D81282F3327FD
:1086B00088859985821B930B029799878887EA851D
:1086C000FB8580818F3F31F08885998518161906C2
:1086D0000CF43ACEEA85FB8580818F3F79F4EE81F8
:1086E000FF818081823089F0EE81FF818081853039
:1086F00061F0EE81FF818081863039F08E819F812B
:108700000E942241198A188A54C0EE81FF81858D0A
:10871000968DA78DB0A10097A105B10581F4EE81DA
:10872000FF8185A196A1A7A1B0A5B695A79597951C
:108730008795EE81FF81858F968FA78FB0A3EE81FD
:10874000FF8181A192A1A3A1B4A10097A105B105C8
:1087500061F5EE81FF81258D368D478D50A1EE812B
:10876000FF81858D968DA78DB0A1B695A79597951C
:108770008795280F391F4A1F5B1FEE81FF81858D6A
:10878000968DA78DB0A1B695A79597958795B69527
:10879000A79597958795820F931FA41FB51FEE810C
:1087A000FF8181A392A3A3A3B4A3AE81BF81B98BA0
:1087B000A88B8889998961960FB6F894DEBF0FBEA1
:1087C000CDBFDF91CF910895CF93DF93CDB7DEB7C3
:1087D00024970FB6F894DEBF0FBECDBF69837A83AE
:1087E0008B839C8389819A81AB81BC81082E8B2FDE
:1087F000B02D092E9A2FA02D89839A83AB83BC8339
:1088000089819A81AB81BC81BC01CD0124960FB6D0
:10881000F894DEBF0FBECDBFDF91CF910895CF9307
:10882000DF93CDB7DEB726970FB6F894DEBF0FBE45
:10883000CDBF9A8389836B835D834C832E83E981CB
:10884000FA818B81808389819A8101969A838983B9
:10885000E981FA818E81808389819A8101969A8348
:1088600089838E81482F552789819A812C813D816A
:10887000FC01CA01AC01B901CF010E9405F18E8152
:108880009927029626960FB6F894DEBF0FBECDBF8D
:10889000DF91CF910895CF93DF93CDB7DEB72497C3
:1088A0000FB6F894DEBF0FBECDBF9A8389836B836A
:1088B0004C83E981FA818B81808389819A81019639
:1088C0009A838983E981FA8181E0808389819A8111
:1088D00001969A838983E981FA818C8180838981D9
:1088E0009A8101969A83898383E090E024960FB65B
:1088F000F894DEBF0FBECDBFDF91CF910895CF9327
:10890000DF93CDB7DEB725970FB6F894DEBF0FBE65
:10891000CDBF9A8389836B835D834C83E981FA8120
:108920008B81808389819A8101969A838983E981E9
:10893000FA8182E0808389819A8101969A83898372
:108940008C819D810E94B9449D838C83A981BA81C9
:10895000FE013496808191818D939C9384E090E018
:1089600025960FB6F894DEBF0FBECDBFDF91CF9135
:108970000895CF93DF93CDB7DEB722970FB6F89463
:10898000DEBF0FBECDBF9A83898389819A81082E6D
:10899000892F902D9A83898389819A8122960FB697
:1089A000F894DEBF0FBECDBFDF91CF910895CF9376
:1089B000DF93CDB7DEB722970FB6F894DEBF0FBEB8
:1089C000CDBF9A838983E981FA8187E38083898196
:1089D0009A8101969A838983E981FA8183E0808371
:1089E00089819A8101969A838983E981FA8181E05C
:1089F000808389819A8101969A838983E981FA81AA
:108A000083E0808389819A8101969A838983E981B1
:108A1000FA8186E0808389819A8101969A8389838D
:108A200085E090E022960FB6F894DEBF0FBECDBF72
:108A3000DF91CF910895CF92DF92EF92FF920F9343
:108A40001F93CF93DF93CDB7DEB764970FB6F8943B
:108A5000DEBF0FBECDBF9C838B836D832E833F8390
:108A600048875987EA86FB860C871D87DF86CE8676
:108A70008B819C8124E232E0FC01DF01C9011D925F
:108A80000197E9F7EB81FC8181E08083EB81FC8138
:108A900081E08183EB81FC8186E082838B819C81F4
:108AA0004C96998B888BAAE7B8E0BB8BAA8BB6E073
:108AB000BC8BEA89FB8900808A899B8901969B8B04
:108AC0008A8BA889B9890C92E889F9893196F98B42
:108AD000E88BFC89F150FC8B8C89882351F7EB8162
:108AE000FC818E819F81A885B98584839583A68327
:108AF000B7838E859F850E94B944EB81FC81918765
:108B00008087EB81FC818A859B85AC85BD858487C8
:108B10009587A687B7878B819C8184519F4F9A83C5
:108B20008983E981FA8183E6808389819A8101962C
:108B30009A838983E981FA8182E8808389819A8195
:108B400001969A838983E981FA8183E5808389810B
:108B50009A8101969A838983E981FA8183E68083E9
:108B600089819A8101969A83898389819A814D812D
:108B700065E30E944B44049664960FB6F894DEBFFA
:108B80000FBECDBFDF91CF911F910F91FF90EF905E
:108B9000DF90CF900895EF92FF920F931F93CF93A2
:108BA000DF93CDB7DEB72C970FB6F894DEBF0FBEBC
:108BB000CDBF9A8389834B835C836D837E833887A3
:108BC0002F831A87098729853A858F819885820F97
:108BD000931FFC01E451FF4F8FEF808389859A85B5
:108BE00001969A87898789859A8584519F4F9A87AC
:108BF000898789859A8521E08C32920720F48CE25E
:108C000091E09A87898729853A854F8158858B819C
:108C10009C81AD81BE81E981FA8179018A0123E4D9
:108C200030E0AC01BD01CF010E94D6AD99235CF4C8
:108C300083E190E090938507809384078FEF9FEF07
:108C40009C878B8702C01C861B868B859C852C96F7
:108C50000FB6F894DEBF0FBECDBFDF91CF911F914D
:108C60000F91FF90EF900895CF92DF92EF92FF92D5
:108C70000F931F93CF93DF93CDB7DEB76C970FB6EB
:108C8000F894DEBF0FBECDBF9A8B898B4B8B5C8B6C
:108C90006D8B7E8B388F2F8BE98EFA8E0B8F1C8F0E
:108CA0000E94278ADC01CB018D839E83AF83B88726
:108CB000898D9A8DAB8DBC8D89839A83AB83BC8360
:108CC00089819A81AB81BC812F89388DAE01455F46
:108CD0005F4FBE01635F7F4FE989FA896C017D01B7
:108CE00004E212E0CF010E943FAE9A87898789850E
:108CF0009A851816190664F089859A8599230CF0CF
:108D00005BC084E190E0909385078093840754C012
:108D100089859A85823F9105A0F0EF89F88D808141
:108D2000823079F4EF89F88D24813581468157812D
:108D30008B899C89AD89BE89281739074A075B074B
:108D4000D9F10E94278A9B01AC018D819E81AF8160
:108D5000B88579018A01E81AF90A0A0B1B0BD801B8
:108D6000C70189839A83AB83BC83898D9A8DAB8D30
:108D7000BC8D9C01AD012A5F30404040504089814C
:108D80009A81AB81BC8182179307A407B50718F0BD
:108D90001A86198611C0898D9A8DAB8DBC8D29815B
:108DA0003A814B815C81821B930BA40BB50B8983A9
:108DB0009A83AB83BC8384CF89859A856C960FB6E2
:108DC000F894DEBF0FBECDBFDF91CF911F910F9101
:108DD000FF90EF90DF90CF900895CF92DF92EF92C7
:108DE000FF920F931F93CF93DF93CDB7DEB76497B6
:108DF0000FB6F894DEBF0FBECDBF98878F837A87FA
:108E000069872B873C874D875E87EF86F88A098BB9
:108E10001A8BDC8ACB8A89859A8584519F4F9A83E5
:108E200089832B893C898B859C85AD85BE85E985A9
:108E3000FA856901EE24FF2487019C01AD0161E000
:108E4000CF010E941B459E838D838F859889A989B8
:108E5000BA890097A105B105B1F02D813E818981C4
:108E60009A81F901E80FF91FCE010F9624E0AC01B9
:108E700062E3CF010E940F449C018D819E81820F8D
:108E8000931F9E838D832D813E8189819A81820FDC
:108E9000931F0E94D7449C018D819E81820F931F56
:108EA0009E838D838CE598E0DC01FD01019000201C
:108EB000E9F73197CF018A1B9B0B9C838B838B81B6
:108EC0009C8118161906BCF44B812D813E81898145
:108ED0009A81F901E80FF91F8CE598E0242FAC0185
:108EE0006CE0CF010E940F449C018D819E81820F16
:108EF000931F9E838D832D813E8189819A81820F6C
:108F0000931F40E452E069E30E947F449C018D81FD
:108F10009E81820F931F9E838D838D819E812985E3
:108F20003A85EF81F8858C014FEF5FEF6FEF7FEFB0
:108F3000CF010E94CB4564960FB6F894DEBF0FBEFA
:108F4000CDBFDF91CF911F910F91FF90EF90DF90F8
:108F5000CF900895AF92BF92CF92DF92EF92FF929F
:108F60000F931F93CF93DF93CDB7DEB766970FB6FE
:108F7000F894DEBF0FBECDBF98878F8349875A878D
:108F80006B877C873E872D87EF86F88A098B1A8B43
:108F9000AB8ABC8ACD8ADE8A8D859E8584519F4F9F
:108FA0009A8389836BA57CA58B899C89AD89BE89B1
:108FB0002F85388949895A89ED85FE856B017C01A9
:108FC0008D0163E0CF010E941B459E838D838BA1A1
:108FD0009CA1ADA1BEA10097A105B105A1F02D8175
:108FE0003E8189819A81820F931F24E0AE014D5DFD
:108FF0005F4F62E30E940F449C018D819E81820F2E
:10900000931F9E838D838FA198A5A9A5BAA50097CC
:10901000A105B105B1F02D813E8189819A81F901C7
:10902000E80FF91FCE01879624E0AC0166E3CF017B
:109030000E940F449C018D819E81820F931F9E830D
:109040008D832D813E8189819A81820F931F0E9499
:10905000D7449C018D819E81820F931F9E838D83B7
:109060008CE598E0DC01FD0101900020E9F73197E3
:10907000CF018A1B9B0B9C838B838B819C81181651
:109080001906BCF44B812D813E8189819A81F901B9
:10909000E80FF91F8CE598E0242FAC016CE0CF01BC
:1090A0000E940F449C018D819E81820F931F9E839D
:1090B0008D832D813E814D855E8589859A85AB8521
:1090C000BC85EF81F88589019A01AC01BD01CF0112
:1090D0000E94CB4566960FB6F894DEBF0FBECDBF9B
:1090E000DF91CF911F910F91FF90EF90DF90CF9084
:1090F000BF90AF900895AF92BF92CF92DF92EF9260
:10910000FF920F931F93CF93DF93CDB7DEB7609796
:109110000FB6F894DEBF0FBECDBF9A8389837C83E0
:109120006B832D833E834F835887E986FA860B87AE
:109130001C87AD86BE86CF86D88A29853A854B8521
:109140005C85ED80FE800F8118856B817C81E981D3
:10915000FA8189A19AA19F938F938D8D9E8DAF8D5A
:10916000B8A1BF93AF939F938F938D859E85AF8555
:10917000B889BF93AF939F938F9359016A019B0165
:109180004FEF5FEF6FEF7FEFCF010E94AA472DB740
:109190003EB7265F3F4F0FB6F8943EBF0FBE2DBFC0
:1091A00060960FB6F894DEBF0FBECDBFDF91CF91B2
:1091B0001F910F91FF90EF90DF90CF90BF90AF90F5
:1091C0000895AF92BF92CF92DF92EF92FF920F93EA
:1091D0001F93CF93DF93CDB7DEB764970FB6F894A4
:1091E000DEBF0FBECDBF9E838D834F8358876987B7
:1091F0007A873C872B87ED86FE860F87188BA98A96
:10920000BA8ACB8ADC8A8B859C8584519F4F9A834E
:10921000898389899A89AB89BC892D853E854F854B
:109220005889EB85FC85CC24DD247C018D0167E029
:10923000CF010E941B459C838B8389A19AA1ABA17E
:10924000BCA10097A105B105A1F02B813C818981CA
:109250009A81820F931F24E0AE014F5D5F4F66E35A
:109260000E940F449C018B819C81820F931F9C83E1
:109270008B832B813C814B855C858F819885A9856B
:10928000BA85ED81FE8189019A01AC01BD01CF0152
:109290000E94CB4564960FB6F894DEBF0FBECDBFDB
:1092A000DF91CF911F910F91FF90EF90DF90CF90C2
:1092B000BF90AF900895AF92BF92CF92DF92EF929E
:1092C000FF920F931F93CF93DF93CDB7DEB76697CF
:1092D0000FB6F894DEBF0FBECDBF98878F83498746
:1092E0005A876B877C873E872D87EF86F88A098BA4
:1092F0001A8BAB8ABC8ACD8ADE8A8D859E85845185
:109300009F4F9A8389838B899C89AD89BE892F85DC
:10931000388949895A89ED85FE85CC24DD247C0174
:109320008D0168E0CF010E941B459E838D832D81B6
:109330003E8189819A81820F931F0E94D7449C01AC
:109340008D819E81820F931F9E838D838CE598E093
:10935000DC01FD0101900020E9F73197CF018A1B64
:109360009B0B9C838B838B819C810097B9F04B81F5
:109370002D813E8189819A81F901E80FF91F8CE5E1
:1093800098E0242FAC016CE0CF010E940F449C01B7
:109390008D819E81820F931F9E838D832D813E81BF
:1093A00089819A81820F931F40E452E069E30E9411
:1093B0007F449C018D819E81820F931F9E838D83AC
:1093C0002D813E814D855E8589859A85AB85BC85DD
:1093D000EF81F88589019A01AC01BD01CF010E949E
:1093E000CB4566960FB6F894DEBF0FBECDBFDF91BA
:1093F000CF911F910F91FF90EF90DF90CF90BF9092
:10940000AF900895CF93DF93CDB7DEB72A970FB60D
:10941000F894DEBF0FBECDBF9C838B837E836D83AC
:1094200058874F838F8198852D813E81BC01C9016A
:109430000E9457419A83898389819A81009729F4F0
:109440008B819C819A87898780C0E981FA8180819C
:10945000823049F089819A810E9422418B819C81CE
:109460009A87898772C08B819C81009729F48981B2
:109470009A819C838B8365C080918008909181083C
:10948000A0918208B09183082091840830918508CA
:10949000409186085091870882239323A423B52303
:1094A0000097A105B10579F1EB81FC812181328121
:1094B000438154818091800890918108A091820815
:1094C000B0918308281739074A075B07D1F1E98172
:1094D000FA81218132814381548180918008909169
:1094E0008108A0918208B0918308281739074A079C
:1094F0005B0739F58B819C810E94224189819A8189
:109500009C838B831EC0E981FA8125A136A147A1E6
:1095100050A5EB81FC8185A196A1A7A1B0A58217DA
:109520009307A407B50748F48B819C810E942241D0
:1095300089819A819C838B8304C089819A810E944E
:1095400022418B819C819A87898789859A852A9671
:109550000FB6F894DEBF0FBECDBFDF91CF91089557
:10956000CF93DF93CDB7DEB7E4970FB6F894DEBFA5
:109570000FBECDBF99AB88AB1DA61CA61BA61AA615
:1095800019A618A61F8E1E8E0E94088ADC01CB0128
:109590008A8F9B8FAC8FBD8F1E8A1F8A188E198E63
:1095A00080EA9FE0A0E0B0E08D879E87AF87B88B10
:1095B0008091800890918108A0918208B0918308E1
:1095C00089879A87AB87BC87E8A9F9A9878590899D
:1095D00099A388A31AA21BA21CA21DA2198A2FC09C
:1095E0008AA19BA1ACA1BDA1BA2FA92F982F882732
:1095F0008AA39BA3ACA3BDA38989282F332785E029
:1096000090E03C01621A730A930188A199A1820F2C
:10961000931FFC0131968081282F3327442755273B
:109620008AA19BA1ACA1BDA1820F931FA41FB51F4E
:109630008AA39BA3ACA3BDA389898F5F898B8989EA
:10964000843070F2198A00C08FEF9FEFAFEFBFEF49
:109650008D839E83AF83B8878989882331F12D85D7
:109660003E854F8558898D859E85AF85B889820F47
:10967000931FA41FB51F8D879E87AF87B88B8D85DD
:109680009E85AF85B88981300AEF900700E0A0077A
:1096900000E0B00708F43EC080E09AEFA0E0B0E040
:1096A0008D879E87AF87B88B35C080EA9FE0A0E0AA
:1096B000B0E08D879E87AF87B88B8091830783301A
:1096C00059F08AA19BA1ACA1BDA10196A11DB11D1C
:1096D0008AA39BA3ACA3BDA380917F079091800731
:1096E0000097C1F0E0917F07F0918007818D928D06
:1096F000A38DB48D0097A105B10561F0E0917F07BE
:10970000F0918007818D928DA38DB48D8D839E8382
:10971000AF83B88780918307882309F46CC0809158
:109720008A0790918B07A0918C07B0918D070097C5
:10973000A105B10509F45FC00E94278A9B01AC0115
:1097400080918E0790918F07A0919007B09191071B
:1097500039014A01681A790A8A0A9B0AD401C301AD
:1097600089839A83AB83BC8320918A0730918B07CE
:1097700040918C0750918D0789819A81AB81BC8182
:1097800082179307A407B50748F081E090E0909313
:109790008507809384071092830756CF20918A070C
:1097A00030918B0740918C0750918D0789819A8168
:1097B000AB81BC8149015A01881A990AAA0ABB0ADD
:1097C000D501C40189839A83AB83BC8329813A8103
:1097D0004B815C818D859E85AF85B88928173907B7
:1097E0004A075B0740F489819A81AB81BC818D87F0
:1097F0009E87AF87B88B80918307823041F080913C
:109800008307863021F0809183078730A1F589890D
:10981000882339F10E94088ADC01CB012A8D3B8D17
:109820004C8D5D8D821B930BA40BB50B803000E03B
:10983000900701E0A00700E0B00728F08FEF9FEF4E
:109840009F8F8E8F18C00E94088ADC01CB019C017B
:109850008A8D9B8DA901481B590BCA019F8F8E8F42
:109860000AC00E94088ADC01CB018A8F9B8FAC8FD3
:10987000BD8F1F8E1E8E80918307853021F08091D1
:1098800083078823B1F48AA59BA5009731F08AA5A8
:109890009BA50E94EDAE1BA61AA688A599A50097C8
:1098A00009F457C088A599A50E94CEE819A618A664
:1098B00050C080917F0790918007009769F4E8A1DC
:1098C000F9A187819085A185B2850097A105B10591
:1098D00019F010928307B8CE8AA59BA5009721F0B6
:1098E00088A599A50097A9F58AA59BA5009731F4AD
:1098F00084E490E00E943BAD9BA78AA788A599A528
:10990000009731F484E292E00E94A7E899A788A723
:109910008AA59BA5009721F088A599A5009749F4F1
:1099200082E190E0909385078093840710928307EB
:109930008BCE80EC96E09FA78EA7CE018E96EAA5EF
:10994000FBA522E030E0AC0162E070E1CF010E94B3
:1099500086AF80918307813041F5198A8AA19BA146
:10996000ACA1BDA10196A11DB11D8AA39BA3ACA36F
:10997000BDA32091840830918508409186085091BC
:10998000870889859A85AB85BC8582239323A42388
:10999000B5230097A105B10521F482E080938307E8
:1099A000A6C584E080938307A2C580918307823097
:1099B00009F08AC01CAA8989843010F051E05CABA0
:1099C00089898F5F898B8CA9882349F081E090E099
:1099D00090938507809384071092830788C56E8DC6
:1099E0007F8D89859A85AB85BC852AA13BA14CA139
:1099F0005DA1E8A5F9A5AAA4BBA46B017C018D011A
:109A0000BF01C5010E94ED46992394F5109283078A
:109A10006EC52EA13FA1E0917F07F091800788A538
:109A200099A5A901BC01CF010E94024A9093800729
:109A300080937F0780917F07909180070097C1F006
:109A400080918A0790918B07A0918C07B0918D0728
:109A5000803E0EE2900700E0A00700E0B00708F1AA
:109A600080EA9FE0A0E0B0E08D879E87AF87B88B4B
:109A70008D859E85AF85B88928A539A54AA15BA1AA
:109A80006CA17DA1EAA5FBA57C018D01CF010E94FF
:109A900034469FA38EA38EA19FA1181619060CF41D
:109AA000B8CF8EA19FA199231CF4109283071FC5E4
:109AB00080917F0790918007009709F418C5198A53
:109AC00083E08093830713C580918307833009F077
:109AD000A0C01BAA8989843010F011E01BAB8989D2
:109AE0008F5F898B2BA9222321F081E0809383074C
:109AF000FEC4E0917F07F0918007218D328D438D68
:109B0000548DE0917F07F0918007E180F28003811E
:109B100014816AA07BA08CA09DA068A579A5EAA568
:109B2000FBA58E8D9F8D9F938F935F934F933F9354
:109B30002F9357016801EE24FF248701A4019301AC
:109B4000CF010E947B484DB75EB74A5F5F4F0FB6AB
:109B5000F8945EBF0FBE4DBF99231CF4109283078B
:109B6000C6C48D859E85AF85B88928A539A54AA12B
:109B70005BA16CA17DA1EAA5FBA57C018D01CF01B4
:109B80000E9434469FA38EA38EA19FA199231CF40B
:109B900010928307ACC48EA19FA1181619060CF071
:109BA000A6C48EA19FA128A539A5BC01C9010E9408
:109BB00057419DA78CA78CA59DA5009709F497C434
:109BC000ECA5FDA580818530D1F480917F0790912F
:109BD00080070E9422418CA59DA5909380078093C9
:109BE0007F071DA61CA68A8D9B8DAC8DBD8D8E8B8F
:109BF0009F8BA88FB98F85E08093830778C4ECA5ED
:109C0000FDA58081863009F072C481E080938307CE
:109C10006EC480918307843009F096C089898F5F74
:109C2000898B8989843040F019861A861B861C86A8
:109C300081E0809383075BC429853A854B855C85E9
:109C40006AA07BA08CA09DA068A579A5EAA5FBA52C
:109C50008E8D9F8D9F938F931F921F921F921F92A5
:109C600059016A01EE24FF248701A4019301CF0169
:109C70000E947B480DB71EB70A5F1F4F0FB6F894BE
:109C80001EBF0FBE0DBF99231CF4109283072FC473
:109C90008D859E85AF85B88928A539A54AA15BA188
:109CA0006CA17DA1EAA5FBA57C018D01CF010E94DD
:109CB00034469FA38EA38EA19FA199231CF41092DA
:109CC000830715C48EA19FA1181619060CF00FC4A6
:109CD0008EA19FA128A539A5BC01C9010E945741A9
:109CE0009DA78CA78CA59DA5009709F400C4ECA5A1
:109CF000FDA580818530D1F480917F079091800708
:109D00000E9422418CA59DA59093800780937F0798
:109D10001DA61CA68A8D9B8DAC8DBD8D8E8B9F8BB9
:109D2000A88FB98F85E080938307E1C3ECA5FDA5DB
:109D30008081863009F0DBC319861A861B861C8653
:109D400081E080938307D3C380918307853009F036
:109D500074C0198A88E897E00E94018DE0917F071E
:109D6000F0918007E58CF68C078D10A10E94088A7F
:109D70009B01AC018E899F89A88DB98D39014A015B
:109D8000681A790A8A0A9B0AD401C3018E159F05B5
:109D9000A007B10720F086E080938307A8C3E09175
:109DA0007F07F0918007E58CF68C078D10A10E944B
:109DB000088A9B01AC018E899F89A88DB98D4901C4
:109DC0005A01881A990AAA0ABB0AD501C401570187
:109DD0006801A81AB90ACA0ADB0AD601C5018A8B2A
:109DE0009B8BAC8BBD8B8A899B89AC89BD89883361
:109DF00009E8900701E4A00700E0B00740F087E31E
:109E000099E8A1E4B0E08A8B9B8BAC8BBD8B8A89EF
:109E10009B89AC89BD8928EE33E040E050E0BC016D
:109E2000CD010E94A1F1DC01CB0126E837E0AC01B5
:109E3000BD01C9010E94348B5AC3809183078630CB
:109E400009F027C189898F5F898B8D859E85AF85B4
:109E5000B88928EE33E040E050E0BC01CD010E941B
:109E6000F3F1DA01C9015C016D01E0917F07F09126
:109E70008007E1A0F2A003A114A10E94088A9B011F
:109E8000AC018E899F89A88DB98D39014A01681A64
:109E9000790A8A0A9B0AD401C301A8019701281BE9
:109EA000390B4A0B5B0BDA01C9018A159B05AC051E
:109EB000BD0570F5E0917F07F0918007E1A0F2A069
:109EC00003A114A10E94088A9B01AC018E899F897D
:109ED000A88DB98D39014A01681A790A8A0A9B0A44
:109EE000D401C30128EE33E040E050E0BC01CD01D5
:109EF0000E94A1F1DC01CB0147015801881A990A9F
:109F0000AA0ABB0AD501C4018D879E87AF87B88B8B
:109F1000E0917F07F0918007E1A0F2A003A114A1D6
:109F20000E94088A9B01AC018E899F89A88DB98DFA
:109F300059016A01A81AB90ACA0ADB0AD601C50181
:109F40008E159F05A007B10728F0198A87E0809336
:109F50008307CDC2E0917F07F0918007A180B28096
:109F6000C380D480E0917F07F0918007E180F28088
:109F700003811481E0917F07F0918007618C728CDE
:109F8000838C948C2AA13BA14CA15DA168A579A5E5
:109F9000EAA5FBA58E8D9F8D9F938F931F921F9295
:109FA0001F921F92DF92CF92BF92AF92570168012A
:109FB00079018A019B01B401A301CF010E94AA4744
:109FC0000DB71EB7065F1F4F0FB6F8941EBF0FBE2A
:109FD0000DBF99232CF4198A87E08093830787C2E9
:109FE0008D859E85AF85B88928A539A54AA15BA135
:109FF0006CA17DA1EAA5FBA57C018D01CF010E948A
:10A0000034469FA38EA38EA19FA199231CF4109286
:10A0100083076DC28EA19FA1181619060CF067C2A6
:10A020008EA19FA128A539A5BC01C9010E94574155
:10A030009DA78CA78CA59DA5009709F458C2ECA5F7
:10A04000FDA580818530D1F480917F0790918007B4
:10A050000E9422418CA59DA59093800780937F0745
:10A060001DA61CA68A8D9B8DAC8DBD8D8E8B9F8B66
:10A07000A88FB98F85E08093830739C2ECA5FDA531
:10A080008081863009F033C2198A87E08093830784
:10A090002EC280918307873009F0FDC089898F5FC8
:10A0A000898BE0917F07F0918007E1A0F2A003A1E6
:10A0B00014A10E94088A9B01AC018E899F89A88DFA
:10A0C000B98D39014A01681A790A8A0A9B0AD401B2
:10A0D000C301A8019701281B390B4A0B5B0B8D8527
:10A0E0009E85AF85B889281739074A075B0710F5A1
:10A0F000E0917F07F0918007E1A0F2A003A114A1F5
:10A100000E94088ADC01CB01A8019701281B390BAA
:10A110004A0B5B0B8E899F89A88DB98D49015A0125
:10A12000881A990AAA0ABB0AD501C4018D879E879D
:10A13000AF87B88BE0917F07F0918007E1A0F2A094
:10A1400003A114A10E94088A9B01AC018E899F89FA
:10A15000A88DB98D59016A01A81AB90ACA0ADB0A81
:10A16000D601C5018E159F05A007B10728F0198AF1
:10A1700087E080938307BBC1E0917F07F091800760
:10A18000E180F28003811481E0917F07F0918007E4
:10A1900021813281438154816AA07BA08CA09DA043
:10A1A00068A579A5EAA5FBA58E8D9F8D9F938F93BA
:10A1B0001F921F921F921F925701680179018A0115
:10A1C000A4019301CF010E947B480DB71EB70A5F1F
:10A1D0001F4F0FB6F8941EBF0FBE0DBF99231CF47E
:10A1E0001092830784C18D859E85AF85B88928A587
:10A1F00039A54AA15BA16CA17DA1EAA5FBA57C01C3
:10A200008D01CF010E9434469FA38EA38EA19FA1F2
:10A2100099231CF4109283076AC18EA19FA118167E
:10A2200019060CF064C18EA19FA128A539A5BC0117
:10A23000C9010E9457419DA78CA78CA59DA5009799
:10A2400009F455C1ECA5FDA580818530D1F480913C
:10A250007F07909180070E9422418CA59DA5909335
:10A26000800780937F071DA61CA68A8D9B8DAC8DD1
:10A27000BD8D8E8B9F8BA88FB98F85E080938307D0
:10A2800036C1ECA5FDA58081863009F030C181E0A2
:10A29000809383072CC180918307883009F07EC0AA
:10A2A0001AAA8989843010F011E01AAB89898F5F6E
:10A2B000898B2AA9222319F01092830718C1E8A1DB
:10A2C000F9A187819085A185B2852AA13BA14CA1E6
:10A2D0005DA168A579A56D807E808F809884EAA5B0
:10A2E000FBA55C016D0179018A019B01B401A30109
:10A2F000CF010E945B49992384F48D819E81AF81B7
:10A30000B8858F3F3FEF93073FEFA3073FEFB307BA
:10A3100009F0EDC010928307EAC08D859E85AF8558
:10A32000B88928A539A54AA15BA16CA17DA1EAA5A0
:10A33000FBA57C018D01CF010E9434469FA38EA313
:10A340008EA19FA1009709F4D2C08EA19FA11816DB
:10A3500019060CF58EA19FA128A539A5BC01C9013C
:10A360000E9457419DA78CA78CA59DA5009799F0A9
:10A37000ECA5FDA58081853071F480917F079091D7
:10A3800080070E9422418CA59DA590938007809311
:10A390007F071DA61CA610928307A9C08091830782
:10A3A000893009F089C080917F07909180070097DC
:10A3B000B1F189898F5F898B8989813081F5E0913D
:10A3C0007F07F0918007E18CF28C038D148DE09172
:10A3D0007F07F091800781819281A381B4812AA1B6
:10A3E0003BA14CA15DA168A579A56D807E808F8081
:10A3F0009884EAA5FBA51F930F93FF92EF925C014F
:10A400006D0179018A019B01B401A301CF010E9472
:10A41000E1480F900F900F900F90992384F48D8155
:10A420009E81AF81B8858F3F4FEF94074FEFA40710
:10A430004FEFB40709F05BC01092830758C08D85B9
:10A440009E85AF85B88928A539A54AA15BA16CA1D5
:10A450007DA1EAA5FBA57C018D01CF010E943446B8
:10A460009FA38EA38EA19FA199231CF41092830712
:10A470003EC08EA19FA118161906CCF58EA19FA1F2
:10A4800028A539A5BC01C9010E9457419DA78CA7E9
:10A490008CA59DA5009759F1ECA5FDA5808185307F
:10A4A00019F41092830723C0ECA5FDA580818630A6
:10A4B000F1F4109283071BC0809183078823B9F4BD
:10A4C00080917F07909180070E942241109280071F
:10A4D00010927F07198A88E897E00E94018D86E82C
:10A4E00097E040E050E060E070E00E94348B8CA583
:10A4F0009DA5009709F4A8C88CA59DA50E9422419E
:10A500001DA61CA6A1C8CF93DF93CDB7DEB72D97AC
:10A510000FB6F894DEBF0FBECDBF9E838D836F83D1
:10A52000288739874A875B878D819E810E94208D8D
:10A530009C838B838B819C810097A1F0EB81FC81B4
:10A540008385833079F4EB81FC81878590899A83B8
:10A55000898389819A81009729F0E981FA81808134
:10A56000863059F081E190E09093850780938407CD
:10A570008FEF9FEF9D878C873FC00E94278ADC0169
:10A58000CB0180938E0790938F07A0939007B09391
:10A59000910788859985AA85BB8580938A079093C2
:10A5A0008B07A0938C07B0938D078F8180938307CF
:10A5B0008091810790918207009781F460EB7AE4A3
:10A5C0008B819C81E0ECF3E020E032E0AC01CF0134
:10A5D0000E94788E909382078093810786E897E0A7
:10A5E0000E948A8C88E897E040E050E060E070E0EC
:10A5F0000E94348B1D861C868C859D852D960FB6FA
:10A60000F894DEBF0FBECDBFDF91CF9108956F925A
:10A610007F928F929F92AF92BF92CF92DF92EF92F2
:10A62000FF920F931F93CF93DF93CDB7DEB7A4971D
:10A630000FB6F894DEBF0FBECDBF9A8B898B7C8B93
:10A640006B8B2D8B3E8B4F8B588F89899A890E94FB
:10A65000208D9C838B838B819C810097A1F0EB8163
:10A66000FC818385833079F4EB81FC818785908937
:10A670009A83898389819A81009729F0E981FA81F7
:10A680008081863059F081E190E090938507809336
:10A6900084072FEF3FEF3A8F298F84C1CE010596B3
:10A6A00026E0FC01DF01322F1D923A95E9F7CE0139
:10A6B0000B9646E050E06FEF70E00E940EF189814A
:10A6C0009A819C012F5F3F4FCE01059646E050E0F6
:10A6D000BC01C9010E94F8F0009781F089819A813C
:10A6E0009C012F5F3F4FCE010B9646E050E0BC012E
:10A6F000C9010E94F8F0009709F05FC08B899C891E
:10A70000009711F18B899C89AAE7B8E0BC8FAB8FC9
:10A710009E8F8D8FB6E0BF8FED8DFE8D00802D8DCD
:10A720003E8D2F5F3F4F3E8F2D8FAB8DBC8D0C929A
:10A73000EB8DFC8D3196FC8FEB8FFF8DF150FF8FF1
:10A740002F8D222349F711C089899A890E9410B858
:10A75000009759F082E090E09093850780938407FA
:10A760008FEF9FEF9A8F898F1DC189819A81019602
:10A7700099A388A3AAE7B8E0BBA3AAA3B6E0BCA3A9
:10A78000EAA1FBA100802AA13BA12F5F3F4F3BA381
:10A790002AA3A8A1B9A10C92E8A1F9A13196F9A325
:10A7A000E8A3FCA1F150FCA32CA1222349F764EFFC
:10A7B00071E080E090E00E94038980918C08909184
:10A7C0008D08A0918E08B0918F0820918408309157
:10A7D0008508409186085091870882239323A423FB
:10A7E000B5230097A105B105C1F180918C08909126
:10A7F0008D08A0918E08B0918F0880938008909367
:10A800008108A0938208B093830880918808909172
:10A810008908A0918A08B0918B0820918408309112
:10A820008508409186085091870860908008709054
:10A83000810880908208909083086AE778E0E9892F
:10A84000FA895C016D0179018A01A4019301CF01AC
:10A850000E94FFB61A8E198EA5C08D899E89AF8978
:10A86000B88DE989FA899C01AD0161E0CF010E94B0
:10A870008352009709F092C080918307853009F0D8
:10A8800040C0E0917F07F0918007E584F68407855A
:10A890001089E0917F07F0918007258136814781FB
:10A8A0005085E0917F07F091800781819281A3819B
:10A8B000B481EB81FC816701780189019A01AC01C7
:10A8C000BD01CF010E9448B5E0917F07F09180075C
:10A8D000258936894789508DE0917F07F09180075F
:10A8E00081899289A389B48979018A019C01AD018A
:10A8F00060E070E080E090E00E946B5B1A8E198E41
:10A9000051C0E981FA8187819085A185B285009740
:10A91000A105B10519F01A8E198E44C080918008E6
:10A9200090918108A0918208B091830820918408B9
:10A93000309185084091860850918708822393239F
:10A94000A423B5230097A105B10541F180918808A2
:10A9500090918908A0918A08B0918B082091840871
:10A960003091850840918608509187086090800852
:10A970007090810880908208909083086AE778E060
:10A98000E989FA895C016D0179018A01A4019301C9
:10A99000CF010E94FFB61A8E198E04C08FEF9FEF71
:10A9A0009A8F898F898D9A8DA4960FB6F894DEBF01
:10A9B0000FBECDBFDF91CF911F910F91FF90EF9010
:10A9C000DF90CF90BF90AF909F908F907F906F90CF
:10A9D0000895CF93DF93CDB7DEB728970FB6F894DD
:10A9E000DEBF0FBECDBF9A8389834B835C836D83AB
:10A9F0007E8380918307853059F083E090E09093C7
:10AA00008507809384078FEF9FEF98878F830EC011
:10AA10008B819C81AD81BE81E981FA819C01AD0170
:10AA200069E0CF010E94835298878F838F81988538
:10AA300028960FB6F894DEBF0FBECDBFDF91CF9141
:10AA40000895CF93DF93CDB7DEB728970FB6F8946C
:10AA5000DEBF0FBECDBF9A8389834B835C836D833A
:10AA60007E8380918307882359F083E090E0909360
:10AA70008507809384078FEF9FEF98878F830EC0A1
:10AA80008B819C81AD81BE81E981FA819C01AD0100
:10AA900068E0CF010E94835298878F838F819885C9
:10AAA00028960FB6F894DEBF0FBECDBFDF91CF91D1
:10AAB0000895CF93DF93CDB7DEB722970FB6F89402
:10AAC000DEBF0FBECDBF9A8389838091830799270C
:10AAD00022960FB6F894DEBF0FBECDBFDF91CF91A7
:10AAE0000895CF93DF93CDB7DEB724970FB6F894D0
:10AAF000DEBF0FBECDBF9C838B8380918407909176
:10AB000085079A838983109285071092840789812B
:10AB10009A8124960FB6F894DEBF0FBECDBFDF91A9
:10AB2000CF910895CF93DF93CDB7DEB722970FB6BD
:10AB3000F894DEBF0FBECDBF809183071A821982C1
:10AB4000853021F481E090E09A83898389819A811C
:10AB500022960FB6F894DEBF0FBECDBFDF91CF9126
:10AB60000895CF93DF93CDB7DEB724970FB6F8944F
:10AB7000DEBF0FBECDBF9A8389837C836B838B81BD
:10AB80009C81892F9927E981FA81808389819A8123
:10AB900001969A8389838B81E981FA8180838981F7
:10ABA0009A8101969A83898382E090E024960FB679
:10ABB000F894DEBF0FBECDBFDF91CF910895CF9344
:10ABC000DF93CDB7DEB728970FB6F894DEBF0FBE80
:10ABD000CDBF9E838D8378876F838F819885DC01BD
:10ABE000FD0101900020E9F73197CF018A1B9B0BF3
:10ABF00002969A8389838D819E819C838B838D812C
:10AC00009E8101969E838D83EB81FC8110822EC0F4
:10AC1000EF81F88580818E3291F48D819E819C83B5
:10AC20008B838D819E8101969E838D83EB81FC8138
:10AC300010828F819885019698878F8317C0EF8146
:10AC4000F8858081ED81FE8180838D819E810196D2
:10AC50009E838D838F819885019698878F83EB8162
:10AC6000FC8180818F5FEB81FC818083EF81F8859F
:10AC70008081882369F6ED81FE81108289819A8125
:10AC800028960FB6F894DEBF0FBECDBFDF91CF91EF
:10AC90000895CF93DF93CDB7DEB724970FB6F8941E
:10ACA000DEBF0FBECDBF9A8389837C836B83E9812E
:10ACB000FA8180819927982F8827EB81FC819183E5
:10ACC000808389819A8101969A838983EB81FC81B3
:10ACD00020813181E981FA8180819927822B932B10
:10ACE000EB81FC819183808382E090E024960FB613
:10ACF000F894DEBF0FBECDBFDF91CF910895CF9303
:10AD0000DF93CDB7DEB724970FB6F894DEBF0FBE42
:10AD1000CDBF9A8389837C836B83E981FA818081AB
:10AD20009927AA27BB27EB81FC8180839183A2838B
:10AD3000B38389819A8101969A838983EB81FC810F
:10AD400080819181A281B381BA2FA92F982F882762
:10AD5000EB81FC8180839183A283B383EB81FC81AF
:10AD60002081318142815381E981FA818081992753
:10AD7000AA27BB27822B932BA42BB52BEB81FC811D
:10AD800080839183A283B38389819A8101969A8378
:10AD90008983EB81FC8180819181A281B381BA2F6B
:10ADA000A92F982F8827EB81FC8180839183A28330
:10ADB000B383EB81FC812081318142815381E98120
:10ADC000FA8180819927AA27BB27822B932BA42B5A
:10ADD000B52BEB81FC8180839183A283B38389812E
:10ADE0009A8101969A838983EB81FC81808191818C
:10ADF000A281B381BA2FA92F982F8827EB81FC81DC
:10AE000080839183A283B383EB81FC812081318194
:10AE100042815381E981FA8180819927AA27BB2742
:10AE2000822B932BA42BB52BEB81FC818083918308
:10AE3000A283B38384E090E024960FB6F894DEBF3B
:10AE40000FBECDBFDF91CF910895CF93DF93CDB7E4
:10AE5000DEB72C970FB6F894DEBF0FBECDBF9F8331
:10AE60008E8379876887E885F9858081918100974D
:10AE700051F0E885F985808191810E946A82E88598
:10AE8000F98511821082EE81FF8180819927807C73
:10AE90009070803C910529F482E090E09B878A873E
:10AEA00063C08E819F81DC01FD0101900020E9F7E4
:10AEB0003197CF018A1B9B0B01969C838B838B81DF
:10AEC0009C810E944D81E885F98591838083E88586
:10AED000F985808191819A838983EE81FF818081C8
:10AEE0008D838E819F8101969F838E8333C0EE81F7
:10AEF000FF818081E981FA81808389819A8101962D
:10AF00009A8389838E819F8101969F838E838D8111
:10AF100081508D838D818F3F51F7EE81FF8180813C
:10AF20008D839D819C878C85882311F091E09C877F
:10AF30008C852E813F812F5F3F4F3F832E83882357
:10AF400049F0E981FA818EE2808389819A810196B4
:10AF50009A8389838D818823D1F6E981FA811082D1
:10AF60008B819C819B878A878A859B852C960FB6CF
:10AF7000F894DEBF0FBECDBFDF91CF910895CF9380
:10AF8000DF93CDB7DEB726970FB6F894DEBF0FBEBE
:10AF9000CDBF9A8389837C836B835E834D83EB81F2
:10AFA000FC8180819181009731F0EB81FC8180816F
:10AFB00091810E946A828D819E810E944D81EB81E8
:10AFC000FC8191838083EB81FC8180819181298147
:10AFD0003A81FC018D819E81AC01B901CF010E94B3
:10AFE00005F18D819E8126960FB6F894DEBF0FBEC7
:10AFF000CDBFDF91CF910895CF93DF93CDB7DEB76B
:10B0000024970FB6F894DEBF0FBECDBF9A83898315
:10B010007C836B8389819A81009731F48CE090E086
:10B020000E943E829A83898389819A81009791F058
:10B03000E981FA818B819C8191838083E981FA8106
:10B0400080E091E093838283E981FA8181E090E05E
:10B050009583848389819A8124960FB6F894DEBF04
:10B060000FBECDBFDF91CF910895CF93DF93CDB7C2
:10B07000DEB722970FB6F894DEBF0FBECDBF9A831E
:10B08000898389819A81009721F089819A810E9420
:10B090006A8222960FB6F894DEBF0FBECDBFDF9155
:10B0A000CF910895CF93DF93CDB7DEB726970FB634
:10B0B000F894DEBF0FBECDBF9C838B837E836D83F0
:10B0C000ED81FE81808191812B813C81BC01C90190
:10B0D0000E94B1559A838983ED81FE81428153811B
:10B0E00029813A818B819C81820F931FBA010E9432
:10B0F000B1559C0189819A81820F931F9A8389831C
:10B10000ED81FE814481558129813A818B819C8129
:10B11000820F931FBA010E94B1559C0189819A81C7
:10B12000820F931F9A838983ED81FE814681578127
:10B1300029813A818B819C81820F931FBA010E94E1
:10B14000B1559C0189819A81820F931F9A838983CB
:10B15000ED81FE814085518529813A818B819C81D9
:10B16000820F931FBA010E94B1559C0189819A8177
:10B17000820F931F9A838983ED81FE8142855385D7
:10B1800029813A818B819C81820F931FBA010E9491
:10B19000B1559C0189819A81820F931F9A8389837B
:10B1A00089819A8126960FB6F894DEBF0FBECDBF77
:10B1B000DF91CF910895CF93DF93CDB7DEB7269778
:10B1C0000FB6F894DEBF0FBECDBF9C838B837E830A
:10B1D0006D838B819C812D813E81BC01C9010E94C0
:10B1E00049569A8389838B819C81AC014E5F5F4F66
:10B1F00029813A818D819E81820F931FBA010E941D
:10B2000049569C0189819A81820F931F9A83898371
:10B210008B819C81AC014C5F5F4F29813A818D818C
:10B220009E81820F931FBA010E9449569C01898119
:10B230009A81820F931F9A8389838B819C81AC01B1
:10B240004A5F5F4F29813A818D819E81820F931FD2
:10B25000BA010E9449569C0189819A81820F931FED
:10B260009A8389838B819C81AC01485F5F4F2981E0
:10B270003A818D819E81820F931FBA010E944956A7
:10B280009C0189819A81820F931F9A8389838B8184
:10B290009C81AC01465F5F4F29813A818D819E81FF
:10B2A000820F931FBA010E9449569C0189819A819D
:10B2B000820F931F9A83898389819A8126960FB67C
:10B2C000F894DEBF0FBECDBFDF91CF910895CF932D
:10B2D000DF93CDB7DEB726970FB6F894DEBF0FBE6B
:10B2E000CDBF9A8389837C836B835E834D83898101
:10B2F0009A81009731F486E090E00E943E829A8322
:10B30000898389819A81009799F1E981FA81808105
:10B310009181009731F0E981FA81808191810E94C9
:10B320006A828B819C81DC01FD0101900020E9F79C
:10B330003197CF018A1B9B0B01960E944D81E981B9
:10B34000FA81918380832B813C81E981FA8180811C
:10B350009181B9010E9447F1E981FA818D819E8135
:10B3600093838283E981FA8181E090E095838483ED
:10B3700089819A8126960FB6F894DEBF0FBECDBFA5
:10B38000DF91CF910895CF93DF93CDB7DEB72297AA
:10B390000FB6F894DEBF0FBECDBF9A838983898133
:10B3A0009A81009781F0E981FA81808191810097EB
:10B3B00031F0E981FA81808191810E946A828981DC
:10B3C0009A810E946A8222960FB6F894DEBF0FBE61
:10B3D000CDBFDF91CF910895CF93DF93CDB7DEB787
:10B3E00026970FB6F894DEBF0FBECDBF9C838B832C
:10B3F0007E836D83ED81FE81808191812B813C81F3
:10B40000BC01C9010E94DF559A838983ED81FE81C9
:10B410004281538129813A818B819C81820F931FC4
:10B42000BA010E94B1559C0189819A81820F931FB4
:10B430009A838983ED81FE814481558129813A81F6
:10B440008B819C81820F931FBA010E94B1559C0190
:10B4500089819A81820F931F9A83898389819A8136
:10B4600026960FB6F894DEBF0FBECDBFDF91CF9109
:10B470000895CF93DF93CDB7DEB726970FB6F89434
:10B48000DEBF0FBECDBF9C838B837E836D838B819C
:10B490009C812D813E81BC01C9010E9425579A8360
:10B4A00089838B819C81AC014E5F5F4F29813A81FA
:10B4B0008D819E81820F931FBA010E9449569C0183
:10B4C00089819A81820F931F9A8389838B819C81C2
:10B4D000AC014C5F5F4F29813A818D819E81820F43
:10B4E000931FBA010E9449569C0189819A81820F5B
:10B4F000931F9A83898389819A8126960FB6F8943F
:10B50000DEBF0FBECDBFDF91CF910895CF93DF9304
:10B51000CDB7DEB722970FB6F894DEBF0FBECDBF12
:10B520009A83898389819A81009731F48EE090E033
:10B530000E943E829A83898389819A8122960FB6DE
:10B54000F894DEBF0FBECDBFDF91CF910895CF93AA
:10B55000DF93CDB7DEB722970FB6F894DEBF0FBEEC
:10B56000CDBF9A83898389819A810097E1F0E9812F
:10B57000FA8180819181009731F0E981FA8180819F
:10B5800091810E946A82E981FA818485958500977C
:10B5900031F0E981FA81848595850E946A828981EA
:10B5A0009A810E946A8222960FB6F894DEBF0FBE7F
:10B5B000CDBFDF91CF910895CF93DF93CDB7DEB7A5
:10B5C00026970FB6F894DEBF0FBECDBF9C838B834A
:10B5D0007E836D838B819C812D813E81BC01C9015D
:10B5E0000E9425579A8389838B819C81AC014E5F91
:10B5F0005F4F29813A818D819E81820F931FBA010D
:10B600000E9449569C0189819A81820F931F9A83D7
:10B6100089838B819C81AC014C5F5F4F29813A818A
:10B620008D819E81820F931FBA010E9449569C0111
:10B6300089819A81820F931F9A8389838B819C8150
:10B64000AC014A5F5F4F29813A818D819E81820FD3
:10B65000931FBA010E947F569C0189819A81820FB3
:10B66000931F9A8389838B819C81AC01465F5F4FD6
:10B6700029813A818D819E81820F931FBA010E9498
:10B6800049569C0189819A81820F931F9A838983ED
:10B69000EB81FC81428553858B819C81BC01645F79
:10B6A0007F4F29813A818D819E81820F931F0E9455
:10B6B000BF579C0189819A81820F931F9A83898346
:10B6C00089819A8126960FB6F894DEBF0FBECDBF52
:10B6D000DF91CF910895EF92FF920F931F93CF9335
:10B6E000DF93CDB7DEB72C970FB6F894DEBF0FBE51
:10B6F000CDBF9A8389837C836B832D833E834F8365
:10B700005887E986FA860B871C878091920790916B
:10B710009307009751F080919207909193070E94B0
:10B720006A821092930710929207809194079091E9
:10B730009507009751F080919407909195070E948A
:10B740006A82109295071092940789819A810097D6
:10B75000D9F089819A81DC01FD0101900020E9F78F
:10B760003197CF018A1B9B0B01960E944D819093CC
:10B7700093078093920729813A8180919207909153
:10B780009307B9010E9447F18B819C810097D9F002
:10B790008B819C81DC01FD0101900020E9F731974C
:10B7A000CF018A1B9B0B01960E944D8190939507B8
:10B7B000809394072B813C81809194079091950709
:10B7C000B9010E9447F18D819E81AF81B885809338
:10B7D000960790939707A0939807B0939907898548
:10B7E0009A85AB85BC8580939A0790939B07A0931D
:10B7F0009C07B0939D072C960FB6F894DEBF0FBE42
:10B80000CDBFDF91CF911F910F91FF90EF900895E1
:10B81000EF92FF920F931F93CF93DF93CDB7DEB7D5
:10B8200028970FB6F894DEBF0FBECDBF9A838983E9
:10B830007C836B832D833E834F8358878D819E81CC
:10B84000AF81B8856B817C81E981FA81EE24FF2488
:10B8500087019C01AD01CF010E946B5B28960FB65A
:10B86000F894DEBF0FBECDBFDF91CF911F910F9136
:10B87000FF90EF900895CF93DF93CDB7DEB7229777
:10B880000FB6F894DEBF0FBECDBF9A83898389813E
:10B890009A8161E070E00E94795CDC01CB01BC011F
:10B8A000CD0122960FB6F894DEBF0FBECDBFDF915B
:10B8B000CF910895CF93DF93CDB7DEB722970FB620
:10B8C000F894DEBF0FBECDBF9A83898389819A81A8
:10B8D0006FE070E00E94795CDC01CB01BC01CD011E
:10B8E00022960FB6F894DEBF0FBECDBFDF91CF9189
:10B8F0000895CF92DF92EF92FF920F931F93CF9311
:10B90000DF93CDB7DEB7A4970FB6F894DEBF0FBEB6
:10B91000CDBF9E8F8D8F78A36F8F1B8A1C8A1D8A47
:10B920001E8A1E861D861A86198618861F821E820A
:10B930001D828091960790919707A0919807B091EA
:10B9400099070097A105B10589F480919A07909114
:10B950009B07A0919C07B0919D070097A105B10599
:10B9600029F419A21AA21BA21CA2B6C180E090E081
:10B970000E943BAD9C878B878B859C85009729F423
:10B9800019A21AA21BA21CA2A7C180E092E00E94E9
:10B990004D819A8B898B1A8219827CC18D859E85F7
:10B9A00001969E878D878D859E8529853A85BC0168
:10B9B000C9010E94FC579A8789878F8D98A12D8D88
:10B9C0003E8DEF81F885AC01B901CF010E94675926
:10B9D00098878F8389859A8529893A89BC01C9010D
:10B9E0000E945258988B8F872F85388989899A8928
:10B9F000280F391F8F819885BC01C9010E94EC591D
:10BA00009C018F859889820F931F988B8F878981DE
:10BA10009A8181709070009761F080919A0790915F
:10BA20009B07A0919C07B0919D070097A105B105C8
:10BA3000C9F44091960750919707609198077091CB
:10BA400099078F85988929893A89EB85FC857C013E
:10BA5000890125E330E0CF010E94D6AD99230CF493
:10BA60001FC119C040919A0750919B0760919C0794
:10BA700070919D078F85988929893A89EB85FC8586
:10BA80007C01890125E330E0CF010E94D6AD9923E6
:10BA90000CF406C100C0188A1F8689899A89AE01F4
:10BAA000455E5F4FBE01695E7F4FEB85FC850F2EC3
:10BAB000F8EECF2EF3E0DF2EF0E0EF2EF0E0FF2ED9
:10BAC000F02D00E012E09C01CF010E943FAE9C836C
:10BAD0008B838B819C8118161906CCF48B819C81F9
:10BAE0008D309105C4F289899A8929853A85BC01EE
:10BAF000C9010E94DB58988B8F87E985FA852081E0
:10BB000031818D859E852817390709F0C4CF8F852F
:10BB10009889009709F4B9C0E985FA8584819581EF
:10BB20008130910509F0B1C02F85388989899A89BA
:10BB3000820F931F2F813885BC01C9010E94395A99
:10BB40009C018F859889820F931F988B8F87E98539
:10BB5000FA8586819781009709F4A2C081E090E080
:10BB60009C838B8325C08D819E810E94865A9E83F3
:10BB70008D832F85388989899A89820F931F2D811A
:10BB80003E81BC01C9010E94DC5A9C018F859889C5
:10BB9000820F931F988B8F87ED81FE818281938125
:10BBA0008130910579F08B819C8101969C838B83F8
:10BBB000E985FA85868197819C018B819C81281774
:10BBC00039078CF6ED81FE8182859385843091055D
:10BBD00009F05BC0ED81FE810484F585E02D808154
:10BBE0009927AA27BB278B8B9C8BAD8BBE8BED81B6
:10BBF000FE8184859585FC01319680819927AA274D
:10BC0000BB272227382F492F5A2F8B899C89AD8932
:10BC1000BE89820F931FA41FB51F8B8B9C8BAD8B8E
:10BC2000BE8BED81FE8184859585FC0132968081F5
:10BC30009927AA27BB27AC01332722278B899C8908
:10BC4000AD89BE89820F931FA41FB51F8B8B9C8B60
:10BC5000AD8BBE8BED81FE8184859585FC0133968D
:10BC600080819927AA27BB27582F442733272227CB
:10BC70008B899C89AD89BE89820F931FA41FB51F34
:10BC80008B8B9C8BAD8BBE8B0BC089819A8101966F
:10BC90009A83898389819A81863091050CF47ECEBE
:10BCA00089859A850E9435588F8198850E94C3594D
:10BCB0008D819E810E94A75A89899A890E946A82F1
:10BCC0008B859C850E94EDAE8B899C89AD89BE8950
:10BCD00089A39AA3ABA3BCA389A19AA1ABA1BCA140
:10BCE000BC01CD01A4960FB6F894DEBF0FBECDBF48
:10BCF000DF91CF911F910F91FF90EF90DF90CF9048
:10BD00000895CF93DF93CDB7DEB726970FB6F8949B
:10BD1000DEBF0FBECDBF9C838B837E836D838091FE
:10BD20009E0790919F079A83898327C08B819C816E
:10BD3000009761F0E981FA81828193812B813C81B6
:10BD4000BC01C9010E943EF1009789F48D819E815A
:10BD50000097B9F0E981FA81848195812D813E8136
:10BD6000BC01C9010E943EF1009709F40AC0E981B3
:10BD7000FA81808191819A83898389819A81009750
:10BD8000A9F689819A8126960FB6F894DEBF0FBE78
:10BD9000CDBFDF91CF910895CF93DF93CDB7DEB7BD
:10BDA00028970FB6F894DEBF0FBECDBF9C838B8360
:10BDB0007E836D8386E090E00E944D819A83898323
:10BDC00089819A81009709F45FC080919E079091C4
:10BDD0009F07E981FA81918380838B819C81DC01BB
:10BDE000FD0101900020E9F73197CF018A1B9B0BE1
:10BDF00001960E944D81E981FA8193838283E981D2
:10BE0000FA81828193810097D9F1E981FA812281B7
:10BE100033818B819C81BC01C9010E9447F18D81D6
:10BE20009E81DC01FD0101900020E9F73197CF01EF
:10BE30008A1B9B0B01960E944D81E981FA819583B3
:10BE40008483E981FA8184819581009799F0E98161
:10BE5000FA81248135818D819E81BC01C9010E94B6
:10BE600047F189819A8190939F0780939E07188656
:10BE70001F820EC0E981FA81828193810E946A82C9
:10BE800089819A810E946A828FEF9FEF98878F83C2
:10BE90008F81988528960FB6F894DEBF0FBECDBF70
:10BEA000DF91CF910895CF93DF93CDB7DEB722977F
:10BEB0000FB6F894DEBF0FBECDBF1EC080919E07A7
:10BEC00090919F079A838983E981FA81808191818A
:10BED00090939F0780939E07E981FA8182819381E5
:10BEE0000E946A82E981FA81848195810E946A8236
:10BEF00089819A810E946A8280919E0790919F0712
:10BF00000097E1F622960FB6F894DEBF0FBECDBFC4
:10BF1000DF91CF910895CF93DF93CDB7DEB7289708
:10BF20000FB6F894DEBF0FBECDBF98878F831C82FB
:10BF30001B828FEF9FEF9A838983EF81F88586813B
:10BF400097819E838D838D819E816FE270E00E9438
:10BF500074F19C838B838B819C81009721F0EB8112
:10BF6000FC81108204C086EC93E09E838D838D81DA
:10BF70009E8160E070E00E94815E009759F1EF8140
:10BF8000F88586859785009739F1EF81F8852685B4
:10BF9000378588EC93E046E050E0BC01C9010E947F
:10BFA00066F10097C9F4EF81F88586859785069636
:10BFB0000E94BB60EF81F8858685978506962D8166
:10BFC0003E81BC01C9010E94815E009729F01A825E
:10BFD000198202C01A8219828B819C81009721F0FC
:10BFE000EB81FC818FE2808389819A8128960FB64C
:10BFF000F894DEBF0FBECDBFDF91CF910895CF93F0
:10C00000DF93CDB7DEB728970FB6F894DEBF0FBE2B
:10C01000CDBF9C838B837E836D8386E090E00E94FE
:10C020004D819A83898389819A81009729F48FEFC2
:10C030009FEF98878F831CC08091A0079091A107E4
:10C04000E981FA8191838083E981FA818B819C81E6
:10C0500093838283E981FA818D819E819583848394
:10C0600089819A819093A1078093A00718861F82E7
:10C070008F81988528960FB6F894DEBF0FBECDBF8E
:10C08000DF91CF910895CF93DF93CDB7DEB7269799
:10C090000FB6F894DEBF0FBECDBF9C838B837E832B
:10C0A0006D83ED81FE81808191818130910591F0D8
:10C0B000ED81FE81808191818230910559F08D81E1
:10C0C0009E812B813C8145EF51E0BC01C9010E945A
:10C0D000A96648C08091A0079091A1079A8389839F
:10C0E00016C0ED81FE81868197819C01285F3F4FBC
:10C0F000E981FA8182819381B9010E9415F100974B
:10C1000051F0E981FA81808191819A8389838981C3
:10C110009A81009731F789819A81009759F48D812E
:10C120009E812B813C8144E951E0BC01C9010E9400
:10C13000A96618C0E981FA810480F581E02D8D811E
:10C140009E812B813C81BC01C9010995009751F06A
:10C150008D819E812B813C8144EF51E0BC01C9015E
:10C160000E94A96626960FB6F894DEBF0FBECDBF1B
:10C17000DF91CF910895CF93DF93CDB7DEB72E97A0
:10C180000FB6F894DEBF0FBECDBF9C878B878FEFB5
:10C190008D831C828B859C85998788878885998566
:10C1A0009F838E839DC0E885F985808180320CF461
:10C1B00092C0E885F9858081992787FD90959C013B
:10C1C0008DEB9DE68097820F931F9B838A83EA8184
:10C1D000FB818491898389818A878A858F3F09F4CD
:10C1E0007AC08C81282F332727FD30953E872D87F5
:10C1F0008C818F5F8C838D859E858230910569F15E
:10C200002D853E852330310509F448C08D859E85F6
:10C210008130910509F05DC08D81992787FD90954A
:10C22000880F991F880F991F282F8A85992787FDC6
:10C230009095807390709595879595958795959530
:10C24000879595958795822BEE81FF8180838E81DE
:10C250009F8101969F838E833CC08D81992787FDA6
:10C2600090958F70907082959295907F9827807F9F
:10C270009827282F8A85992787FD90958C73907031
:10C280009595879595958795822BEE81FF81808383
:10C290008E819F8101969F838E831BC08D819927FC
:10C2A00087FD9095837090700024969587950794EC
:10C2B000969587950794982F802D982F8A85892B9E
:10C2C000EE81FF8180838E819F8101969F838E8383
:10C2D0001C828A858D8388859985019699878887B0
:10C2E000E885F9858081882309F05DCFEE81FF81A3
:10C2F00010828B859C852E960FB6F894DEBF0FBEFC
:10C30000CDBFDF91CF910895CF93DF93CDB7DEB747
:10C3100023970FB6F894DEBF0FBECDBF8983898106
:10C3200080336CF089818A3354F48981992787FDA1
:10C3300090959C01205330403B832A8324C08981FF
:10C3400081366CF08981873654F48981992787FD7D
:10C3500090959C01275530403B832A8314C08981E6
:10C3600081346CF08981873454F48981992787FD61
:10C3700090959C01275330403B832A8304C08FEF64
:10C380009FEF9B838A838A819B8123960FB6F894C3
:10C39000DEBF0FBECDBFDF91CF910895CF93DF9366
:10C3A000CDB7DEB72D970FB6F894DEBF0FBECDBF69
:10C3B0009B878A878A859B859D838C838A859B85BD
:10C3C0009B838A83EA85FB858081898389818F327B
:10C3D00009F460C01D861C866FC0EC81FD818081E0
:10C3E000853291F58C819D81FC01319680810E947E
:10C3F0008461998788878885998599232CF18C8118
:10C400009D81FC01329680810E9484619F838E838E
:10C410008E819F819923C4F08C819D8102969D839A
:10C420008C838885998582959295907F9827807FC7
:10C430009827982F8E81890FEC81FD818083EC8174
:10C44000FD818081882389F1EC81FD8180818C359B
:10C4500021F4EC81FD818FE2808389818E3219F095
:10C4600089818F3251F4EC81FD8180818E3291F08F
:10C47000EC81FD8180818F3269F0EC81FD818081CA
:10C480008983EA81FB81898180838A819B810196EE
:10C490009B838A838C819D8101969D838C83EC8113
:10C4A000FD818081882309F098CFEA81FB81108289
:10C4B0008A859B859D878C878C859D852D960FB65B
:10C4C000F894DEBF0FBECDBFDF91CF910895CF931B
:10C4D000DF93CDB7DEB72C970FB6F894DEBF0FBE53
:10C4E000CDBF9A83898389819A8120E8FC01DF018D
:10C4F000822F1D928A95E9F78091AC079091AD0744
:10C50000A091AE07B091AF07E981FA818083918352
:10C51000A283B383E981FA8181E08483E981FA818E
:10C5200080E1858389819A8106969C838B83AAE723
:10C53000B8E0BE83AD83B6E0BF83ED81FE810080AD
:10C540008D819E8101969E838D83AB81BC810C92EF
:10C55000EB81FC813196FC83EB83FF81F150FF83FB
:10C560008F81882351F78091800890918108A09154
:10C570008208B0918308E981FA8184879587A6872C
:10C58000B7878091840890918508A0918608B09122
:10C590008708E981FA81808B918BA28BB38B809184
:10C5A000880890918908A0918A08B0918B08E98148
:10C5B000FA81848B958BA68BB78B80918C08909198
:10C5C0008D08A0918E08B0918F08E981FA81808F43
:10C5D000918FA28FB38F89819A814C969987888792
:10C5E000ACE5B8E0BB87AA87B8E0BC87EA85FB85E5
:10C5F00000808A859B8501969B878A87A885B98557
:10C600000C92E885F9853196F987E887FC85F15029
:10C61000FC878C85882351F784E290E02C960FB636
:10C62000F894DEBF0FBECDBFDF91CF910895CF93B9
:10C63000DF93CDB7DEB72C970FB6F894DEBF0FBEF1
:10C64000CDBF9A83898389819A814C962CE538E005
:10C650003C832B839E838D8330E13F83ED81FE817C
:10C6600000802D813E812F5F3F4F3E832D83EB81E4
:10C67000FC8100822B813C812F5F3F4F3C832B83C9
:10C680003F8131503F838F81882341F70E94E78D9E
:10C6900089819A810696EAE7F8E0F987E8879B871F
:10C6A0008A87F6E0FC87EA85FB8500802A853B8542
:10C6B0002F5F3F4F3B872A87E885F98500822885D1
:10C6C00039852F5F3F4F398728873C8531503C871C
:10C6D0008C85882341F7E981FA8184859585A68533
:10C6E000B7858093800890938108A0938208B093C7
:10C6F0008308E981FA8180899189A289B38980932D
:10C70000840890938508A0938608B0938708E981F0
:10C71000FA8184899589A689B7898093880890933E
:10C720008908A0938A08B0938B08E981FA81808DEB
:10C73000918DA28DB38D80938C0890938D08A093DA
:10C740008E08B0938F080E945CB82C960FB6F894B0
:10C75000DEBF0FBECDBFDF91CF9108950F931F9322
:10C76000CF93DF93CDB7DEB72C970FB6F894DEBF2B
:10C770000FBECDBF6B837C838D839E8358874F8391
:10C780003A8729871C870B878FEF9FEF9A838983CE
:10C790008B859C858432910508F447C0E985FA852C
:10C7A0008481882339F489859A850E9467629A83F7
:10C7B00089833BC0E985FA8584818230B1F5E985BA
:10C7C000FA8520813181428153818091AC0790911B
:10C7D000AD07A091AE07B091AF07281739074A07F8
:10C7E0005B0719F5E985FA8585818031F0F00E94B3
:10C7F000DE899B01AC018091AC079091AD07A091BF
:10C80000AE07B091AF07820F931FA41FB51F80938F
:10C81000AC079093AD07A093AE07B093AF0789859F
:10C820009A850E9417639A83898389819A812C96BD
:10C830000FB6F894DEBF0FBECDBFDF91CF911F9131
:10C840000F910895CF93DF93CDB7DEB760970FB602
:10C85000F894DEBF0FBECDBF988B8F8706C068EE01
:10C8600073E080E090E00E94038980E890E00E94FD
:10C87000A7E89C838B838B819C81009781F306C002
:10C8800068EE73E080E090E00E9403898091A80741
:10C890009091A9070E943BAD9E838D838D819E81DF
:10C8A000009771F380E891E09E878D87CE010D9609
:10C8B000ED81FE8122E030E0AC0162E070E1CF0169
:10C8C0000E9486AFECE7F8E080819181A281B3817C
:10C8D0008093AC079093AD07A093AE07B093AF07DA
:10C8E0000E94DE899B01AC018091AC079091AD075D
:10C8F000A091AE07B091AF07820F931FA41FB51F81
:10C900008093AC079093AD07A093AE07B093AF07A9
:10C910008091AA079091AB0781709070882391F164
:10C920008091AC079091AD07A091AE07B091AF0791
:10C930009770A070B0708C509E4FAF4FBF4FBC012E
:10C94000CD010E9403898B819C810E9467629A833A
:10C95000898389819A8118161906A4F429813A815C
:10C960004091A8075091A9078B819C81ED81FE81A0
:10C9700079018C019A014FEF5FEF6FEF7FEFCF01ED
:10C980000E94D6AD8B819C81AE01455F5F4FBE0199
:10C99000695F7F4FED81FE81CC24DD24760100E8C4
:10C9A00010E09C01CF010E943FAE9A8389832091C1
:10C9B000A4073091A5074091A6075091A7078F8142
:10C9C0009885A985BA85282339234A235B238F813B
:10C9D0009885A985BA85281739074A075B0709F0A2
:10C9E00070C089819A81181619060CF06AC080916E
:10C9F000CF039091D003009709F463C0E091CF0377
:10CA0000F091D0034B855C85CF80D884E984FA848B
:10CA100089819A812B813C818C01C701B6010995DE
:10CA20009A83898389819A81181619060CF049C066
:10CA3000209184083091850840918608509187089C
:10CA40008F819885A985BA8579018A01E822F92222
:10CA50000A231B232091800830918108409182088D
:10CA6000509183088091840890918508A091860850
:10CA7000B091870882239323A423B523E816F906EF
:10CA80000A071B0741F08FEF9FEFAFEFBFEF8F83D8
:10CA90009887A987BA8749815A816091A8077091C0
:10CAA000A9078F819885A985BA852B813C81ED8165
:10CAB000FE817A0189019B01AC01BD01CF010E9479
:10CAC000D6AD64E670E080E090E00E9403895ACF22
:10CAD000CF93DF93CDB7DEB724970FB6F894DEBFC0
:10CAE0000FBECDBF9C838B838091CF039091D003E9
:10CAF0009A8389838B819C819093D0038093CF0309
:10CB000089819A8124960FB6F894DEBF0FBECDBFFF
:10CB1000DF91CF910895CF93DF93CDB7DEB72C97F8
:10CB20000FB6F894DEBF0FBECDBF69837A838B83C7
:10CB30009C835E834D8338872F838091A2079091D9
:10CB4000A307009709F03EC089819A81AB81BC811F
:10CB50008093A4079093A507A093A607B093A70777
:10CB60008D819E81009729F08D819E819C878B8786
:10CB700004C08EE496E29C878B878B859C8590937E
:10CB8000A9078093A8078F8198859093AB0780931E
:10CB9000AA0782E294E6E1EDF3E020E831E040E02C
:10CBA00050E0BC01CF010E94788E9093A307809340
:10CBB000A2078091A2079091A307009719F01A8607
:10CBC000198604C08FEF9FEF9A87898789859A8598
:10CBD0002C960FB6F894DEBF0FBECDBFDF91CF917C
:10CBE0000895EF92FF920F931F93CF93DF93CDB7EA
:10CBF000DEB728970FB6F894DEBF0FBECDBF9A837D
:10CC000089837C836B835E834D8338872F830E9467
:10CC1000248E8C01EB81FC81828193812AE030E0BB
:10CC2000B9010E94E0F17C01EB81FC81828193815A
:10CC30002AE030E0B9010E94E0F1CB019C011F9392
:10CC40000F938F8198859F938F938D819E819F9362
:10CC50008F93FF92EF923F932F938DE19EE69F93E8
:10CC60008F9389819A819F938F930E9405E88DB756
:10CC70009EB70E960FB6F8949EBF0FBE8DBF289636
:10CC80000FB6F894DEBF0FBECDBFDF91CF911F91DD
:10CC90000F91FF90EF900895CF93DF93CDB7DEB75C
:10CCA00028970FB6F894DEBF0FBECDBF9A83898355
:10CCB0007C836B832D833E834F8358878B819C813C
:10CCC0000097B1F08B819C819F938F9381E79EE6C3
:10CCD0009F938F9389819A819F938F930E9405E8F8
:10CCE0008DB79EB706960FB6F8949EBF0FBE8DBF48
:10CCF0008D819E81AF81B885BB23D4F08D819E81CB
:10CD0000AF81B885BF93AF939F938F938BE59EE6DA
:10CD10009F938F9389819A819F938F930E9405E8B7
:10CD20008DB79EB708960FB6F8949EBF0FBE8DBF05
:10CD300089819A8125E43EE6BC01C9010E942BE865
:10CD400028960FB6F894DEBF0FBECDBFDF91CF910E
:10CD50000895CF93DF93CDB7DEB72E970FB6F89433
:10CD6000DEBF0FBECDBF98878F837A8769875C87C8
:10CD70004B878B859C859E878D878D859E8521E041
:10CD80008439920751F18D859E8521E0853992077E
:10CD90006CF48D859E8521E080399207A1F08D8508
:10CDA0009E8521E08139920799F026C08D859E8568
:10CDB00021E0843F9207B1F08D859E8521E0853F7B
:10CDC0009207A9F019C08CEC94E09E838D8318C063
:10CDD00088ED94E09E838D8313C085EE94E09E835E
:10CDE0008D830EC08FEE94E09E838D8309C08EEFFD
:10CDF00094E09E838D8304C08EE095E09E838D83B6
:10CE00008D819E814B855C8569857A85EF81F8856A
:10CE10009C01CF010E94F1658B859C8521E08139C1
:10CE20009207D1F51C821B82E985FA85868197815C
:10CE30009A83898389819A816FE270E00E9474F1FC
:10CE40009C838B838B819C81009721F0EB81FC81FB
:10CE5000108204C084E195E09A83898389819A8154
:10CE60009F938F9384E89EE69F938F938F819885FD
:10CE70009F938F930E9405E88DB79EB706960FB6D5
:10CE8000F8949EBF0FBE8DBF8B819C81009721F0CF
:10CE9000EB81FC818FE280838DEE93E0EF81F8855A
:10CEA0002FEF3FEF4FEF5FEFBC01CF010E944C66C9
:10CEB0008D819E819F938F938B859C859F938F936C
:10CEC0008D819E819F938F938B859C859F938F935C
:10CED00089EA9EE69F938F938F8198859F938F9386
:10CEE0000E9405E88DB79EB70C960FB6F8949EBFCA
:10CEF0000FBE8DBF2E960FB6F894DEBF0FBECDBF0E
:10CF0000DF91CF910895CF93DF93CDB7DEB7289708
:10CF10000FB6F894DEBF0FBECDBF9E838D838D818B
:10CF20009E81009789F08D819E81DC01FD01019039
:10CF30000020E9F73197CF018A1B9B0B9A838983E5
:10CF400089819A81009739F420918C0430918D0465
:10CF500038872F835BC01C821B824CC02B813C8195
:10CF6000C901880F991F820F931F880F991FFC0119
:10CF7000EC57FB4F4081518169817A812B813C8143
:10CF8000C901880F991F820F931F880F991FFC01F9
:10CF9000EC57FB4F80819181DC01FD010190002065
:10CFA000E9F73197CF018A1B9B0B9B01281B390B9B
:10CFB000C9019C018D819E81820F931FBA010E943D
:10CFC00015F1009791F42B813C81C901880F991FBD
:10CFD000820F931F880F991FFC01EA57FB4F0190A6
:10CFE000F081E02DF887EF8311C08B819C81019641
:10CFF0009C838B838B819C818C30910508F4AECF10
:10D00000809186049091870498878F838F8198857B
:10D0100028960FB6F894DEBF0FBECDBFDF91CF913B
:10D020000895CF93DF93CDB7DEB728970FB6F89466
:10D03000DEBF0FBECDBF9E838D838D819E81009705
:10D0400089F08D819E81DC01FD0101900020E9F7CE
:10D050003197CF018A1B9B0B9A83898389819A819F
:10D06000009739F420918E0430918F0438872F83F4
:10D070005BC01C821B824CC02B813C81C901880F84
:10D08000991F820F931F880F991FFC01EC57FB4FCC
:10D090004081518169817A812B813C81C901880F4E
:10D0A000991F820F931F880F991FFC01EC57FB4FAC
:10D0B00080819181DC01FD0101900020E9F7319729
:10D0C000CF018A1B9B0B9B01281B390BC9019C01BB
:10D0D0008D819E81820F931FBA010E9415F10097E6
:10D0E00091F42B813C81C901880F991F820F931FF6
:10D0F000880F991FFC01E857FB4F0190F081E02D4C
:10D10000F887EF8311C08B819C8101969C838B8370
:10D110008B819C818C30910508F4AECF809188047E
:10D120009091890498878F838F81988528960FB670
:10D13000F894DEBF0FBECDBFDF91CF910895CF939E
:10D14000DF93CDB7DEB728970FB6F894DEBF0FBEDA
:10D15000CDBF9C838B837E836D838B819C81009765
:10D1600029F481E090E098878F833AC01A8219826F
:10D170002EC029813A81C901880F991F820F931F00
:10D18000880F991FFC01EC57FB4F808191812B8107
:10D190003C81BC01C9010E9415F1009799F42981D5
:10D1A0003A81C901880F991F820F931F880F991F19
:10D1B000FC01E857FB4F8D819E8191838083188607
:10D1C0001F820EC089819A8101969A838983898101
:10D1D0009A818C30910568F281E090E098878F8386
:10D1E0008F81988528960FB6F894DEBF0FBECDBF0D
:10D1F000DF91CF910895CF93DF93CDB7DEB72C9712
:10D200000FB6F894DEBF0FBECDBF9E838D831A820A
:10D2100019828D819E81009719F41C861B86FDC0A2
:10D220008D819E819A87898741C0E985FA858081B1
:10D23000992787FD90950E9415F2009769F1E9857D
:10D24000FA858081853241F1E985FA8580818632CF
:10D2500019F1E985FA8580818B32F1F0E985FA854B
:10D2600080818C32C9F0E985FA8580818A33A1F00A
:10D27000E985FA8580818B3379F0E985FA858081AB
:10D280008D3351F0E985FA8580818F3329F0E98566
:10D29000FA858081803429F489819A8101969A8364
:10D2A000898389859A8501969A878987E985FA8590
:10D2B0008081882309F0B9CF8D819E81DC01FD0139
:10D2C00001900020E9F731979F012A1B3B0B8981D0
:10D2D0009A81880F991F820F931F01960E944D819A
:10D2E0009C838B838B819C8198878F83ED81FE81CA
:10D2F000FA87E98785C0E985FA858081992787FDC6
:10D3000090950E9415F2009769F5E985FA8580816C
:10D31000853241F1E985FA858081863219F1E98506
:10D32000FA8580818B32F1F0E985FA8580818C3233
:10D33000C9F0E985FA8580818A33A1F0E985FA850B
:10D3400080818B3379F0E985FA8580818D3351F0C6
:10D35000E985FA8580818F3329F0E985FA85808116
:10D36000803461F4E985FA858081EF81F8858083D6
:10D370008F819885019698878F833DC085E2EF81E4
:10D38000F88580838F819885019698878F83E985BA
:10D39000FA8580818595859585958595992787FD61
:10D3A00090959C018091270590912805F901E80F3F
:10D3B000F91F8081EF81F88580838F8198850196A0
:10D3C00098878F83E985FA858081992787FD9095D5
:10D3D0008F7090709C018091270590912805F9012C
:10D3E000E80FF91F8081EF81F88580838F81988510
:10D3F000019698878F83E985FA853196FA87E987C0
:10D40000E985FA858081882309F075CFEF81F88559
:10D4100010828B819C819C878B878B859C852C9629
:10D420000FB6F894DEBF0FBECDBFDF91CF91089548
:10D43000CF93DF93CDB7DEB72E970FB6F894DEBF4C
:10D440000FBECDBF9D838C83CE0101969B878A87BB
:10D45000E9E2F5E0FD87EC87F3E0FE87EC85FD85EA
:10D4600000808C859D8501969D878C87EA85FB854C
:10D4700000828A859B8501969B878A879E8591502D
:10D480009E87EE85EE2351F78C819D819F838E834D
:10D49000EE81FF81F987E88746C0E885F9858081BC
:10D4A0008B3251F480E2EE81FF8180838E819F81F7
:10D4B00001969F838E8332C0E885F985808185320D
:10D4C00011F5E885F985319680818983E885F985AC
:10D4D000329680818A8340E150E060E070E0CE01C6
:10D4E00001960E947EEFDC01CB01EE81FF818083FB
:10D4F0008E819F8101969F838E83E885F985329680
:10D50000F987E8870BC0E885F9858081EE81FF8186
:10D5100080838E819F8101969F838E83E885F98524
:10D520003196F987E887E885F9858081882309F0B5
:10D53000B4CFEE81FF8110822E960FB6F894DEBF35
:10D540000FBECDBFDF91CF910895CF93DF93CDB7BD
:10D55000DEB726970FB6F894DEBF0FBECDBF9A8315
:10D560008983E981FA8180859185009709F405C155
:10D57000E981FA8181E090E0958B848BE981FA81E1
:10D580000084F185E02DFC83EB8314C0EB81FC81EA
:10D590008081863249F4E981FA81848995890196EE
:10D5A000E981FA81958B848B2B813C812F5F3F4FE2
:10D5B0003C832B83EB81FC818081882339F7E981CF
:10D5C000FA8184899589880F991F880F991F0E9475
:10D5D0004D81E981FA81938B828BE981FA8182897D
:10D5E0009389009729F4E981FA81158A148AC5C0C4
:10D5F000E981FA81A289B389E981FA8180859185DF
:10D6000011969C938E93E981FA8182899389FC011A
:10D61000329611821082E981FA810084F185E02D31
:10D62000FC83EB8322E030E03E832D8331C0EB812D
:10D63000FC818081863239F5E981FA81228933893A
:10D640008D819E81880F991FF901E80FF91F8B8149
:10D650009C81019691838083E981FA8122893389B3
:10D660008D819E81880F991F820F931FFC01329636
:10D6700011821082EB81FC8110822D813E812E5F10
:10D680003F4F3E832D838B819C8101969C838B83AE
:10D69000EB81FC818081882351F61E821D8263C04C
:10D6A000E981FA81228933898D819E81880F991FB2
:10D6B000880F991FF901E80FF91F0190F081E02D03
:10D6C000FC83EB8334C0EB81FC8180818D3349F591
:10D6D000E981FA81228933898D819E81880F991F82
:10D6E000880F991F820F931FFC0132968B819C81BA
:10D6F000019691838083EB81FC811082E981FA811C
:10D70000228933898D819E81880F991F880F991FE7
:10D71000820F931FFC013296808191810E94186ACA
:10D720000BC02B813C812F5F3F4F3C832B83EB81D0
:10D73000FC818081882339F6E981FA812289338945
:10D740008D819E81880F991F880F991FF901E80F1D
:10D75000F91F808191810E94186A2D813E812F5F7F
:10D760003F4F3E832D83E981FA8184899589ED813C
:10D77000FE81E817F9070CF493CF26960FB6F894BC
:10D78000DEBF0FBECDBFDF91CF910895CF93DF9362
:10D79000CDB7DEB728970FB6F894DEBF0FBECDBF6A
:10D7A0009A8389837C836B83EB81FC81808591855F
:10D7B000009709F061C189819A81009709F45CC1E1
:10D7C000EB81FC81808191818230910509F054C107
:10D7D000EB81FC818481958101960E943E82EB81E0
:10D7E000FC8191878087EB81FC8180859185009702
:10D7F00059F4EB81FC81158A148AEB81FC818085C8
:10D8000091850E946A8238C118861F8221C0EB81EF
:10D81000FC81848195812F813885821B930BAC011B
:10D82000EB81FC81208531858F819885F901E80F96
:10D83000F91F89819A819C0161E070E0CF010E940B
:10D8400039E69C018F819885820F931F98878F837B
:10D85000EB81FC8184819581EF81F885E817F907D8
:10D86000B4F2EB81FC8181E090E0958B848BEB81BD
:10D87000FC810084F185E02DFE83ED8314C0ED81F1
:10D88000FE818081863249F4EB81FC81848995890F
:10D890000196EB81FC81958B848B2D813E812F5FDE
:10D8A0003F4F3E832D83ED81FE818081882339F7B0
:10D8B000EB81FC8184899589880F991F880F991FB6
:10D8C0000E944D81EB81FC81938B828BEB81FC81EB
:10D8D00082899389009759F4EB81FC81158A148A17
:10D8E000EB81FC81808591850E946A82C5C0EB81B5
:10D8F000FC81A289B389EB81FC8180859185119699
:10D900009C938E93EB81FC8182899389FC013296F2
:10D9100011821082EB81FC810084F185E02DFE8371
:10D92000ED8322E030E038872F8331C0ED81FE8126
:10D930008081863239F5EB81FC81228933898F81A0
:10D940009885880F991FF901E80FF91F8D819E8135
:10D95000019691838083EB81FC81228933898F81B9
:10D960009885880F991F820F931FFC0132961182B0
:10D970001082ED81FE8110822F8138852E5F3F4F0E
:10D9800038872F838D819E8101969E838D83ED81C3
:10D99000FE818081882351F618861F8263C0EB8147
:10D9A000FC81228933898F819885880F991F880F80
:10D9B000991FF901E80FF91F0190F081E02DFE8316
:10D9C000ED8334C0ED81FE8180818D3349F5EB819B
:10D9D000FC81228933898F819885880F991F880F50
:10D9E000991F820F931FFC0132968D819E810196B3
:10D9F00091838083ED81FE811082EB81FC812289FD
:10DA000033898F819885880F991F880F991F820FFE
:10DA1000931FFC013296808191810E94186A0BC08D
:10DA20002D813E812F5F3F4F3E832D83ED81FE810F
:10DA30008081882339F6EB81FC81228933898F81AB
:10DA40009885880F991F880F991FF901E80FF91F12
:10DA5000808191810E94186A2F8138852F5F3F4F06
:10DA600038872F83EB81FC8184899589EF81F88544
:10DA7000E817F9070CF493CF28960FB6F894DEBF99
:10DA80000FBECDBFDF91CF910895CF93DF93CDB778
:10DA9000DEB728970FB6F894DEBF0FBECDBF9C83CC
:10DAA0008B837E836D831A82198230C0EB81FC8167
:10DAB0002289338989819A81880F991F880F991F3C
:10DAC000F901E80FF91F208131818D819E81BC0110
:10DAD000C9010E943EF10097A1F4EB81FC812289EB
:10DAE000338989819A81880F991F880F991F820F26
:10DAF000931FFC0132960190F081E02DF887EF83AF
:10DB000010C089819A8101969A838983EB81FC8177
:10DB10002489358989819A81821793073CF2188676
:10DB20001F828F81988528960FB6F894DEBF0FBEAE
:10DB3000CDBFDF91CF910895CF93DF93CDB7DEB7FF
:10DB400022970FB6F894DEBF0FBECDBF9A838983AC
:10DB5000E981FA818489958922960FB6F894DEBF0F
:10DB60000FBECDBFDF91CF910895CF93DF93CDB797
:10DB7000DEB726970FB6F894DEBF0FBECDBF9A83EF
:10DB800089837C836B838B819C81992354F0898169
:10DB90009A810E949C6D9C018B819C8182179307C6
:10DBA0001CF01E821D8212C0E981FA81228933890C
:10DBB0008B819C81880F991F880F991FF901E80FAD
:10DBC000F91F0190F081E02DFE83ED838D819E8110
:10DBD00026960FB6F894DEBF0FBECDBFDF91CF9172
:10DBE0000895CF93DF93CDB7DEB726970FB6F8949D
:10DBF000DEBF0FBECDBF9A8389837C836B838B810D
:10DC00009C81992354F089819A810E949C6D9C018A
:10DC10008B819C81821793071CF01E821D8213C08A
:10DC2000E981FA81228933898B819C81880F991F30
:10DC3000880F991F820F931FFC0132960190F0818B
:10DC4000E02DFE83ED838D819E8126960FB6F8949C
:10DC5000DEBF0FBECDBFDF91CF9108950F931F930D
:10DC6000CF93DF93CDB7DEB7A7970FB6F894DEBF9B
:10DC70000FBECDBF9E8B8D8B788F6F8B18861F82CA
:10DC80008F89988D0E948B5F009759F08F89988DAE
:10DC90002D893E8941E951E0BC01C9010E94A96674
:10DCA00019C3EF89F88D268137818CE295E048E031
:10DCB00050E0BC01C9010E944EF1009749F48F89E0
:10DCC000988D2D893E89BC01C9010E94436002C321
:10DCD0008091B0079091B107009761F18091B007F2
:10DCE0009091B107DC01FD0101900020E9F7319727
:10DCF0009F012A1B3B0BEF89F88D86819781DC0100
:10DD0000FD0101900020E9F73197CF018A1B9B0BA1
:10DD1000820F931F01960E944D8198878F83809177
:10DD2000B0079091B1072F813885BC01C9010E94CD
:10DD300047F132C0EF89F88D86819781DC01FD01C2
:10DD400001900020E9F73197CF018A1B9B0B0696C3
:10DD50000E944D8198878F838F8198859A8F898FB4
:10DD600085E395E09C8F8B8F96E09D8FEB8DFC8DEE
:10DD700000808B8D9C8D01969C8F8B8FE98DFA8D09
:10DD80000082898D9A8D01969A8F898F9D8D9150F1
:10DD90009D8FED8DEE2351F7EF89F88D8681978168
:10DDA0002F813885BC01C9010E9428F18F81988597
:10DDB0000E9411689E838D838F81988560E070E852
:10DDC0000E9499E09C8B8B8B8F8198850E946A8240
:10DDD0008B899C89FFEF8F3F9F0709F0B8C1EF89BE
:10DDE000F88D86819781DC01FD0101900020E9F723
:10DDF0003197CF018A1B9B0B9A83898389819A81F2
:10DE00000C960E943E829C838B838B819C81009721
:10DE100059F48F89988D2D893E8944EF51E0BC01DA
:10DE2000C9010E94A96656C289819A81009751F062
:10DE3000EF89F88D868197812B813C81BC01C901D6
:10DE40000E9447F189819A81009799F029813A814E
:10DE50008B819C81820F931FFC01319780818F32CF
:10DE600041F08BE395E02B813C81BC01C9010E940C
:10DE700028F18DE395E02B813C81BC01C9010E9412
:10DE800028F18091B0079091B107009751F18091EE
:10DE9000B0079091B107DC01FD0101900020E9F786
:10DEA00031979F012A1B3B0B8B819C81DC01FD017B
:10DEB00001900020E9F73197CF018A1B9B0B820F5D
:10DEC000931F01960E944D8198878F838091B007A0
:10DED0009091B1072F813885BC01C9010E9447F19B
:10DEE00030C08B819C81DC01FD0101900020E9F7AD
:10DEF0003197CF018A1B9B0B06960E944D81988714
:10DF00008F838F8198859F8F8E8F85E395E099A36E
:10DF100088A396E09AA3E8A1F9A1008088A199A11D
:10DF2000019699A388A3EE8DFF8D00828E8D9F8D23
:10DF300001969F8F8E8F9AA191509AA3EAA1EE230A
:10DF400051F78B819C812F813885BC01C9010E94CA
:10DF500028F18B819C810E946A828F8198850E9422
:10DF600011689E838D838F81988560E070E80E94A0
:10DF700099E09C8B8B8B8F8198850E946A828B891C
:10DF80009C89FFEF8F3F9F0709F0E1C0EF89F88D73
:10DF900086819781DC01FD0101900020E9F731972E
:10DFA000CF018A1B9B0B9A83898389819A810D9665
:10DFB0000E943E829C838B838B819C81009759F4C5
:10DFC0008F89988D2D893E8944EF51E0BC01C901AC
:10DFD0000E94A9667FC189819A81009751F0EF89DB
:10DFE000F88D868197812B813C81BC01C9010E94FB
:10DFF00047F189819A81009799F029813A818B8133
:10E000009C81820F931FFC01319780818F3241F0F8
:10E010008BE395E02B813C81BC01C9010E9428F172
:10E0200088E495E02B813C81BC01C9010E9428F164
:10E030008091B0079091B107009751F18091B0079E
:10E040009091B107DC01FD0101900020E9F73197C3
:10E050009F012A1B3B0B8B819C81DC01FD01019000
:10E060000020E9F73197CF018A1B9B0B820F931F8A
:10E0700001960E944D8198878F838091B00790917F
:10E08000B1072F813885BC01C9010E9447F130C01A
:10E090008B819C81DC01FD0101900020E9F7319723
:10E0A000CF018A1B9B0B06960E944D8198878F8318
:10E0B0008F8198859CA38BA385E395E09EA38DA378
:10E0C00096E09FA3EDA1FEA100808DA19EA10196E7
:10E0D0009EA38DA3EBA1FCA100828BA19CA1019624
:10E0E0009CA38BA39FA191509FA3EFA1EE2351F777
:10E0F0008B819C812F813885BC01C9010E9428F148
:10E100008B819C810E946A828F8198850E94116810
:10E110009E838D838F81988560E070E80E9499E0EE
:10E120009C8B8B8B8F8198850E946A828B899C89BE
:10E13000FFEF8F3F9F0759F48F89988D2D893E8976
:10E1400044E951E0BC01C9010E94A966C3C08B89A2
:10E150009C890E94A8E2DC01CB0189879A87AB8762
:10E16000BC878D819E81009709F082C084E595E08F
:10E170006F89788DED89FE899C0148EC50E0CF01D4
:10E180000E94F165EF89F88D868197810E948367EF
:10E19000BC0189859A85AB85BC85ED89FE899C018A
:10E1A000AD01CF010E944C66EF89F88D808191818D
:10E1B0008330910509F48AC080E092E09E878D87C4
:10E1C0008D859E850E944D81988B8F878F8598893C
:10E1D000009709F47BC03EC089859A85AB85BC85D4
:10E1E000803022E0920720E0A20720E0B20724F46A
:10E1F00089859A859E878D878D859E852F8538890F
:10E20000EB89FC89AC01B901CF010E941BE19A8B1B
:10E21000898B49895A898D899E89EF85F8899C0166
:10E2200061E070E0CF010E9426E70097E1F0898964
:10E230009A899C01442737FD4095542F89859A85FA
:10E24000AB85BC85821B930BA40BB50B89879A8782
:10E25000AB87BC8789859A85AB85BC850097A1056E
:10E26000B10509F0B9CF8F8598890E946A822EC0C6
:10E2700084E595E06F89788DED89FE899C0148ECF5
:10E2800050E0CF010E94F165EF89F88D868197817A
:10E290000E948367ED89FE892FEF3FEF4FEF5FEF1D
:10E2A000BC01CF010E944C662091B0073091B107AC
:10E2B00049855A858F89988D6B897C89ED89FE897E
:10E2C000AD81BE818C01CF01FD0109958B899C89AF
:10E2D0000E9407E0A7960FB6F894DEBF0FBECDBF31
:10E2E000DF91CF911F910F910895CF93DF93CDB719
:10E2F000DEB722970FB6F894DEBF0FBECDBF9A836C
:10E30000898305C089819A8101969A838983E981ED
:10E31000FA818081882351F0E981FA8180818032FD
:10E3200029F0E981FA818081893061F7E981FA81F8
:10E330008081882371F0E981FA81108289819A8134
:10E3400001969A83898305C089819A8101969A836F
:10E350008983E981FA8180818032B1F3E981FA8190
:10E360008081893089F389819A8122960FB6F89449
:10E37000DEBF0FBECDBFDF91CF910895CF93DF9366
:10E38000CDB7DEB786E190E00E943E82DF91CF916B
:10E390000895CF93DF93CDB7DEB722970FB6F894E9
:10E3A000DEBF0FBECDBF9A838983E981FA81868162
:10E3B0009781009731F0E981FA81868197810E94E7
:10E3C0006A82E981FA8180859185009731F0E9813F
:10E3D000FA81808591850E946A82E981FA8182852D
:10E3E0009385009731F0E981FA81828593850E94B7
:10E3F0006A82E981FA8184859585009731F0E98107
:10E40000FA81848595850E946A82E981FA818685F0
:10E410009785009731F0E981FA81868597850E947A
:10E420006A82E981FA8180899189009731F0E981D6
:10E43000FA81808991890E946A82E981FA818289C0
:10E440009389009731F0E981FA81828993890E944A
:10E450006A8289819A810E946A8222960FB6F89414
:10E46000DEBF0FBECDBFDF91CF910895CF93DF9375
:10E47000CDB7DEB724970FB6F894DEBF0FBECDBF81
:10E480009C838B838091B0079091B107009731F006
:10E490008091B0079091B1070E946A828B819C8124
:10E4A000009759F18B819C81DC01FD0101900020D6
:10E4B000E9F73197CF018A1B9B0B9A838983898166
:10E4C0009A810097D1F089819A8101960E944D81AD
:10E4D0009093B1078093B0078091B0079091B107F6
:10E4E000009779F02091B0073091B1078B819C8122
:10E4F000BC01C9010E9447F104C01092B1071092FB
:10E50000B00780E090E024960FB6F894DEBF0FBE0F
:10E51000CDBFDF91CF910895CF93DF93CDB7DEB715
:10E520002E970FB6F894DEBF0FBECDBF9E878D87A6
:10E530000E94BE719C878B878B859C85009709F410
:10E54000F6C280E091E00E944D819A878987898593
:10E550009A85009729F48B859C850E94C971E7C232
:10E560008D859E8529853A85AC0160E071E0C90101
:10E570000E94E2E589859A856DE070E00E9433F1A2
:10E580009A83898389819A81009719F0E981FA81B8
:10E59000108289859A856AE070E00E9433F19A833F
:10E5A000898389819A81009719F0E981FA81108223
:10E5B00080E091E00E944D819E838D838D819E81BC
:10E5C000009749F489859A850E946A828B859C858B
:10E5D0000E94C971ACC28D859E852D813E81AC01A2
:10E5E00060E071E0C9010E94E2E5009709F481C191
:10E5F0008D819E816DE070E00E9433F19A83898362
:10E6000089819A81009719F0E981FA8110828D81C0
:10E610009E816AE070E00E9433F19A838983898148
:10E620009A81009719F0E981FA811082ED81FE81CB
:10E630008081882309F45DC187E595E02D813E81C5
:10E640004EE050E0BC01C9010E944EF1009709F074
:10E6500040C0EB85FC8586859785009709F0BBCF88
:10E660008D819E810E969A83898305C089819A81C6
:10E6700001969A838983E981FA8180818032B1F39E
:10E68000E981FA818081893089F389819A81DC016D
:10E69000FD0101900020E9F73197CF018A1B9B0B08
:10E6A00001960E944D81EB85FC8597878687EB85D7
:10E6B000FC8586859785009709F41BC1EB85FC8551
:10E6C0002685378589819A81BC01C9010E9447F15D
:10E6D00082CF86E695E02D813E814FE050E0BC017F
:10E6E000C9010E944EF10097F1F48D819E810F9631
:10E6F0009A83898305C089819A8101969A83898347
:10E70000E981FA8180818032B1F3E981FA818081E7
:10E71000893089F389819A810E94ABF0EB85FC8571
:10E720009583848358CF86E795E02D813E814DE027
:10E7300050E0BC01C9010E944EF1009709F040C0B1
:10E74000EB85FC8582859385009709F044CF8D8108
:10E750009E810D969A83898305C089819A8101964D
:10E760009A838983E981FA8180818032B1F3E981DA
:10E77000FA818081893089F389819A81DC01FD01E8
:10E7800001900020E9F73197CF018A1B9B0B01967E
:10E790000E944D81EB85FC8593878287EB85FC8504
:10E7A00082859385009709F4A4C0EB85FC852285BA
:10E7B000338589819A81BC01C9010E9447F10BCF41
:10E7C00084E895E02D813E8147E050E0BC01C9011D
:10E7D0000E944EF1009709F040C0EB85FC858485CE
:10E7E0009585009709F0F7CE8D819E8107969A83D3
:10E7F000898305C089819A8101969A838983E981F9
:10E80000FA8180818032B1F3E981FA818081893097
:10E8100089F389819A81DC01FD0101900020E9F7EB
:10E820003197CF018A1B9B0B01960E944D81EB858E
:10E83000FC8595878487EB85FC8584859585009785
:10E8400009F457C0EB85FC852485358589819A813B
:10E85000BC01C9010E9447F1BECE8CE895E02D8134
:10E860003E814BE050E0BC01C9010E944EF100978F
:10E8700009F0B1CEEB85FC8580899189009709F07C
:10E88000AACE8D819E810B969A83898305C089814A
:10E890009A8101969A838983E981FA818081803205
:10E8A000B1F3E981FA818081893089F389819A8184
:10E8B000DC01FD0101900020E9F73197CF018A1BAF
:10E8C0009B0B01960E944D81EB85FC85918B808B83
:10E8D000EB85FC8580899189009759F0EB85FC8553
:10E8E0002089318989819A81BC01C9010E9447F13F
:10E8F00072CE8D819E810E946A8289859A850E944E
:10E90000757198878F838F8198850E9475719C831C
:10E910008B838B819C810E94757188E995E02985A4
:10E920003A85BC01C9010E9415F1009739F4EB85C5
:10E93000FC8581E090E09183808335C08CE995E08F
:10E9400029853A85BC01C9010E9415F1009739F467
:10E95000EB85FC8583E090E09183808324C081EA8D
:10E9600095E029853A85BC01C9010E9415F10097FF
:10E9700039F4EB85FC8582E090E09183808313C0BD
:10E9800089859A850E946A828B859C852D853E8526
:10E9900045EF51E0BC01C9010E94A9668B859C85A9
:10E9A0000E94C971C4C0EF81F8858081882329F055
:10E9B000EB81FC818081882399F489859A850E9466
:10E9C0006A828B859C852D853E8540E951E0BC019E
:10E9D000C9010E94A9668B859C850E94C971A7C048
:10E9E000EB85FC858AE090E09383828386EA95E05C
:10E9F0002B813C81BC01C9010E9415F1009731F4C3
:10EA0000EB85FC8589E090E0938382838F819885F4
:10EA10006FE370E00E9433F19A83898389819A8140
:10EA20000097B9F1E981FA81108289819A81019672
:10EA30009A83898389819A81DC01FD0101900020FC
:10EA4000E9F73197CF018A1B9B0B01960E944D81FC
:10EA5000EB85FC8591878087EB85FC85808591859A
:10EA6000009749F489859A850E946A828B859C85E6
:10EA70000E94C9715CC0EB85FC8520853185898148
:10EA80009A81BC01C9010E9447F18B859C850E9437
:10EA9000A56A8F819885DC01FD0101900020E9F7CE
:10EAA0003197CF018A1B9B0B01960E944D81EB850C
:10EAB000FC8597838683EB85FC858681978100970B
:10EAC00049F489859A850E946A828B859C850E947B
:10EAD000C9712DC0EB85FC85268137818F81988592
:10EAE000BC01C9010E9447F189859A850E946A820A
:10EAF000EB85FC85868197810E94CE61009759F451
:10EB00008B859C852D853E8540E951E0BC01C9017E
:10EB10000E94A96608C08B859C852D853E85BC0119
:10EB2000C9010E942E6E8B859C850E94C9712E960C
:10EB30000FB6F894DEBF0FBECDBFDF91CF91089521
:10EB4000CF93DF93CDB7DEB724970FB6F894DEBF2F
:10EB50000FBECDBF9A8389837C836B838FEA95E058
:10EB600029813A81BC01C9010E947FF1009751F0CF
:10EB70000E94248E9C018B819C81BC01C9010E9452
:10EB8000F8E6ABC08BEB95E029813A81BC01C90165
:10EB90000E947FF10097B1F180917F08A82FBB27D9
:10EBA00080917E08282F332780917D08482F552794
:10EBB00080917C08682F772780917B08E82FFF27BA
:10EBC00080917A089927BF93AF933F932F935F93D8
:10EBD0004F937F936F93FF93EF939F938F9388EC63
:10EBE00095E09F938F938B819C819F938F930E943D
:10EBF000D2E68DB79EB740960FB6F8949EBF0FBE73
:10EC00008DBF6BC086EE95E029813A81BC01C901B8
:10EC10000E947FF10097A1F0809180089091810877
:10EC2000A0918208B0918308BC01CD010E9485B3F8
:10EC30009C018B819C81BC01C9010E94F8E64DC0FA
:10EC400082EF95E029813A81BC01C9010E947FF1E0
:10EC50000097A1F08091840890918508A091860882
:10EC6000B0918708BC01CD010E9485B39C018B81C6
:10EC70009C81BC01C9010E94F8E62FC08EEF95E08F
:10EC800029813A81BC01C9010E947FF10097A1F05E
:10EC90008091880890918908A0918A08B0918B088A
:10ECA000BC01CD010E9485B39C018B819C81BC017C
:10ECB000C9010E94F8E611C08091B2079091B30794
:10ECC000009759F0E091B207F091B3078B819C81D6
:10ECD00029813A81BC01C901099524960FB6F8949F
:10ECE000DEBF0FBECDBFDF91CF9108950F931F936D
:10ECF000CF93DF93CDB7DEB7A1970FB6F894DEBF01
:10ED00000FBECDBF9F8B8E8B798F688F5B8F4A8FA5
:10ED10003D8F2C8F1F8F0E8F1B8A1A8A198A188A93
:10ED20001F861E861E82888D998D0E94A8E2DC01B6
:10ED3000CB018F839887A987BA8780E091E09C8771
:10ED40008B871B821A82198280E490E00E944D8199
:10ED50009F878E878B859C850E944D819B8B8A8B9C
:10ED60008B859C8501960E944D81998B888B8A8921
:10ED70009B89009709F41CC188899989009709F437
:10ED800017C18E859F85009709F412C108C18F8134
:10ED90009885A985BA858F3F9105A105B10509F030
:10EDA00024F48F8198859C878B878B859C852A8905
:10EDB0003B89E88DF98DAC01B901CF010E941BE1BF
:10EDC0009D8B8C8B1D821C8298C08C819D819C01A7
:10EDD0008A899B89F901E80FF91F80818D878E81CF
:10EDE000282F332739A328A388A199A18130910521
:10EDF00001F128A139A12230310509F44DC088A1C3
:10EE000099A1009709F074C08D858C3311F481E0CD
:10EE10008E838A819B819C0188899989F901E80FF9
:10EE2000F91F8D8580838A819B8101969B838A83CC
:10EE30005FC08D858532F9F482E08E838A819B8163
:10EE4000009729F08A819B8101979B838A838A811D
:10EE50009B81009709F44CC08A819B812E893F8950
:10EE6000E889F989AC0161E070E0CF010E9426E7F2
:10EE70001B821A823DC01E828A819B819C018889E7
:10EE80009989F901E80FF91F8D8580838A819B811B
:10EE900001969B838A832CC08D858E33A1F41E82BC
:10EEA000898199279C018E859F85F901E80FF91FBB
:10EEB00010828E899F892E853F85BC01C9010E94E1
:10EEC000A075198215C08D85853209F41D8689814A
:10EED00099279C018E859F85F901E80FF91F8D8583
:10EEE000808389818F5F89838981803408F01982CA
:10EEF0008C819D8101969D838C832C813D818C89A1
:10EF00009D89281739070CF460CF8A819B8100976F
:10EF100099F12A813B8188899989820F931FFC018D
:10EF2000319780818C33D1F48A819B8101979B83B7
:10EF30008A834A815B818E899F89E889F9899C014E
:10EF400061E070E0CF010E9426E7E889F9898CE34F
:10EF5000808381E090E09B838A830EC08A819B81BD
:10EF60002E893F89E889F989AC0161E070E0CF0121
:10EF70000E9426E71B821A828C899D899C01442766
:10EF800037FD4095542F8F819885A985BA85821BBE
:10EF9000930BA40BB50B8F839887A987BA878F81B2
:10EFA0009885A985BA850097A105B10509F0EFCE2E
:10EFB0008A899B89009721F08A899B890E946A82AD
:10EFC00088899989009721F0888999890E946A82A5
:10EFD0008E859F85009721F08E859F850E946A828D
:10EFE000A1960FB6F894DEBF0FBECDBFDF91CF91D3
:10EFF0001F910F910895CF93DF93CDB7DEB724977C
:10F000000FB6F894DEBF0FBECDBF9A8389831C82F2
:10F010001B828091B2079091B307009739F48981E0
:10F020009A819093B3078093B20704C08FEF9FEF4C
:10F030009C838B838B819C8124960FB6F894DEBFD2
:10F040000FBECDBFDF91CF910895CF93DF93CDB7A2
:10F05000DEB786E796E72AE036E0BC01C9010E94E8
:10F060009F68DF91CF910895CF93DF93CDB7DEB73F
:10F0700060970FB6F894DEBF0FBECDBF9E878D8719
:10F08000788B6F878F85988960E070E80E9499E09F
:10F090009C878B878B859C852FEF8F3F9207B9F4D8
:10F0A0008AEE9EE62F8538893F932F939F938F9307
:10F0B0008D859E859F938F930E9405E88DB79EB79F
:10F0C00006960FB6F8949EBF0FBE8DBF69C08B85A4
:10F0D0009C850E94A8E2DC01CB0189839A83AB83E3
:10F0E000BC8380E092E09E838D838D819E810E940F
:10F0F0004D8198878F838F819885009709F44CC044
:10F100003EC089819A81AB81BC81803022E0920728
:10F1100020E0A20720E0B20724F489819A819E832F
:10F120008D838D819E812F813885EB85FC85AC0197
:10F13000B901CF010E941BE19A87898749855A85C9
:10F140008D859E85EF81F8859C0161E070E0CF019F
:10F150000E9426E70097E1F089859A859C01442763
:10F1600037FD4095542F89819A81AB81BC81821BE8
:10F17000930BA40BB50B89839A83AB83BC838981E2
:10F180009A81AB81BC810097A105B10509F0B9CF87
:10F190008F8198850E946A828B859C850E9407E0FA
:10F1A00060960FB6F894DEBF0FBECDBFDF91CF9152
:10F1B0000895CF93DF93CDB7DEB722970FB6F894BB
:10F1C000DEBF0FBECDBF9A838983E981FA81868134
:10F1D0009781009731F0E981FA81868197810E94B9
:10F1E0006A82E981FA8180859185009731F0E98111
:10F1F000FA81808591850E946A82E981FA818285FF
:10F200009385009731F0E981FA81828593850E9488
:10F210006A82E981FA8184859585009731F0E981D8
:10F22000FA81848595850E946A82E981FA818685C2
:10F230009785009731F0E981FA81868597850E944C
:10F240006A82E981FA8180899189009731F0E981A8
:10F25000FA81808991890E946A82E981FA81828992
:10F260009389009731F0E981FA81828993890E941C
:10F270006A8289819A810E946A8222960FB6F894E6
:10F28000DEBF0FBECDBFDF91CF9108950F931F93C7
:10F29000CF93DF93CDB7DEB7AF970FB6F894DEBF4D
:10F2A0000FBECDBF9A8F898F7C8F6B8F5E8F4D8FF6
:10F2B00038A32F8F1C861B868B8D9C8D0E94CE6160
:10F2C000009779F48CE99FE69F938F93898D9A8DAF
:10F2D0009F938F930E9405E80F900F900F900F90CF
:10F2E000F6C38FE096E02B8D3C8D48E050E0BC01EA
:10F2F000C9010E944EF1009709F037C186E190E004
:10F300000E943E829E838D838D819E81009779F439
:10F3100088E89FE69F938F93898D9A8D9F938F9313
:10F320000E9405E80F900F900F900F90D0C3ED81D1
:10F33000FE8181E090E091838083EF8DF8A182814E
:10F340009381ED81FE8193838283ED81FE8115821D
:10F350001482EF8DF8A1808991890097C1F1EF8D1A
:10F36000F8A180899189DC01FD0101900020E9F775
:10F370003197CF018A1B9B0B01960E944D81ED8135
:10F38000FE81918B808BED81FE8180899189009730
:10F3900099F484E79FE69F938F93898D9A8D9F932D
:10F3A0008F930E9405E80F900F900F900F908D8122
:10F3B0009E810E94D9788BC3EF8DF8A12089318975
:10F3C000ED81FE8180899189B9010E9447F1EF8D1D
:10F3D000F8A1848595850097C1F1EF8DF8A184850A
:10F3E0009585DC01FD0101900020E9F73197CF01FF
:10F3F0008A1B9B0B01960E944D81ED81FE819587B2
:10F400008487ED81FE8184859585009799F480E657
:10F410009FE69F938F93898D9A8D9F938F930E94E0
:10F4200005E80F900F900F900F908D819E810E94A4
:10F43000D9784DC3EF8DF8A124853585ED81FE8106
:10F4400084859585B9010E9447F18B8D9C8D6FE372
:10F4500070E00E9433F198878F838F8198850097A1
:10F4600009F441C0EF81F88510828F81988501965B
:10F4700098878F838F819885DC01FD0101900020A2
:10F48000E9F73197CF018A1B9B0B01960E944D81B2
:10F49000ED81FE8191878087ED81FE818085918558
:10F4A000009799F48CE49FE69F938F93898D9A8DB2
:10F4B0009F938F930E9405E80F900F900F900F90ED
:10F4C0008D819E810E94D97802C3ED81FE812085C5
:10F4D00031858F819885BC01C9010E9447F18D81DA
:10F4E0009E810E94A56A8B8D9C8DDC01FD0101909F
:10F4F0000020E9F73197CF018A1B9B0B01960E94F0
:10F500004D81ED81FE8197838683ED81FE81868129
:10F510009781009799F488E39FE69F938F93898D55
:10F520009A8D9F938F930E9405E80F900F900F90F4
:10F530000F908D819E810E94D978C9C2ED81FE8194
:10F54000268137818B8D9C8DBC01C9010E9447F1BA
:10F550008D819E81298D3A8DBC01C9010E94436035
:10F560008D819E810E94D978B2C28D8D9E8D00972B
:10F5700031F18D8D9E8DDC01FD0101900020E9F7B8
:10F5800031979F012A1B3B0B8B8D9C8DDC01FD016C
:10F5900001900020E9F73197CF018A1B9B0B820F66
:10F5A000931F01960E944D819C878B878D8D9E8D28
:10F5B0002B853C85BC01C9010E9447F130C08B8D71
:10F5C0009C8DDC01FD0101900020E9F73197CF010E
:10F5D0008A1B9B0B06960E944D819C878B878B858F
:10F5E0009C859AA389A388E196E09CA38BA396E0CF
:10F5F0009DA3EBA1FCA100808BA19CA101969CA3E3
:10F600008BA3E9A1FAA1008289A19AA101969AA3EC
:10F6100089A39DA191509DA3EDA1EE2351F78B8D60
:10F620009C8D2B853C85BC01C9010E9428F18B85EE
:10F630009C850E9411689A8789878B859C8560E0EC
:10F6400070E80E9499E0988F8F8B8B859C850E9433
:10F650006A828F89988DFFEF8F3F9F0709F0B8C1AD
:10F660008B8D9C8DDC01FD0101900020E9F7319725
:10F67000CF018A1B9B0B9A83898389819A810C967F
:10F680000E943E829C838B838B819C81009779F4BE
:10F6900084E29FE69F938F93898D9A8D9F938F939A
:10F6A0000E9405E80F900F900F900F9010C2898173
:10F6B0009A81009741F08B8D9C8D2B813C81BC0100
:10F6C000C9010E9447F189819A81009799F02981A7
:10F6D0003A818B819C81820F931FFC01319780813D
:10F6E0008F3241F08EE196E02B813C81BC01C90153
:10F6F0000E9428F180E296E02B813C81BC01C90187
:10F700000E9428F18D8D9E8D009731F18D8D9E8DFB
:10F71000DC01FD0101900020E9F731979F012A1BD0
:10F720003B0B8B819C81DC01FD0101900020E9F7FE
:10F730003197CF018A1B9B0B820F931F01960E946A
:10F740004D819C878B878D8D9E8D2B853C85BC0143
:10F75000C9010E9447F130C08B819C81DC01FD0111
:10F7600001900020E9F73197CF018A1B9B0B069689
:10F770000E944D819C878B878B859C859FA38EA340
:10F7800088E196E099A788A796E09AA7E8A5F9A549
:10F79000008088A599A5019699A788A7EEA1FFA149
:10F7A00000828EA19FA101969FA38EA39AA591503E
:10F7B0009AA7EAA5EE2351F78B819C812B853C8586
:10F7C000BC01C9010E9428F18B819C810E946A8240
:10F7D0008B859C850E9411689A8789878B859C857B
:10F7E00060E070E80E9499E0988F8F8B8B859C85F4
:10F7F0000E946A828F89988DFFEF8F3F9F0709F0E3
:10F80000E7C08B8D9C8DDC01FD0101900020E9F7A4
:10F810003197CF018A1B9B0B9A83898389819A81B7
:10F820000D960E943E829C838B838B819C810097E6
:10F8300079F480E19FE69F938F93898D9A8D9F93B2
:10F840008F930E9405E80F900F900F900F903FC18B
:10F8500089819A81009741F08B8D9C8D2B813C8111
:10F86000BC01C9010E9447F189819A81009799F0F2
:10F8700029813A818B819C81820F931FFC013197F2
:10F8800080818F3241F08EE196E02B813C81BC017A
:10F89000C9010E9428F18BE296E02B813C81BC01DA
:10F8A000C9010E9428F18D8D9E8D009731F18D8DBB
:10F8B0009E8DDC01FD0101900020E9F731979F0149
:10F8C0002A1B3B0B8B819C81DC01FD0101900020F8
:10F8D000E9F73197CF018A1B9B0B820F931F01968B
:10F8E0000E944D819C878B878D8D9E8D2B853C85BD
:10F8F000BC01C9010E9447F130C08B819C81DC01B1
:10F90000FD0101900020E9F73197CF018A1B9B0B85
:10F9100006960E944D819C878B878B859C859CA732
:10F920008BA788E196E09EA78DA796E09FA7EDA5FF
:10F93000FEA500808DA59EA501969EA78DA7EBA58F
:10F94000FCA500828BA59CA501969CA78BA79FA5D3
:10F9500091509FA7EFA5EE2351F78B819C812B85BA
:10F960003C85BC01C9010E9428F18B819C810E94C9
:10F970006A828B859C850E9411689A8789878B850E
:10F980009C8560E070E80E9499E0988F8F8B8B8552
:10F990009C850E946A828F89988DFFEF8F3F9F0719
:10F9A000B9F48DEF9EE62B853C853F932F939F9373
:10F9B0008F93898D9A8D9F938F930E9405E88DB7C1
:10F9C0009EB706960FB6F8949EBF0FBE8DBF7FC040
:10F9D0008F89988D0E94A8E2DC01CB018D879E87DC
:10F9E000AF87B88B89859A85009709F05CC080E065
:10F9F00092E09A8B898B89899A890E944D819C8B90
:10FA00008B8B8B899C89009709F45DC03EC08D85E6
:10FA10009E85AF85B8898030E2E09E07E0E0AE07C2
:10FA2000E0E0BE0724F48D859E859A8B898B8989B9
:10FA30009A892B893C89EF89F88DAC01B901CF01F6
:10FA40000E941BE19E8B8D8B4D895E89898D9A8DDD
:10FA5000EB89FC899C0161E070E0CF010E9426E700
:10FA60000097E1F08D899E899C01442737FD4095E0
:10FA7000542F8D859E85AF85B889821B930BA40B6F
:10FA8000B50B8D879E87AF87B88B8D859E85AF859B
:10FA9000B8890097A105B10509F0B9CF8B899C8978
:10FAA0000E946A8210C04D855E858F8D98A12D8D34
:10FAB0003E8D6F89788DE98DFA8DA985BA858C0187
:10FAC000CF01FD0109958F89988D0E9407E0AF96BF
:10FAD0000FB6F894DEBF0FBECDBFDF91CF911F915F
:10FAE0000F910895CF93DF93CDB7DEB726970FB66A
:10FAF000F894DEBF0FBECDBF9A8389837C836B836E
:10FB00005E834D8309C0EB81FC81808191810196E8
:10FB1000EB81FC8191838083EB81FC8120813181A9
:10FB20008D819E8128173907A8F5EB81FC818081A2
:10FB300091819C0189819A81F901E80FF91F8081E7
:10FB40008A3009F3EB81FC81808191819C0189815C
:10FB50009A81F901E80FF91F80818D30A1F2EB81C4
:10FB6000FC81808191819C0189819A81F901E80F52
:10FB7000F91F8081893039F2EB81FC81808191818C
:10FB80009C0189819A81F901E80FF91F80818032F7
:10FB900009F4B9CF26960FB6F894DEBF0FBECDBFDD
:10FBA000DF91CF9108950F931F93CF93DF93CDB73C
:10FBB000DEB763970FB6F894DEBF0FBECDBF9F834D
:10FBC0008E83798768875B874A873D872C871F8765
:10FBD0000E8784E090E09D838C8384E090E09D8399
:10FBE0008C838A859B859E012C5F3F4FE885F98534
:10FBF000AC01B901CF010E94727D2C813D818A85C3
:10FC00009B852817390719F41B8A1A8A71C18C81C0
:10FC10009D819C0188859985280F391F87E396E08F
:10FC200048E050E0BC01C9010E944EF1009741F448
:10FC30008C819D8108969D838C8382E089831CC082
:10FC40008C819D819C0188859985280F391F80E4CE
:10FC500096E045E050E0BC01C9010E944EF10097DA
:10FC600041F48C819D8105969D838C8383E08983FB
:10FC700003C01B8A1A8A3CC12C813D818A859B85E1
:10FC80002817390718F01B8A1A8A32C18A859B8582
:10FC90009E012C5F3F4FE885F985AC01B901CF018A
:10FCA0000E94727D2C813D818A859B8528173907AA
:10FCB00019F41B8A1A8A1CC18981823099F58C81BA
:10FCC0009D819C0188859985280F391F86E496E0DF
:10FCD00047E050E0BC01C9010E944EF1009731F4A9
:10FCE0008C819D8107969D838C8336C08C819D81FC
:10FCF0009C0188859985280F391F8EE496E044E0A1
:10FD000050E0BC01C9010E944EF1009741F48C8182
:10FD10009D8104969D838C8381E089831DC01B8A0D
:10FD20001A8AE6C08C819D819C0188859985280F5F
:10FD3000391F83E596E043E050E0BC01C9010E9411
:10FD40004EF1009731F48C819D8103969D838C83C5
:10FD500003C01B8A1A8ACCC02C813D818A859B8571
:10FD60002817390718F01B8A1A8AC2C08A859B8512
:10FD70009E012C5F3F4FE885F985AC01B901CF01A9
:10FD80000E94727D2C813D818A859B8528173907C9
:10FD900019F41B8A1A8AACC08C819D819C018885CC
:10FDA0009985F901E80FF91F80818D3319F01B8ABD
:10FDB0001A8A9EC08C819D8101969D838C838A8541
:10FDC0009B859E012C5F3F4FE885F985AC01B90109
:10FDD000CF010E94727D2C813D818A859B852817E9
:10FDE000390719F41B8A1A8A83C08C819D819C0172
:10FDF00088859985F901E80FF91F8081823209F021
:10FE000073C08C819D8101969D838C832C813D8163
:10FE10008A859B852817390719F41B8A1A8A68C0B6
:10FE20008C819D819C0188859985820F931F9B837E
:10FE30008A830FC08C819D8101969D838C832C8148
:10FE40003D818A859B852817390719F41B8A1A8AF0
:10FE50004FC08C819D819C0188859985F901E80FAF
:10FE6000F91F8081823231F78C819D819C018885C8
:10FE70009985F901E80FF91F10828981282F33270E
:10FE8000398B288B8889998982309105A1F028893E
:10FE9000398923303105E1F08889998981309105CC
:10FEA00009F022C08A819B812E813F81BC01C9015A
:10FEB0000E94347819C08E859F854C855D856A8146
:10FEC0007B81EE81FF819C01CF010E9446790CC0AD
:10FED0008E859F854C855D856A817B81EE81FF8162
:10FEE0009C01CF010E94467921E030E03B8B2A8BB8
:10FEF0008A899B8963960FB6F894DEBF0FBECDBF8B
:10FF0000DF91CF911F910F9108950F931F93CF937E
:10FF1000DF93CDB7DEB7AC970FB6F894DEBF0FBE58
:10FF2000CDBF9E878D87788B6F875A8B498B3C8B93
:10FF30002B8B1E8B0D8B29893A893AA329A349A1C2
:10FF40005AA182E04130580724F020E032E03AA381
:10FF500029A349A15AA1598748878885998501967F
:10FF60000E944D819C878B871A861F821E826FC1DB
:10FF70008885998501969C018B859C85FC01C9012A
:10FF8000AC0160E070E0CF010E940EF129893A894E
:10FF90008E819F81A901481B590BCA01288539858B
:10FFA0003CA32BA398A38F8F4F8D58A18BA19CA10D
:10FFB0008417950724F42BA13CA138A32F8F8F8D94
:10FFC00098A12B853C85EF85F889AC01B901CF015B
:10FFD0000E941BE19D838C838A85882309F0ABC036
:10FFE00087E596E02B853C85BC01C9010E947FF125
:10FFF0009B838A838A819B81009709F06BC0298942
:020000021000EC
:100000003A8988859985821793070CF04EC08885B8
:100010009985845690404C815D815EA34DA39E8F4F
:100020008D8F8D8D9E8D2DA13EA12817390724F42B
:100030004DA15EA15E8F4D8F4D8D5E8D8D859E8510
:10004000EB85FC859C0161E070E0CF010E9426E712
:1000500088859985845690402C813D8138A72FA3AF
:100060009C8F8B8F4B8D5C8D8FA198A584179507E6
:1000700024F42FA138A53C8F2B8F8E819F814B8D2F
:100080005C8D840F951F9F838E838E819F81AA270D
:1000900097FDA095BA2FEF85F88920E030E0AC01FC
:1000A000BD01CF010E9483E5D2C04C815D818D8569
:1000B0009E85EB85FC859C0161E070E0CF010E948C
:1000C00026E72E813F818C819D81820F931F9F8324
:1000D0008E83BDC08A819B81282F8B859C85522F62
:1000E000581B852F89838981482F55278D859E85AB
:1000F000EB85FC859C0161E070E0CF010E9426E762
:100100008981282F33278E819F81820F931F9F83A0
:100110008E838E819F81AA2797FDA095BA2FEF85A8
:10012000F88920E030E0AC01BD01CF010E9483E5F9
:1001300081E08A878CC08CE596E02B853C85BC01EC
:10014000C9010E947FF19B838A838A819B810097EA
:10015000E1F5888599859AA789A72C813D813A8FF9
:10016000298F498D5A8D89A59AA58417950724F45E
:1001700029A53AA53A8F298F898D9A8D2D853E859F
:10018000EB85FC85AC0161E070E0CF010E9426E7C1
:10019000488559855CA74BA78C819D81988F8F8B53
:1001A0002F89388D4BA55CA54217530724F48BA5E6
:1001B0009CA5988F8F8B8E819F812F89388D820F80
:1001C000931F9F838E831A8642C08A819B81282F2A
:1001D0008B859C85322F381B832F89838981482FFB
:1001E00055278D899E892B893C896B857C85ED857A
:1001F000FE858C01CF010E94D37D882371F4898113
:1002000099270396AC018D859E85EB85FC859C0125
:1002100061E070E0CF010E9426E78981282F332713
:100220008E819F81820F931F03969F838E838E8181
:100230009F81AA2797FDA095BA2FEF85F88920E026
:1002400030E0AC01BD01CF010E9483E51A86298907
:100250003A898E819F812817390709F089CE8B85CD
:100260009C850E946A82AC960FB6F894DEBF0FBEE2
:10027000CDBFDF91CF911F910F910895CF93DF9361
:10028000CDB7DEB785E89FE720E636E0BC01C901BF
:100290000E949F68DF91CF910895CF93DF93CDB7F0
:1002A000DEB72C970FB6F894DEBF0FBECDBF9A878E
:1002B00089871C821B821A8219822091B40730918F
:1002C000B50789859A858217930718F01C861B86C7
:1002D000CAC089859A8506969A87898789859A856D
:1002E0008430910520F484E090E09A87898780919A
:1002F000490890914A0898878F8389E498E09E8303
:100300008D833DC0EF81F8852081318189859A8573
:100310002817390748F1EF81F885208131818985D7
:100320009A852817390749F48F8198859C838B8398
:100330008D819E819A83898327C08B819C810097C0
:1003400059F0EB81FC8120813181EF81F88580813A
:1003500091818217930740F48F8198859C838B83CA
:100360008D819E819A8389838F81988502969E8351
:100370008D83EF81F8858281938198878F838F8128
:100380009885009709F0BECF8B819C81009709F476
:1003900066C0EB81FC812081318189859A850A962E
:1003A0008217930760F58B819C819C0189859A85D2
:1003B000820F931F98878F83EB81FC81208131818D
:1003C00089859A85A901481B590BCA01EF81F885D7
:1003D00091838083EB81FC8182819381EF81F88519
:1003E00093838283EB81FC8189859A8591838083C5
:1003F000E981FA818F8198859183808308C0EB81A0
:10040000FC8182819381E981FA81918380832091AB
:10041000B4073091B507EB81FC8180819181A901FE
:10042000481B590BCA019093B5078093B407EB8121
:10043000FC81808191819C018B819C81820F931F23
:100440000497FC018FEE9EEBADEABEED80839183B5
:10045000A283B3838B819C8102969C838B838B8147
:100460009C819C878B878B859C852C960FB6F894F6
:10047000DEBF0FBECDBFDF91CF910895CF93DF9345
:10048000CDB7DEB724970FB6F894DEBF0FBECDBF51
:100490009C838B838B819C810E944D819A8389836D
:1004A00089819A81009759F089819A819C018B8179
:1004B0009C81AC0160E070E0C9010E940EF189816D
:1004C0009A8124960FB6F894DEBF0FBECDBFDF91A0
:1004D000CF910895CF93DF93CDB7DEB72C970FB6AA
:1004E000F894DEBF0FBECDBF9A87898789859A852C
:1004F00002979C838B83EB81FC81808191819A831D
:1005000089838091490890914A0898878F8389E46C
:1005100098E09E838D839EC0EF81F8852081318194
:100520008F819885280F391F8B819C812817390767
:10053000D9F5EF81F88520813181EB81FC818081C3
:100540009181820F931FEF81F88591838083EF81E2
:10055000F885208131818F819885280F391FEF819F
:10056000F885828193812817390709F078C0EF81D7
:10057000F88520813181EF81F8850280F381E02DBB
:1005800080819181820F931FEF81F8859183808311
:10059000EF81F8850280F381E02D82819381EF81E4
:1005A000F885938382835BC08F8198859C018B81C2
:1005B0009C818217930788F5ED81FE818B819C8158
:1005C00091838083EB81FC81208131818B819C81AF
:1005D000280F391F8F81988528173907B9F4EB81C7
:1005E000FC8120813181EF81F88580819181820FAA
:1005F000931FEB81FC8191838083EF81F885828159
:100600009381EB81FC819383828329C0EB81FC8100
:100610008F8198859383828322C0EF81F885208122
:1006200031818F819885280F391F8B819C8182179A
:10063000930728F48FEF9FEF9C878B872EC08F81C5
:10064000988502969E838D83EF81F88582819381C0
:1006500098878F838F819885009709F05DCF8F8170
:100660009885009761F4EB81FC818F819885938355
:100670008283ED81FE818B819C8191838083809137
:10068000B4079091B50729813A81820F931F909307
:10069000B5078093B4071C861B868B859C852C969A
:1006A0000FB6F894DEBF0FBECDBFDF91CF91089596
:1006B000CF93DF93CDB7DEB724970FB6F894DEBFA4
:1006C0000FBECDBF9A8389837C836B83E981FA81D6
:1006D0008B819C819183808389819A8102960E947B
:1006E0006A8224960FB6F894DEBF0FBECDBFDF91AD
:1006F000CF910895CF93DF93CDB7DEB78091B40744
:100700009091B507DF91CF910895CF93DF93CDB747
:10071000DEB726970FB6F894DEBF0FBECDBF9C8321
:100720008B837E836D83EB81FC818D819E81908F95
:10073000878BEB81FC81158214820FB6F8940F929F
:10074000ED81FE81808191819A83898389819A815B
:100750002FEF8F3F920761F41A821982EB81FC819F
:10076000848195810196EB81FC819583848321C0EE
:1007700089819A810097E9F00F900FBE0BC08981A3
:100780009A8102969E838D83E981FA818281938189
:100790009A83898389819A81009741F0E981FA815E
:1007A0009289EB81FC818289891748F70FB6F8940A
:1007B0000F92EB81FC8189819A8193838283ED8101
:1007C000FE818B819C8191838083EB81FC8182817E
:1007D0009381009709F1EB81FC810280F381E02D88
:1007E000848195810097C1F0EB81FC812481358162
:1007F000EB81FC810280F381E02D84819581820F61
:10080000931FEB81FC8195838483EB81FC810280C3
:10081000F381E02D158214820F900FBE26960FB63D
:10082000F894DEBF0FBECDBFDF91CF910895CF9377
:10083000DF93CDB7DEB726970FB6F894DEBF0FBEB5
:10084000CDBF9C838B837E836D830FB6F8940F920C
:10085000ED81FE81808191819A8389830F900FBE03
:1008600089819A812FEF8F3F920709F449C043C0D5
:1008700029813A818B819C812817390789F50FB628
:10088000F8940F92EB81FC8182819381ED81FE814E
:1008900091838083EB81FC81848195810097A9F00D
:1008A000EB81FC8182819381009759F0EB81FC817F
:1008B000A281B381EB81FC8184819581FD019583C7
:1008C0008483EB81FC81158214820F900FBEEB8133
:1008D000FC8113821282EB81FC81108E178A10C07A
:1008E00089819A8102969E838D83E981FA81828132
:1008F00093819A83898389819A81009709F0B8CF7F
:1009000026960FB6F894DEBF0FBECDBFDF91CF9114
:100910000895CF93DF93CDB7DEB728970FB6F8943D
:10092000DEBF0FBECDBF80914B0890914C089887D9
:100930008F8339C00FB6F8940F92EF81F8858481C8
:1009400095819A8389830F900FBE89819A81009740
:1009500021F1EF81F8858789908D9E838D830FB675
:10096000F8940F92EF81F885848195810197EF814A
:10097000F88595838483ED81FE81808191819C83BC
:100980008B830F900FBE8B819C812FEF8F3F92073F
:1009900021F08D819E810E94FF8BEF81F8858081FF
:1009A000918198878F838F819885009709F0C2CFB6
:1009B0000E94348720914F083091500880914D0853
:1009C00090914E0828173907A1F0E0914F08F09157
:1009D00050088785813031F4E0914F08F09150083C
:1009E00082E087870FB6F8940F920E94358E0F90A1
:1009F0000FBE28960FB6F894DEBF0FBECDBFDF91B5
:100A0000CF910895CF93DF93CDB7DEB724970FB67C
:100A1000F894DEBF0FBECDBF9A8389837C836B833E
:100A2000EB81FC81168A158AEB81FC8182E0878745
:100A30008DE498E02B813C81BC01C9010E94858333
:100A400024960FB6F894DEBF0FBECDBFDF91CF91D5
:100A50000895CF93DF93CDB7DEB7E0914F08F091C3
:100A60005008828193810097A1F08DE498E0209155
:100A70004F0830915008BC01C9010E9417848DE4D1
:100A800098E020914F0830915008BC01C9010E94A4
:100A900085830E948984DF91CF910895CF93DF935E
:100AA000CDB7DEB722970FB6F894DEBF0FBECDBF2D
:100AB0008A83E0914F08F0915008828989838DE400
:100AC00098E020914F0830915008BC01C9010E9464
:100AD0001784E0914F08F09150088A81828B8A81B7
:100AE0008F3F59F08DE498E020914F0830915008E5
:100AF000BC01C9010E94858302C00E94CC8520915F
:100B00004F083091500880914D0890914E08281759
:100B1000390739F4E0914F08F091500881E0878758
:100B20000DC0E0914F08F091500882E087870FB622
:100B3000F8940F920E94358E0F900FBE89819927ED
:100B400022960FB6F894DEBF0FBECDBFDF91CF91D6
:100B50000895CF93DF93CDB7DEB78FEF0E944E8518
:100B6000DF91CF910895CF93DF93CDB7DEB780911A
:100B7000510890915208009761F0E0915108F0916E
:100B80005208838994890E946A82109252081092B6
:100B90005108DF91CF910895CF93DF93CDB7DEB7A2
:100BA00024970FB6F894DEBF0FBECDBF80914B08DF
:100BB00090914C089C838B838BE498E09A83898383
:100BC0000E94B3851CC020914F08309150088B8142
:100BD0009C818217930749F4EB81FC81808191818C
:100BE000E981FA81918380830EC08B819C819A83F5
:100BF0008983EB81FC81808191819C838B838B81B4
:100C00009C81009701F780914F0890915008909334
:100C100052088093510824960FB6F894DEBF0FBE99
:100C2000CDBFDF91CF910895CF93DF93CDB7DEB7DE
:100C300026970FB6F894DEBF0FBECDBF9C838B8383
:100C400080914B0890914C089A83898318C08981C0
:100C50009A819C012A5F3F4F8B819C81BC01C90115
:100C60000E943EF1009729F489819A819E838D83A9
:100C70000CC0E981FA81808191819A83898389817D
:100C80009A81009721F71E821D828D819E81269672
:100C90000FB6F894DEBF0FBECDBFDF91CF910895A0
:100CA000CF93DF93CDB7DEB722970FB6F894DEBFB0
:100CB0000FBECDBF9A8389838091550890915608C5
:100CC000A0915708B09158080196A11DB11D8093BD
:100CD000550890935608A0935708B0935808229649
:100CE0000FB6F894DEBF0FBECDBFDF91CF91089550
:100CF000CF93DF93CDB7DEB780E596E80E9456909C
:100D0000A7E5B0E0E7E5F0E0808182608C93DF91B9
:100D1000CF910895EF92FF920F931F93CF93DF939C
:100D2000CDB7DEB724970FB6F894DEBF0FBECDBFA8
:100D30009C838B83EB81FC81138212828091530808
:100D4000909154089A83898352C0EB81FC8120855D
:100D5000318542855385E981FA8180859185A28517
:100D6000B385281739074A075B07D8F4E981FA8168
:100D70002085318542855385EB81FC818085918575
:100D8000A285B38579018A01E81AF90A0A0B1B0BBF
:100D9000D801C701E981FA8180879187A287B3874B
:100DA0002BC0EB81FC812085318542855385E9810B
:100DB000FA8180859185A285B38579018A01E81A37
:100DC000F90A0A0B1B0BD801C701EB81FC81808754
:100DD0009187A287B387EB81FC8189819A81938374
:100DE0008283E981FA81808191819A8389838981D3
:100DF0009A81009709F0A9CFEB81FC8189819A81C2
:100E000091838083EB81FC8180819181009749F0FF
:100E1000EB81FC810190F081E02D8B819C8193839B
:100E20008283EB81FC8182819381009751F0EB8179
:100E3000FC810280F381E02D8B819C8191838083F2
:100E400006C08B819C81909354088093530824960C
:100E50000FB6F894DEBF0FBECDBFDF91CF911F91CB
:100E60000F91FF90EF900895EF92FF920F931F93D1
:100E7000CF93DF93CDB7DEB72A970FB6F894DEBFD6
:100E80000FBECDBF0E94DE89DC01CB018D839E8326
:100E9000AF83B8872091B6073091B7074091B80764
:100EA0005091B9078D819E81AF81B885821B930BCC
:100EB000A40BB50B89839A83AB83BC838D819E8100
:100EC000AF81B8858093B6079093B707A093B80712
:100ED000B093B9079EC080915308909154089A87A7
:100EE0008987E985FA852085318542855385898101
:100EF0009A81AB81BC8182179307A407B507E8F4F8
:100F0000E985FA85208531854285538589819A81D5
:100F1000AB81BC8179018A01E81AF90A0A0B1B0B23
:100F2000D801C701E985FA8580879187A287B387B1
:100F300019821A821B821C8218C0E985FA852085D5
:100F400031854285538589819A81AB81BC81821B21
:100F5000930BA40BB50B89839A83AB83BC83E98580
:100F6000FA851086118612861386E985FA858085B2
:100F70009185A285B3850097A105B10509F049C007
:100F8000E985FA8584859585009771F0E985FA856C
:100F900044855585E985FA858685978529853A852D
:100FA000BC01C901FA010995E985FA858481958119
:100FB000A681B781E985FA8580879187A287B38763
:100FC000E985FA8580859185A285B3850097A1057D
:100FD000B10529F489859A850E947A891AC0E09121
:100FE0005308F09154088081918190935408809324
:100FF00053088091530890915408009731F0E09184
:101000005308F09154081382128289859A850E94B0
:101010008A868091530890915408009749F08981FD
:101020009A81AB81BC810097A105B10509F053CF2E
:101030002A960FB6F894DEBF0FBECDBFDF91CF91D9
:101040001F910F91FF90EF900895EF92FF920F93F1
:101050001F93CF93DF93CDB7DEB72B970FB6F894DE
:10106000DEBF0FBECDBF6B837C838D839E8358878D
:101070004F833A8729870B8780E190E00E944D815A
:101080009A83898389819A81009709F445C00E94D7
:10109000DE899B01AC018B819C81AD81BE81280FD3
:1010A000391F4A1F5B1F8091B6079091B707A09127
:1010B000B807B091B90779018A01E81AF90A0A0B51
:1010C0001B0BD801C701E981FA8180879187A2872C
:1010D000B3878B85992781709070882339F0E981D7
:1010E000FA8114821582168217820AC0E981FA8178
:1010F0008B819C81AD81BE8184839583A683B783D8
:10110000E981FA818F81988595878487E981FA81C1
:1011100089859A859787868789819A812B960FB6CC
:10112000F894DEBF0FBECDBFDF91CF911F910F911D
:10113000FF90EF9008950F93CF93DF93CDB7DEB775
:101140002B970FB6F894DEBF0FBECDBF6B837C83A9
:101150008D839E8358874F833A8729870B872985FC
:101160003A854F8158858B819C81AD81BE810B85ED
:10117000BC01CD010E9425889A83898389819A8147
:10118000009721F089819A810E948A8689819A81BB
:101190002B960FB6F894DEBF0FBECDBFDF91CF9177
:1011A0000F9108950F93CF93DF93CDB7DEB72997B3
:1011B0000FB6F894DEBF0FBECDBF69837A838B83F1
:1011C0009C835E834D8338872F83098789819A8129
:1011D000AB81BC81BC01CD010E94C490DC01CB017C
:1011E0002F8138854D815E810985BC01CD010E942A
:1011F0009B8829960FB6F894DEBF0FBECDBFDF9156
:10120000CF910F910895EF92FF920F93CF93DF93B9
:10121000CDB7DEB724970FB6F894DEBF0FBECDBFB3
:1012200069837A838B839C8389819A81AB81BC811A
:101230000097A105B10509F44FC08DE498E0209115
:101240004F0830915008BC01C9010E941784E091F9
:101250004F08F091500883E08787E0904F08F090A6
:10126000500820914F083091500842E055E889819C
:101270009A81AB81BC8101E0BC01CD010E94D28882
:10128000F701968B858BF70185899689009719F070
:101290000E94898423C0E0914F08F09150088DE4AA
:1012A00098E0908F878BE0914F08F09150088091E3
:1012B0004D0890914E0893838283E0914F08F091FE
:1012C000500881E0878780914F0890915008909353
:1012D0004E0880934D0802C00E94298524960FB6BF
:1012E000F894DEBF0FBECDBFDF91CF910F91FF907D
:1012F000EF900895CF93DF93CDB7DEB724970FB665
:10130000F894DEBF0FBECDBF9C838B838B819C8105
:101310009A838983E981FA8182819381009761F0C0
:10132000E981FA81A281B381E981FA818081918189
:1013300011969C938E9308C0E981FA8180819181F6
:101340009093540880935308E981FA8180819181B8
:10135000009739F1E981FA81A081B181E981FA81AF
:1013600082819381FD0193838283E981FA81608187
:101370007181E981FA810190F081E02D208531852C
:1013800042855385E981FA8180859185A285B3855F
:10139000820F931FA41FB51FFB0180879187A2872F
:1013A000B38789819A810E946A8224960FB6F89445
:1013B000DEBF0FBECDBFDF91CF910895CF93DF93F6
:1013C000CDB7DEB724970FB6F894DEBF0FBECDBF02
:1013D0000FB6F8940F928091550890915608A091FD
:1013E0005708B091580889839A83AB83BC830F90C8
:1013F0000FBE89819A81AB81BC81BC01CD0124964D
:101400000FB6F894DEBF0FBECDBFDF91CF91089528
:10141000EF92FF920F931F93CF93DF93CDB7DEB779
:101420000E94DE897B018C010E94B7909B01AC0178
:10143000C801B7010E94F3F1DA01C901BC01CD0175
:10144000DF91CF911F910F91FF90EF900895AF9290
:10145000BF92CF92DF92EF92FF920F931F93CF93A1
:10146000DF93CDB7DEB728970FB6F894DEBF0FBE77
:10147000CDBF0E94DE89DC01CB018D839E83AF83CB
:10148000B8870E94B7909B01AC018D819E81AF818E
:10149000B885BC01CD010E94F3F1DA01C90189834D
:1014A0009A83AB83BC830E94B790DC01CB01298176
:1014B0003A814B815C81BC01CD010E94A1F19B016D
:1014C000AC018D819E81AF81B885821B930BA40BEB
:1014D000B50B8D839E83AF83B88789819A81AB8159
:1014E000BC8128EE33E040E050E0BC01CD010E9419
:1014F000A1F15B016C018D819E81AF81B88528EEE1
:1015000033E040E050E0BC01CD010E94A1F17B013D
:101510008C010E94B7909B01AC01C801B7010E94E9
:10152000F3F1DA01C9018A0D9B1DAC1DBD1DBC0183
:10153000CD0128960FB6F894DEBF0FBECDBFDF9168
:10154000CF911F910F91FF90EF90DF90CF90BF90C0
:10155000AF900895CF93DF93CDB7DEB728970FB63E
:10156000F894DEBF0FBECDBF9E838D8378876F83D7
:101570008F8198859A8389830FB6F8940F92E981B9
:10158000FA81808191819C838B830F900FBE8B8128
:101590009C812FEF8F3F920709F45DC057C0EB810C
:1015A000FC81258936898D819E812817390709F0AC
:1015B00042C00FB6F8940F92EB81FC818281938137
:1015C000E981FA8191838083EB81FC81848195811B
:1015D0000097E1F0EB81FC8182819381009761F0BB
:1015E000EB81FC81A281B381EB81FC8184819581B7
:1015F000FD019583848306C0E981FA818FEF9FEF17
:1016000091838083EB81FC81158214820F900FBE41
:10161000EB81FC8182E087878DE498E02B813C811F
:10162000BC01C9010E948583EB81FC818FEF9FEF94
:10163000968B858B10C08B819C8102969A838983BF
:10164000EB81FC81828193819C838B838B819C8144
:10165000009709F0A4CF28960FB6F894DEBF0FBE0E
:10166000CDBFDF91CF910895EF92FF920F93CF936B
:10167000DF93CDB7DEB72A970FB6F894DEBF0FBE63
:10168000CDBF9C838B834D835E836F8378870FB63A
:10169000F8940F92EB81FC81808191819A838983F8
:1016A0000F900FBE89819A812FEF8F3F920771F4BF
:1016B0000FB6F8940F92EB81FC81118210820F908B
:1016C0000FBE0E9429851A86198656C08DE498E0BF
:1016D00020914F0830915008BC01C9010E94178425
:1016E0008B819C8120914F0830915008BC01C90129
:1016F0000E948583E0914F08F091500883E087872E
:101700008D819E81AF81B8850097A105B105A9F0B3
:10171000E0904F08F09050082B813C814AEA5AE84B
:101720008D819E81AF81B88501E0BC01CD010E9411
:10173000D288F701968B858B06C0E0914F08F09117
:101740005008168A158A0E948984E0914F08F0910A
:10175000500885899689FFEF8F3F9F0759F4E091E4
:101760004F08F0915008168A158A8FEF9FEF9A87DD
:10177000898702C01A86198689859A852A960FB6A6
:10178000F894DEBF0FBECDBFDF91CF910F91FF90D8
:10179000EF900895CF93DF93CDB7DEB726970FB6BE
:1017A000F894DEBF0FBECDBF9A8389834B835C83E1
:1017B0006D837E830FB6F8940F92E981FA81808160
:1017C00091812FEF8F3F920721F4E981FA811182F5
:1017D00010820F900FBE8B819C81AD81BE812981CB
:1017E0003A81AC01BD01C9010E94348B26960FB627
:1017F000F894DEBF0FBECDBFDF91CF910895CF9398
:10180000DF93CDB7DEB726970FB6F894DEBF0FBED5
:10181000CDBF9C838B830FB6F8940F92EB81FC8134
:10182000808191819A8389830F900FBE89819A81EB
:101830002FEF8F3F920709F460C089819A8100974A
:1018400009F450C00FB6F8940F92E981FA818281B1
:101850009381EB81FC8191838083E981FA8184818A
:1018600095810097E1F0E981FA8182819381009767
:1018700061F0E981FA81A281B381E981FA818481F1
:101880009581FD019583848306C0EB81FC818FEFF8
:101890009FEF91838083E981FA81158214820F90F2
:1018A0000FBEE981FA8185899689009751F0E98117
:1018B000FA81858996890E947A89E981FA81168A56
:1018C000158AE981FA8182E087878DE498E0298191
:1018D0003A81BC01C9010E94858381E090E09E832A
:1018E0008D830DC00FB6F8940F92EB81FC818FEFC2
:1018F0009FEF918380830F900FBE1E821D828D818A
:101900009E8126960FB6F894DEBF0FBECDBFDF9145
:10191000CF910895CF93DF93CDB7DEB724970FB65D
:10192000F894DEBF0FBECDBF9C838B838B819C81DF
:101930000E94FF8B9A8389830E94298589819A81DD
:1019400024960FB6F894DEBF0FBECDBFDF91CF91C6
:101950000895CF93DF93CDB7DEB726970FB6F894EF
:10196000DEBF0FBECDBF9E838D831C821B820FB650
:10197000F8940F92ED81FE81808191819A83898311
:101980000F900FBE89819A812FEF8F3F920751F4FC
:101990000FB6F8940F92ED81FE81118210820F90A4
:1019A0000FBE24C089819A81009701F18D819E81AB
:1019B0000E94FF8B9C018B819C81820F931F9C83D3
:1019C0008B830FB6F8940F92ED81FE818081918117
:1019D0009A8389830F900FBE89819A81009731F095
:1019E00089819A812FEF8F3F920701F78B819C812C
:1019F00026960FB6F894DEBF0FBECDBFDF91CF9114
:101A00000895CF93DF93CDB7DEB724970FB6F89440
:101A1000DEBF0FBECDBF9C838B838B819C810E94D8
:101A2000A98C9A8389830E94298589819A81249629
:101A30000FB6F894DEBF0FBECDBFDF91CF910895F2
:101A4000CF93DF93CDB7DEB724970FB6F894DEBF00
:101A50000FBECDBF9C838B838091BA079091BB074B
:101A60009A83898313C089819A819C012E5F3F4F9D
:101A70008B819C81BC01C9010E943EF1009751F00D
:101A8000E981FA81808191819A83898389819A8110
:101A9000009749F789819A8124960FB6F894DEBFA2
:101AA0000FBECDBFDF91CF910895CF93DF93CDB718
:101AB000DEB727970FB6F894DEBF0FBECDBF9C836D
:101AC0008B837E836D834F838FEF9FEF9A83898310
:101AD0008B819C810097C1F18D819E81009731F0AF
:101AE000EB81FC818D819E81958784878F818823FE
:101AF00021F0EB81FC818F8186878B819C8102960E
:101B00000E94208D009701F5EB81FC8183899489E7
:101B1000009751F0EB81FC810388F489E02D8B81E3
:101B20009C810995009781F48091BA079091BB0739
:101B3000EB81FC81918380838B819C819093BB0797
:101B40008093BA071A82198289819A8127960FB6E3
:101B5000F894DEBF0FBECDBFDF91CF910895CF9334
:101B6000DF93CDB7DEB722970FB6F894DEBF0FBE76
:101B7000CDBF89E598E043E150E0BC0180E090E012
:101B80000E9430A1009729F08FEF9FEF9A838983FD
:101B900013C080915908833141F480915A088F34E1
:101BA00021F480915B08833529F08FEF9FEF9A83B2
:101BB000898302C01A82198289819A8122960FB67E
:101BC000F894DEBF0FBECDBFDF91CF910895CF93C4
:101BD000DF93CDB7DEB722970FB6F894DEBF0FBE06
:101BE000CDBF83E1809359088FE480935A0883E541
:101BF00080935B0889E598E043E150E0BC0180E018
:101C000090E00E9454A1009729F08FEF9FEF9A83F4
